:020000040800F2
:10200000005000207D900008799000087990000829
:10201000799000087990000879900008000000008D
:10202000000000000000000000000000799000089F
:10203000799000080000000079900008799000086D
:10204000799000087990000879900008799000084C
:10205000799000087990000879900008799000083C
:10206000799000086D510008799000087990000877
:10207000799000087990000879900008799000081C
:10208000799000087990000879900008799000080C
:1020900091940008799000087990000879900008E0
:1020A00079900008799000087990000879900008EC
:1020B00079900008799000087990000879900008DC
:1020C00079900008799000087990000879900008CC
:1020D00079900008799000087990000879900008BC
:1020E00079900008799000087990000800000000BD
:1020F00000000000000000000000000000000000E0
:1021000000000000000000005FF808F10348044BE5
:10211000834202D0034B03B118477047840100206B
:10212000840100200000000005480649091A8910B2
:1021300001EBD171491002D0034B03B1184770472E
:1021400084010020840100200000000010B5064C2E
:10215000237843B9FFF7DAFF044B13B10448AFF318
:1021600000800123237010BD8801002000000000C2
:102170009400010808B5044B1BB104490448AFF3AF
:102180000080BDE80840CFE7000000008C0100207F
:1021900094000108A3F5803A704700BF154B002B4F
:1021A00008BF114B9D46FFF7F5FF00218B460F46F8
:1021B0001148124A121A09F053FE0C4B002B00D0A2
:1021C00098470B4B002B00D09847002000210400BB
:1021D0000D000B4809F0DCFD09F00EFE200029007F
:1021E00003F05AFC09F0DAFD0000080000000000CE
:1021F000000000000000000088010020741600208C
:10220000C5BD000870B51F24104E114D3168284619
:10221000E14011F0010118BF012103F0D7F80C488B
:1022200003F09DF901210A4803F0C8F8084803F0BB
:1022300096F90021064803F0C1F814F1FF34E5D205
:102240000021BDE87040024803F0C0B84002002001
:10225000BC08002010B5074C0121204603F0CAF845
:10226000204603F07CF92046BDE81040002103F031
:10227000C1B800BFBC08002010B50446FFF7C2FF7C
:102280001CB1BDE81040FFF7E5BF10BDF8B504462E
:10229000082540F2471626FA05F111F0010118BF92
:1022A0000121204603F092F8204603F058F901215D
:1022B000204603F083F8204603F051F90021204620
:1022C00003F07CF815F1FF35E5D20021204603F03C
:1022D0007DF80121204603F08DF8204603F03FF9F8
:1022E000112600250121204603F068F8204603F05E
:1022F00036F9112E06F1FF3706D02EB1204603F035
:102300006DF8B8400543ADB20021204603F056F801
:10231000204603F024F97B1C3E46E3D120460021F1
:1023200003F068F805F07F00C5F3C315062D8EBFD6
:102330000023044B5B5D18444010C0F1820080B262
:10234000F8BD00BF8CC4000800232DE9F3418DF8CF
:102350000730037A0446002B48D003F067F8474B58
:1023600005461A68904241D0454E18603378002BDC
:102370003FD1002871D1DFF81C8198F80030EBB113
:10238000404F3B78D3B93378C3B1BDB920461A2149
:1023900003F0E2F80121204603F02CF800BF00BF53
:1023A00000BF2946204603F025F82946204603F0C1
:1023B0000DF8012388F8005035703B70236D324AC8
:1023C00001332365136801331360B4F85430226C71
:1023D00001339BB2A4F8543044F61F639A4284BF81
:1023E00000232364236C0BB10133236402B0BDE8E6
:1023F000F0810028BFD1234F244A0DF1070104F1D9
:10240000200000F04BFE3A7882F001023A709DF80D
:10241000072002B30121DFF88080204603F012F884
:1024200098F80030002BA6D000BF00BF00BF0121EC
:10243000204602F0DFFF00BF00BF00BF00212046A2
:1024400002F0D8FF0021204602F0C0FF002388F8E8
:1024500000303B708FE72946DDE70D4B1B78002BE2
:1024600089D1204602F0D6FF084B01468DF80700BF
:102470001A7804F10C0000F0CBFD7CE7040000208A
:102480002B0E002008000020240E00201D0E00202E
:10249000200E0020660200206702002010B50446CE
:1024A000012103F021F8094B1A68094B1A60FFF764
:1024B000A9FE0121204602F06BFF0122054B1A7094
:1024C000204602F0B3FF0028FAD110BD4C020020D4
:1024D000400200206702002038B50C460546002166
:1024E00003F002F8094B20461A68094B1A60FFF7FF
:1024F000C3FE0021284602F04BFF34B90122054BF0
:102500001A701A780AB100BFFBE738BD48020020F4
:1025100040020020660200202DE9F04F612985B0BD
:1025200004460E461546DFF88883C14F04D00629BD
:1025300000F01382BF4B1970D8F800203968BE48EC
:1025400002F066FB6DB10021204602F05BFF2046E1
:1025500002F0FEFF2046012102F054FF204602F067
:10256000F7FFD8F800A0B54BB54A53449342DFF8C3
:102570004493B44B00F28A80B34AC9F80020012288
:102580001A601D683868012D14BF01220222AF4B6A
:10259000A0F5C3301A60A03808F07AFD012D40F094
:1025A00087809FA3D3E9002308F016FF09F0A4F861
:1025B000029008F0EDFB09F0C3FB5FFA80FB84F8A2
:1025C00000B0584609F0A2F9029B0146184609F0EE
:1025D000E7F84FF08E4109F0EDF908F07BFD00229D
:1025E0009B4B08F019FC08F04FFB09F065F880B22E
:1025F00060800001974B40EACB4040F0904018606B
:10260000504608F045FD012D56D185A3D3E900239E
:1026100008F0E2FE09F070F8834608F0B9FB09F013
:102620008FFB5FFA80FA84F804A0504609F06EF937
:102630000146584609F0B4F84FF08E4109F0BAF956
:1026400008F048FD824B002208F0E6FB08F01CFB76
:1026500009F032F880B2E080000140EACA407E4BC7
:1026600040F08040042E186000F04E8128D8022EE1
:1026700000F0D08000F22881012E00F0BD804FF0E4
:10268000000AD3465346524655463DE0734A7449C4
:1026900052448A427FF670AF724A734952448A426A
:1026A00001D9724A69E7724AC9F80020022267E735
:1026B0005DA3D3E9002377E75BA3D3E90023A7E772
:1026C000062E14D0C0F02D81072E00F03881612E27
:1026D000D5D1684B1B78B3FBF5F540F29D3A664BBC
:1026E000DFF8D4B143EAC545644B654A0CE0654B5D
:1026F0004FF00D0A1B88DFF8C4B1B3FBF5F5624A51
:10270000ED04624B45F00055D9F80010DFF8B091A8
:10271000CDE90223C9F80010FFF774FDFFF79AFD19
:10272000029AC9F80020FFF76DFDFFF793FD039BA8
:10273000C9F80030FFF766FDFFF78CFD544BC9F870
:102740000030FFF75FFDFFF785FD42F2F543C9F862
:102750000030FFF757FDFFF77DFD204602F0F4FE45
:1027600001212046FFF7B8FE4A4B1B7845EA433566
:1027700045F4C45545F00205C9F80050FFF742FD85
:10278000FFF768FD0E23C9F80030FFF73BFDFFF7A8
:1027900061FD414BC9F80030FFF734FDFFF75AFDEA
:1027A000C9F800B0FFF72EFDFFF754FD3B23C9F831
:1027B0000030FFF727FDFFF74DFD4FF48673C9F892
:1027C0000030FFF71FFDFFF745FDC9F800A0FFF738
:1027D00019FDFFF73FFD314BC9F80030FFF712FD3F
:1027E000FFF738FD062E04D1009BC8F80030019B8E
:1027F0003B6005B0BDE8F08F294B4FF00D0A1B88F8
:10280000DFF8C0B0B3FBF5F5ED0445F01005254B3E
:10281000254A79E7254B1B885DE700BFAFF30080B1
:102820000000000000203C410000000000204C415E
:1028300074020020290E0020BC08002000BC6AF7AA
:10284000FF083D005002002041501F0254020020AA
:102850000000E03F480200204C0200204053F2F20A
:102860007F8D5B008019D0CDFFF26F06415057007D
:1028700041505300150000207000002034270685C9
:10288000D3804C2A6202002093004F2A845A16807B
:10289000160E070580020020E93102000F000E002D
:1028A0005A020020942AA80093414C2A5802002082
:1028B00078020020440200202A479E043A479614DA
:1028C000400200203A47960C94F834302849002BF7
:1028D00008BF4FF40121274B274A08BF1A46274B50
:1028E00018BF4FF4187A43EA0103254908BF4FF493
:1028F000966A09884AF00D0AB1FBF5F52149DFF81F
:10290000A8B041EAC545FFE61F4B40F2FD2A1B88EF
:10291000DFF894B0B3FBF5F51A4B43EAC5451B4B02
:10292000E3E61B4B40F2AD1A1B88DFF87CB0B3FB2B
:10293000F5F5144B174A43EAC545174BE4E6174B28
:1029400040F2BD3A1B88DFF860B0B3FBF5F50D4BE4
:10295000084A43EAC545124BD6E6D8F80030009342
:102960003B6801930F4B1B68C8F800303B60E3E500
:102970000024060093C04C2AD3804C2A34034081A3
:10298000640200207000002060020020342B6600EA
:102990005E02002013C14C2A349F74005C020020A8
:1029A000343B79807C0200202A479E04014B890831
:1029B00019707047800200202B2041431648C90936
:1029C00010B5018017214A439DF818401349D209D8
:1029D0000A80FCB1DB08124A138016239DF80820F8
:1029E0005343104ADB0913800D239DF80C205343F9
:1029F0000D4ADB0913801C239DF8102053430B4A1A
:102A0000DB091380A0239DF814205343084ADB09F7
:102A1000138010BD9B08DEE75A02002058020020F8
:102A200064020020600200205E0200205C020020A0
:102A30006202002000000000F8B54F4C4F4B2168A7
:102A40004F4A0B44934205464E4B4F4E60D84F4A77
:102A50001A600122326002221B684D494D4F0A6004
:102A60003B60FFF7CFFBFFF7F5FB4B4B1B78022BCF
:102A700060D14A4B32681B88B3FBF2F2484B43EA01
:102A8000C243484A127843EA423343F4C45343F002
:102A900002033B60FFF7B6FBFFF7DCFB33682068FF
:102AA000012B55D108F0F4FA2FA3D3E9002308F045
:102AB00093FC08F021FE064608F06AF909F040F997
:102AC000C4B22C71204608F021FF0146304608F0C0
:102AD00067FE4FF08E4108F06DFF08F0FBFA324BB5
:102AE000002208F099F908F0CFF808F0E5FD80B26F
:102AF000E88000012D4B40EAC44040F0804018605F
:102B00002B4B1B7853B32846BDE8F840FFF7C6BCF3
:102B1000284A29480A44824299D9284A0A4428491D
:102B20008A4201D9274A93E7274A1A600222326073
:102B3000012291E7062B03BF244B32681B884FF01C
:102B4000005302BFB3FBF2F3DB0443F0005398E7FA
:102B500008F09EFA06A3D3E90023A8E72846BDE8BB
:102B6000F8400121FFF7B8BC0000000000203C4104
:102B70000000000000204C417802002000BC6AF7F1
:102B8000FF083D00440200205002002041501F0277
:102B90005402002040020020280E0020580200208D
:102BA00070000020800200200000E03F4C02002066
:102BB0002B0E00204053F2F27F8D5B008019D0CDA8
:102BC000FFF26F064150570041505300620200204F
:102BD00038B50278408800EBC23008F097FE08F064
:102BE00079FA00224FF07C5308F0CCFA104B0446DF
:102BF00018680D4608F04CFA02460B460AA1D1E9C6
:102C0000000108F0E9FB08F077FD08F063FA0246DE
:102C10000B462046294608F0B5FA08F04DFD00F5B0
:102C2000C330A03038BD00BF0000000000204C4180
:102C3000540200200000000038B50279C08800EB83
:102C4000C23008F063FE08F045FA00224FF07C53D2
:102C500008F098FA0E4B044618680D4608F018FA6A
:102C600002460B4608A1D1E9000108F0B5FB08F0C7
:102C700043FD08F02FFA02460B462046294608F08D
:102C800081FA08F019FD38BD0000000000204C4119
:102C9000540200200000000038B50F4B188808F0DF
:102CA00007FA0BA3D3E9002308F06CFA0B4B044698
:102CB00018680D46000408F0EBF902460B46204662
:102CC000294608F089FB08F0F7FC80B238BD00BF48
:102CD0000000000000204C415A0200205402002055
:102CE00038B50F4B188808F0E3F90BA3D3E900239C
:102CF00008F048FA0B4B044618680D46000408F02B
:102D0000C7F902460B462046294608F065FB08F045
:102D1000D3FC80B238BD00BF0000000000204C4151
:102D2000580200205402002038B50F4B188808F0D4
:102D3000BFF90BA3D3E9002308F024FA0B4B044698
:102D400018680D46000408F0A3F902460B46204619
:102D5000294608F041FB08F0AFFC80B238BD00BF47
:102D60000000000000204C416402002054020020BA
:102D700038B50F4B188808F09BF90BA3D3E9002353
:102D800008F000FA0B4B044618680D46000408F0E2
:102D90007FF902460B462046294608F01DFB08F045
:102DA0008BFC80B238BD00BF0000000000204C4109
:102DB000600200205402002038B50F4B188808F03C
:102DC00077F90BA3D3E9002308F0DCF90B4B044699
:102DD00018680D46000408F05BF902460B462046D1
:102DE000294608F0F9FA08F067FC80B238BD00BF48
:102DF0000000000000204C415E0200205402002030
:102E000038B50F4B188808F053F90BA3D3E900230A
:102E100008F0B8F90B4B044618680D46000408F09A
:102E200037F902460B462046294608F0D5FA08F045
:102E300043FC80B238BD00BF0000000000204C41C0
:102E40005C0200205402002038B50F4B188808F0AF
:102E50002FF90BA3D3E9002308F094F90B4B044698
:102E600018680D46000408F013F902460B46204688
:102E7000294608F0B1FA08F01FFC80B238BD00BF47
:102E80000000000000204C4162020020540200209B
:102E900038B505462A4C2B49204603F09DFF2846AD
:102EA000FFF7CAFE28490246204604F083FA284666
:102EB000FFF78EFE25490246204604F07BFA244B9C
:102EC00024491A78204604F0A4FA2846FFF7E4FEC5
:102ED000214902B2204604F09CFA2846FFF700FF81
:102EE0001E4902B2204604F094FA2846FFF71CFF60
:102EF0001B4902B2204604F08CFA2846FFF738FF3F
:102F0000184902B2204604F084FA2846FFF754FF1D
:102F1000154902B2204604F07CFA2846FFF770FFFC
:102F2000124902B2204604F074FA2846FFF78CFFDB
:102F30000F4902B22046BDE8384004F06ABA00BF2B
:102F4000C411002093C40008AEC40008BCC400082B
:102F500080020020CAC40008D5C40008E6C40008E6
:102F6000FBC4000810C5000825C500083BC50008C3
:102F700050C5000838B50023CD0883810446C381BD
:102F80000180C0E9013303744374284607F04FFE03
:102F90006060284607F04BFEA060204638BDC1891E
:102FA000838902889BB28B4205D1037C002B0CBF26
:102FB000104600207047C3898189994287BF838961
:102FC000C089C389808986BF8018C01A181A80B248
:102FD000904288BF00207047C28983899BB2934288
:102FE00005D1027C02F0FF0382B100887047C389DB
:102FF00082899A429DBFC2898389008883898BBF59
:10300000C089C018181A801A80B2704718467047D5
:10301000037C30B51BB101234374002030BD83898C
:103020004568DB081C4CEB5C41B3818901F007016A
:10303000615C0B438189C9086B5483898168DB0813
:10304000CB5C12B3828902F00702A25C134382892F
:10305000D2088B548389028801339BB28381838990
:103060009A429CBF002383818289C3899BB2934289
:103070004FF0010308BF03741846CFE7818901F0C0
:103080000701615C23EA0103D4E7828902F00702A9
:10309000A25C23EA0203DAE761C5000870B50346C3
:1030A0008489C08980B2A04203D11C7C04F0FF0057
:1030B0005CB3D8895C68C008205CDE89DC89134D6C
:1030C000E44306F00706AE5D04F0070430402041FB
:1030D0000870D9899868C908415CDC89D88904F0EE
:1030E0000704C0432C5D00F007002140014111702E
:1030F00000211974DA891888013292B2DA81DA89EA
:1031000090424FF0010098BFD98170BD61C50008A1
:1031100003460022407C5A74704700000246002398
:1031200010B522F8023B114600F1240402F8013BDD
:103130009442FBD1074A80F8243083620B4602F1A7
:10314000200152F8044B8A4243F8044BF9D112880B
:103150001A8010BDB5C5000830B50F4DC1EBC101D7
:103160006B185A78047C42749A78695C8274DA78B5
:1031700024F00F04C2741A7901F00F0102755A7914
:103180009B794275827D23F00F0302F00F020C43FE
:103190001A430474827530BD69C5000810B5044631
:1031A0001C4800F0E9FC1B4800F04EFD68B1637854
:1031B000022B0BD0032B23D0012B28D1222216491E
:1031C000144800F08FFC0223637010BD94F82410A3
:1031D0002046FFF7C1FF2222A11C0E4800F082FC0E
:1031E00094F82430052B07D1002384F82430237869
:1031F000002BEAD10323E7E7013384F82430E4E726
:1032000022220649034800F06DFC0023DCE700237E
:103210006370F2E78004002093C50008D7C500085A
:1032200007B51A4A1278622A06D0642A14D05C2A9A
:103230000BD1FFF7B3FF08E0017849B11448012131
:1032400000F080FC124800F097FC03B05DF804FB2E
:103250000F4800F077FCF8E7826A0E4901328A4293
:1032600001D88262F1E7002201A982620DF1060213
:10327000094801F067FFBDF80420BDF90630520887
:103280000649074804F054FBDFE700BF1C0E00208E
:103290008004002001B10100BC080020F9C500082D
:1032A000C4110020012A08B514D10B78012B0CBFE2
:1032B0000122002202700BD1427822B9064A12780C
:1032C0005C2A00D14370012202210448FFF724F94F
:1032D000002000E0042008BD1C0E0020BC080020D7
:1032E00000220260027182604FF6FF72C260704776
:1032F000036813B50133B3F5FA4F0446036029D3CD
:103300001548FEF7C3FF0023E18922798142A18994
:10331000236002F10102A368D2B238BFE08181428A
:10332000034488BFA081052A2271A36012D9E268F4
:10333000694612BA00920622B3FBF2F307485BBA61
:10334000ADF8043003F020FD00232371A3604FF695
:10335000FF73E36002B010BDBC080020C411002060
:103360000246002300F5967102F8013B9142FBD121
:10337000A0F82C31A0F82E3180F8303170470000D1
:103380002DE9F041B0F82C310446002B38D01D480F
:1033900001F034FC05461C4FDFF87480194E0C2DEB
:1033A0002ED9B4F82E313046D91003F00702BA5C9A
:1033B000635C0C3D13401DBF00230C2213490C22FB
:1033C00008BF414601F0F6FB94F83031ADB201334D
:1033D000DBB2272B84F8303107D9B4F82E31013312
:1033E000A4F82E31002384F83031B4F82E21B4F83B
:1033F0002C319A42D3D30023A4F82E31A4F82C31D7
:10340000BDE8F081BC0800201CC8000809000020AD
:10341000680200202DE9F74F0D46924600214FF437
:10342000967208F01DFD0822A0F82C210022034608
:1034300029464FF00C09DFF8B8C0A0F82E2180F81B
:103440003021AA448A453ED00020C2B209FB02F2D4
:103450000CEB02041CF802209AB30D78013095425F
:10346000F3D100264FF0004594F808B00194F0B273
:103470008345B3F82C2124D91A4C02F0070714F81D
:103480000780019C4FEAE20E676813F80E0035EAE8
:1034900007040CBF40EA080020EA0800B2F5937F59
:1034A00003F80E0006F1010606D900220420A3F855
:1034B0002C2103B0BDE8F08F0132A3F82C216D0858
:1034C000D5E70131BEE7B3F82C21082AEDD005324B
:1034D00092B2A3F82C21044812B2044903F099FFD8
:1034E0000020E6E71CC80008C411002024C800081A
:1034F0000CC600080023A0F82C31A0F82E3180F86B
:103500003031704730B50346002400250022E3E83F
:10351000024500F1500103F8012B9942FBD1034B06
:103520004267C0E91E32A0F8802030BD00000F279E
:103530000023044A80F87F30A0F876308267A0F834
:103540007C30704700000F2710B58188036804465F
:10355000294881F45541584081F0D70104F0B0FB6F
:10356000032817D8402384F87C30B4F8743003F271
:10357000A51292B2B2F5107FA4F8763039D2A4F831
:10358000782003F16C0292B2B2F5107F1CD2A4F83D
:103590007A201DE0A1882368184881F457415840DB
:1035A00081F0550104F08CFB0328DBD9A188236846
:1035B000134881F4FE41584081F07D0104F080FB06
:1035C000032809D82023CEE7A3F5EA73A4F87A30BC
:1035D00000220C4B1A6010BDA18823680A4881F4B0
:1035E000FB41584081F07F0104F06AFB0328E9D9D0
:1035F000F1E7A3F19B02C2E757D77FF7F5F75F7FAB
:10360000FD7DD55D240E00205F5DF5D5F0B500276A
:10361000724E1A449A4200F0E0801F7000EBD10411
:1036200001F0070C257A16F80C402540CC4304F035
:1036300007042541ED011D706CB24D1CADB2B5F50E
:10364000107F24BFA1F23F218DB200EBD50105F020
:10365000070C097A16F80CC001EA0C016FEA050C98
:103660000CF0070C41FA0CF144EA8114691C1FFAB2
:1036700081FCBCF5107F24BFA5F23F251FFA85FC15
:1036800064B21C7000EBDC010CF00705097A755D73
:1036900029406FEA0C0505F00705294144EA411469
:1036A0000CF101018DB2B5F5107F24BFACF23F21C2
:1036B0008DB264B21C7000EBD50105F0070E91F8D5
:1036C00008C016F80E100CEA010CE94301F00701DE
:1036D0004CFA01FC691C44EA0C141FFA81FCBCF58D
:1036E000107F24BFA5F23F211FFA81FC64B21C7039
:1036F00000EBDC010CF0070E0D7A16F80E100D40F1
:103700006FEA0C0101F007010D410CF101011FFAF4
:1037100081FEBEF5107F28BFACF23F2144EAC5040C
:1037200028BF1FFA81FE64B21C7000EBDE010EF0B0
:10373000070C0D7A16F80C100D406FEA0E0101F01F
:1037400007010D410EF101011FFA81FCBCF5107F4C
:1037500028BFAEF23F2144EA850428BF1FFA81FC4E
:1037600064B21C7000EBDC010CF0070E0D7A16F849
:103770000E100D406FEA0C0101F007010D410CF134
:1037800001011FFA81FEBEF5107F28BFACF23F2178
:1037900044EA450428BF1FFA81FE64B21C7000EBA6
:1037A000DE010EF0070591F808C0715D0CEA010C0E
:1037B0006FEA0E0101F007014CFA01FC0EF1010164
:1037C00089B244EA0C04B1F5107F03F8014BFFF411
:1037D00021AFAEF23F2189B21CE7F0BD40C800081E
:1037E00080F87E107047000010B508480C46FEF7C0
:1037F0004DFD030A84F8223084F823002246BDE8F8
:10380000104024230121024803F0C8B8BC0800205E
:10381000C411002073B50446B0F874009D4E04EB4B
:10382000D00200F00705137A755D002950D02B43B4
:103830001372D4E90032DB18524100294BD1C4E99C
:10384000003294F87F30002B48D12046FFF77CFEF1
:10385000B4F87420B4F87A309A4270D194F87C307D
:1038600004F1510584F8503021222B46B4F8781029
:103870002046FFF7CBFE94F87C30402B40F0B3801D
:1038800001A800F0F1F90DF107030DF10602294638
:1038900001A800F017FA94F87E209DF806309A42AD
:1038A0004AD1002394F8502084F87D3084F8803089
:1038B0009DF807301A4384F850200A2B00F28F80BD
:1038C000DFE803F072637A8D8D8D2951518D51009F
:1038D00023EA0503ACE743F00103B0E7B4F8761040
:1038E00001F23E239BB2B3F5107F01F1020292B2C6
:1038F00024BF8B1E9BB2B2F5107F24BFA1F23E22E3
:1039000092B2934204D28342A2D88242A0D39CE7CF
:103910008342FAD899E7B4F976205F495F4803F00B
:1039200078FD04F150012046FFF75EFF022384F882
:103930007F30002384F88130002384F87C30B4F891
:10394000743094F87F1001339BB2B3F5107F28BF19
:1039500000230031A4F8743018BF0121504801F051
:10396000D9FB02B070BD94F87F30022BE4D1B4F9DA
:1039700076204C49494803F04CFD04F150012046A3
:10398000FFF732FF9DF80730D4E7B4F976204649B7
:10399000424803F03EFD04F150012046FFF724FFAA
:1039A000012384F87F30C7E794F87F30012BF7D1EB
:1039B000B4F976203D49EBE794F87F30012BBBD179
:1039C000B4F976203A49354803F023FD204604F146
:1039D0005001FFF709FF2046FFF7AAFDACE7B4F955
:1039E00076203449EFE7202B13D1B4F97620324901
:1039F0002A4803F00EFD04F150012046FFF7F4FEC3
:103A0000012384F87F30002384F87D3084F88030EF
:103A100092E794F87F3073B194F87D300133DBB2D4
:103A20000C2B84F87D3006D91C48012102F0E6FFFA
:103A30002046FFF77DFD94F87F30012B18D194F8D4
:103A4000803004F15002042B83BF202384F85030CF
:103A50000023013397BFDBB284F8803084F88030D4
:103A600084F85030012122230C4802F097FF63E7CD
:103A7000022B7FF461AF94F88130002B3FF45CAFF0
:103A8000214643F0400301F8503F2046FFF7ACFECB
:103A900052E700BF40C8000848C80008C411002011
:103AA000BC08002068C8000889C80008AAC8000827
:103AB000CEC80008F3C800080CC9000810B540F2D1
:103AC0006B31044604F008F8002204F1100304F1FD
:103AD000600103F8012B9942FBD1F0232266636653
:103AE000204610BD222A70B506460C460ED104F0C1
:103AF00006F820280CD904F1210514F8011F3046DE
:103B000004F036F8AC42F8D1002070BD0420FCE788
:103B10000520FAE773B50D460824094EEB098DF828
:103B20000730012200230DF107013046013C01F06E
:103B300041F86D0014F0FF04EDB2EFD102B070BD9A
:103B4000BC08002080F8671070470000094B1B7804
:103B5000622B0BD15F2100F1100300F1310203F859
:103B6000011B9342FBD12123A0F860300023A0F871
:103B7000623070471C0E002070B590F86730044624
:103B8000B0F8605053B305B32C4801F037F8054640
:103B9000082D22D9B4F8623094F866105A1C92B2FB
:103BA000A4F86220002945D05F212046FFF7B2FF2C
:103BB000B4F86220B4F86030083D9A42ADB2E7D361
:103BC0000023236684F8663007E080F86650FFF72C
:103BD000BDFFB4F86030002BD6D170BD002DD3D11D
:103BE00003F0AAFF0028F4D0154B1B7853B901232A
:103BF00084F86630B4F86430A4F860300023A4F888
:103C00006230E6E784F8665004F1310604F11005ED
:103C1000204603F0D0FF05F8010BB542F8D1094B5F
:103C200004F1580213F8011B05F8011BAA42F9D14F
:103C30004823E1E72344197CB7E700BFBC08002014
:103C40002B0E00202BC9000808B503F058FF2323D2
:103C5000B0FBF3F080B208BD01EB4101890001F532
:103C60001671A0F86410704770470000B1F5006F3E
:103C700010B50DD34FF4802340F6754405480B4230
:103C800001D15B08FBE7DA0A624351400142F6D1F9
:103C9000084610BD00F8FFFF10B54C780B78E40023
:103CA00004EBC3248B7804EB53142146FFF7DEFFAB
:103CB000034B53F820006040C0F3C72010BD00BF85
:103CC00054C9000873B51E464B7B0C7B15469A09F8
:103CD00042EA84020C7DC97C9B00890023F03F03EB
:103CE00001F03C01194341EA9411A4008DF805103C
:103CF00024F00F0401A98DF804208DF80640FFF789
:103D0000CBFF030900F00F002B70307002B070BDC4
:103D100002F00F0242EA0111C8B2197B124A21F0E7
:103D20003F0141EA900130B532F810401973597BD8
:103D3000E5B2AA0801F00F0141EA801102F030005B
:103D400001435973D97C02F00F0221F00F01114396
:103D50001A7DA40A02F0030242EA851204F03C0430
:103D60002243D9741A7530BD54E9000830B50024D7
:103D700000250023C0E90245037000F1100200F1A4
:103D8000740102F8013B9142FBD10021C0E91D33CF
:103D9000C0E91F33C0E92133C0F88C3000F59C72B4
:103DA00000F1900343F8041B9A42FBD1002100F577
:103DB000F07342F8041B9342FBD1002100F52272FC
:103DC00043F8041B9A42FBD1002100F54C7342F8E2
:103DD000041B9342FBD1002100F25A3203F8011B6D
:103DE0009A42FBD130BD30B500230024002503707A
:103DF000C0E90245C0E91D3330BD00002DE9F047A0
:103E00000B68D0F88070D0F8886007EB03080B6966
:103E1000C46F06EB030EF045C446A8BFF446F04558
:103E2000B4BFDFF8D4E0DFF8D4E04FEAD40300EB0E
:103E3000830304F00702D3F89050B5BF1EF802E0E8
:103E40001EF802E00EEA05054EEA0505C3F890509B
:103E50004D682F444D69BE462E44B742A8BFB646B2
:103E6000B742B4BF244E254ED3F83851B5BFB65C27
:103E7000B65C35403543C3F83851D0F884808D683E
:103E80008F6908EB050AD0F88C50D3F8E06105EB98
:103E90000709CA455746A8BF4F46CA45B5BFDFF810
:103EA0005890DFF8589019F8029019F80290B4BFB2
:103EB00009EA060649EA0606C3F8E061CE68C96960
:103EC00046440D44AE42B046A8BFA846AE42D3F821
:103ED00088120CDA084DAA5C0A40C3F88822013423
:103EE000C0E920CEC0E92278C467BDE8F087034D61
:103EF000AA5C0A43F1E700BF54ED00085CED00083E
:103F000070B5D1E9003283F0010588B0D11882F094
:103F100001062A44334400917419CDE9051269461B
:103F200001940293CDE903240793FFF767FF08B0DC
:103F300070BD0000002240F249111346F0B5264C36
:103F4000264E032B19D8DFE803F0021C303CCD10BD
:103F500001F007032435E75C50F825303B4018BFDB
:103F6000022300EBD20702F00705755D97F830C316
:103F700005EA0C0587F83053013211F1FF31E0D228
:103F8000F0BDCD1001F007034E35E75C50F8253049
:103F90003B4018BF022300EBD20702F00705655D26
:103FA00097F830C345EA0C05E4E7CB10783301F00D
:103FB000070550F82330655D1D420CBF0123032324
:103FC000CFE7CD10A23501F00707E75D50F8255087
:103FD0002F4208BF0123DEE75CED000854ED000826
:103FE0004FF0FF3230B5104D481E01F1260410F895
:103FF000013F5340DBB235F81330C2F30722534080
:1040000084421A46F3D1DB4391F827009BB2DAB21F
:10401000904207D191F82820B2EB132F0CBF01205A
:10402000002030BD0020FCE754EB00082DE9F043F0
:1040300016460546884899B04B1E01F1520413F804
:10404000017F10F8012B9C4282EA07021A70F6D118
:104050000023184603AA0133542B02F8010BFAD1AE
:10406000DFF8FCE10022744680270EEB4200B2F537
:10407000257F56DB00244FF080084027C5E9204407
:10408000C5E92244EC6718AB03EBE40313F8542CA6
:1040900004F0070328FA03F1114227FA03F314BFCF
:1040A00001210021134214BF01230023029128465D
:1040B00001A902340193FFF723FFB4F5257FE2D174
:1040C000FFF738FF0021731E06F1280203F8011FD5
:1040D0009A42FBD140F24912012710465F4C05EB92
:1040E000E20102F0070E91F830C314F80E10831AA3
:1040F0001CEA010F09D0D90816F801C003F0070324
:1041000007FA03F343EA0C03735412F1FF32E6D2C9
:1041100031462846FFF764FF19B0BDE8F0831A4620
:10412000A5E7D31011F803C01CF0010F0CD090F8D4
:10413000008018AB9844437818F8549C27FA03F38E
:1041400043EA090308F8543C1CF0020F0CD090F825
:10415000028018AB9844C37818F8549C27FA03F3EC
:1041600043EA090308F8543C1CF0040F0CD090F803
:10417000048018AB9844437918F8549C27FA03F349
:1041800043EA090308F8543C1CF0080F0CD090F8DF
:10419000068018AB9844C37918F8549C27FA03F3A7
:1041A00043EA090308F8543C131DB3F5257F00F1D9
:1041B0000800B4DA1CF0100F0FD014F813000DF142
:1041C000600804EB430340445B7810F8548C27FAF2
:1041D00003F343EA080300F8543C1CF0200F10D00E
:1041E000531D14F813000DF1600804EB4303404421
:1041F0005B7810F8548C27FA03F343EA080300F8BD
:10420000543C1CF0400F10D0931D14F813000DF116
:10421000600804EB430340445B7810F8548C27FAA1
:1042200003F343EA080300F8543C1CF0800F10D05D
:10423000D31D14F813000DF1600C04EB430360442C
:104240005B7810F854CC27FA03F343EA0C0300F828
:10425000543C083209E700BF74ED00085CED00082B
:10426000CFED000810B508480C46FEF70FF8030A1A
:1042700084F82A0084F829302146BDE810402B221A
:10428000024802F0F7BA00BFBC080020C4110020A9
:1042900070B5D0E90232DB185241C0E90232426FF8
:1042A000044600EBD2068CB0307C02F0070591B3D7
:1042B00043F00103A3601A4B5B5D18430132B2F572
:1042C000487F3074626702D92046FFF78CFD636F28
:1042D000B3F5257F1BD104F1100501AA294620461C
:1042E000FFF7A4FEA8B101210E4800F013FF01A9B9
:1042F0002046FFF7B7FF0E220021284607F0B0FD49
:1043000000236367022323704FF41653A3670CB096
:1043100070BD2070FBE7044B5B5D1840CEE700BF2B
:104320006CED0008BC08002064ED000810B50748DB
:104330000C46FDF7ABFF030A607323732146BDE80B
:1043400010400E22024802F0C1BA00BFBC08002093
:10435000C411002070B5D0E90232DB180446524186
:1043600071B90025C4E90232A068294680F0AA305C
:1043700003F0A6FC022806D8244B1D60257070BDF2
:1043800043F00103EDE7A068294620F07F43204871
:10439000584003F095FC02280DD81E491E4802F033
:1043A0001BFD5322294604F1100007F059FD01239B
:1043B00065672370E3E7A068294620F07F4317482C
:1043C000584003F07DFC06460028D8D11449124815
:1043D00002F002FD0121134800F09CFE124A04F194
:1043E000100513682946236153682046636193686A
:1043F000A361FFF79BFF0E223146284607F030FDF0
:104400004FF416536667A3670223D2E7240E0020F9
:10441000507655004BF30008C411002068B4AA0080
:1044200074F30008BC080020F7F20008F8B5D0E9E2
:104430000232DB185241C0E90232426F044600EBFF
:10444000D206307C02F00705002900F08B8043F093
:104450000103A360454B5B5D18430132B2F5487F11
:104460003074626702D92046FFF7BDFCA189A368BA
:104470003F4881F42A41584081F0AA0103F020FC12
:1044800001280DD83B493C4802F0A6FC00213B48DE
:1044900000F040FE384802F063FA00232370F8BDB4
:1044A000636F5C2B04D8636F602B22D000230FE076
:1044B000A068002120F07F433148584003F000FC01
:1044C0000328F0D84FF416536022C4E91D230123BA
:1044D000A56F013DA56725BB2A49274802F07CFC52
:1044E0002946264800F016FE234802F01BFA2570E4
:1044F000D5E701256FF07F46214FA06826FA05F326
:10450000034027FA05F05840002103F0D9FB0328A7
:1045100003D8636F5D1B6567C8E70135042DECD1D7
:10452000C4E7626F602ABAD104F11005A3B1552324
:10453000637641F22D63294663832046FFF7F6FE3A
:1045400001210E4800F0E6FD0E220021284607F06A
:1045500087FC00236367A2E70C222946064802F085
:10456000B5F9EDE7084B5B5D184076E76CED0008A8
:104570005E13AAAA03F30008C4110020BC0800209F
:1045800068B4AA0023F3000864ED00080378012B47
:1045900005D013B1022B04D07047FFF7DBBEFFF745
:1045A00077BEFFF743BF10B54FF47A71044603F0AE
:1045B00093FA002304F1100204F16A0102F8013BAE
:1045C0009142FBD14FF47012A4F86A30E26684F88D
:1045D0007030204610BD0000292A70B506460C46F2
:1045E00019D103F08CFA292806D802B20B490C48DD
:1045F00002F00FFF052070BD0021304603F0B8FA2D
:10460000651E283415F8011F304603F0B1FAA542A3
:10461000F8D10020EFE70420EDE700BF27F90008FC
:10462000C41100200C2A70B506460C4619D103F0BF
:1046300066FA0C2806D802B20B490C4802F0E9FED3
:10464000052070BD0121304603F092FA651E0B343F
:1046500015F8011F304603F08BFAA542F8D100206F
:10466000EFE70420EDE700BF64F90008C411002063
:1046700010B5044603F043FA024628B90548064936
:1046800002F0C7FE052010BD0221204603F070FA9B
:104690000020F8E7C411002047F90008501E2DE95A
:1046A000F04F0346002499B003AD02F1520903F81C
:1046B000014F994505F8014BF9D14B1E009300239A
:1046C0001D461C46DFF8B8A10099AC4611F8016FF1
:1046D0002546CDE9001600271E46012101FA07F400
:1046E0000199214214BF0124002404EB0C0EAC44B8
:1046F000A4441CF0010F0EF0010E0CD006F0070CC4
:1047000018A91AF80C8001EBD60C1CF854BC48EA26
:104710000B080CF8548CBEF1000F0ED006F1010C02
:1047200018A901EBDC0E0CF0070C1EF8548C1AF8DB
:104730000CC04CEA080C0EF854CC0137082F06F1D7
:104740000206AC4640F088801033B3F5287FBBD119
:10475000DFF830C10023644601250CEB4301B3F5BB
:10476000257F7DD218AE06EBD30616F8546C3706BB
:104770000AD591F800E04F7812F80E8005FA07F795
:1047800047EA080702F80E7077060AD591F802E0AA
:10479000CF7812F80E8005FA07F747EA080702F803
:1047A0000E70B7060AD591F804E04F7912F80E8022
:1047B00005FA07F747EA080702F80E70F7060AD568
:1047C00091F806E0CF7912F80E8005FA07F747EA6C
:1047D000080702F80E701F1DB7F5257F01F10801CB
:1047E0003CD231070BD514F817E004EB4707797872
:1047F00012F80E7005FA01F1394302F80E10710734
:104800000CD5591D14F8117004EB4101497812F8C8
:1048100007E005FA01F141EA0E01D155B7070CD5C1
:10482000991D14F8117004EB4101497812F807E062
:1048300005FA01F141EA0E01D155F1070AD5D91D5A
:1048400014F8116004EB41014978975D05FA01F114
:1048500039439155083380E725463EE73B467EE7DE
:10486000064A10F8011F12F8013B484583EA01038C
:104870000370F6D119B0BDE8F08F00BFA4F30008B3
:104880009CF30008FFF30008F7B50F460824012544
:104890000B4E35EA07030CBF0123002301228DF8DC
:1048A00007300DF1070100233046013C00F082F98A
:1048B0006D0014F0FF04EDB2EBD103B0F0BD00BF0A
:1048C000BC080020F0B5A3B0044603F035F918B9D0
:1048D000B4F86A30002B49D0204603F067F9B4F8E9
:1048E0006A3000283BD1002B43D1564A12783AB99E
:1048F000012384F87030B4F86E30A4F86A302AE0EE
:1049000084F87030204601AE03F055F9292537466A
:10491000204603F050F96B1E13F0FF0506F8010B5B
:10492000F6D1394620460DF13202FFF7B7FE4AF2C2
:10493000EA63ADF830302B46B4F86A100CA8CA18F8
:1049400010F8015B92B201332244552B1574F6D155
:104950005531A4F86A100023A4F86C3003E0012854
:1049600006D0022840D0B4F86A3013B923B0F0BDA5
:104970001BB3354800F042F90546082DF6D9B4F8C6
:104980006C3094F870105A1C92B2A4F86C20002974
:1049900054D0AA212046FFF777FFB4F86C20B4F872
:1049A0006A30083D9A42ADB2E7D30023A4F86C30D8
:1049B000A4F86A3084F87030D8E784F87030204664
:1049C00003F0F9F80C25B4F86A602046731CA4F8CB
:1049D0006A3003F0F0F8013D264415F0FF0530740D
:1049E000F1D1A4F86C50BEE7002BC2D184F870302E
:1049F000204603F0E0F8C82655217A25B4F86A303D
:104A000003F1120080B2E21811745A1C92B22244CF
:104A100011749A1C92B222441174DA1C92B222448C
:104A200011741A1D92B2224416745A1D063392B2A2
:104A30009BB2224483421574E5D15EE72344197C7E
:104A4000A8E700BF2B0E0020BC08002001EB4101AD
:104A500049009631A0F86E10704708B503F04FF882
:104A60000D23B0FBF3F080B208BDF8B5054606266D
:104A700000277D244FF47A71284600F06DFD013C3B
:104A8000F8D187F00104E4B23946284600F0EAFC88
:104A90002146284600F028FD2146284600F0F2FC79
:104AA0002146284600F0F6FC2146284600F0FAFC94
:104AB0002146284600F0FEFC2146284600F002FD73
:104AC0002146284600F006FD2146284600F004FD58
:104AD0002146284600F010FD013E00D1F8BD2746D2
:104AE000C7E7000070B500250446012605724FF4A3
:104AF00080610C30FEF73EFA4FF4806104F1200033
:104B0000FEF738FA25652046A4F8545084F834504E
:104B1000A56384F83C50256484F8445084F84C60C4
:104B2000A4F8565000F032FB3146204600F06AFCF3
:104B30003146204600F096FC2946204600F0D4FC81
:104B40002946204600F09EFC2946204600F0A2FCA3
:104B50002946204600F0A6FC2946204600F0AAFC83
:104B60002946204600F0AEFC2946204600F0B2FC63
:104B70002946204600F0B0FC2946204600F0BCFC47
:104B80002946204600F076FC2946204600F016FC17
:104B90002946204600F01AFC2946204600F02AFC4F
:104BA0002046FFF762FF024B20461D6070BD00BF2C
:104BB000240E00202DE9F8431E46037A0546884658
:104BC0009146BBB1002400F120074C450AD018F8EB
:104BD00004102EB932463846FEF71AFA0134F4E7CB
:104BE000325DF8E7044C237823B92846FDF756FCDC
:104BF00001232370BDE8F8832B0E00202030FEF740
:104C0000CEB92030FEF784BA0C30FEF781BA00002E
:104C100070B50F480D46164600F07EFC0446A8B954
:104C20000B4800F085FC88B10A4B9E4207D89D4294
:104C30000CD80121BDE87040054800F065BC064B6A
:104C40009E4203D99D4201D92146F3E770BD00BFC2
:104C5000BC080020403A690DFFB0081970B515482E
:104C60000D46164600F058FC044608B1002070BD01
:104C7000104800F05DFC80B10F4B9E4206D89D426B
:104C8000F4D801210B4800F03FFCEFE70B4B9E42AC
:104C9000ECD99D42EAD92146F4E7064800F048FCE9
:104CA0000028E3D1054B9E4201D99D42DED8042065
:104CB000DDE700BFBC080020403A690DFFB00819CD
:104CC000F8B50D46194614460746069EFDF76EFEDA
:104CD0002D4B2E4AE91891421CD9E118914219D95D
:104CE0002B4A2C49A818884214D922448A4211D947
:104CF000294A2A49A81888420CD922448A4209D94B
:104D0000274A2849A818884204D922448A4201D94E
:104D10000420F8BD1D4A334493420ED91C4B1D4A52
:104D20003344934209D91C4B1C4A3344934204D95F
:104D30001B4B1C4A33449342EAD81B4A1B48AB180E
:104D40008342E5D9A3188342E2D9194B194905EBEF
:104D5000030C8C45DCD904EB030C8C45D8D93244C8
:104D60008242D5D933448B42D2D92246294638468D
:104D7000FFF774FF0028CBD10F4B1D600F4B1C6059
:104D80000F4B1E60C5E700BF00BC6AF7FF083D007F
:104D9000004FF7E6BF3B47034053F2F27F8D5B00C5
:104DA0008019D0CDFFF26F06C0444FF7400D0300CD
:104DB000406D12E6C0C62D0074020020780200206B
:104DC0007C020020F8B50D4604464B1E594259415D
:104DD00000F058FBAA1E51425141204600F05AFBF8
:104DE000E91E4F424F413946204600F05BFB281F29
:104DF000464246413146204600F05CFB394620469B
:104E000000F050FB314620466E1F00F053FB71420C
:104E100071412046AF1F00F055FB79427941204691
:104E200000F05AFBA5F1070CDCF100012046BDE8BB
:104E3000F84041EB0C0100F04DBB0000836B37B52F
:104E4000027A013304468363002A00F09380036DE5
:104E5000B3F5964F0DD3694B1A78511E042901D929
:104E6000072A04D1002120461970FFF7ABFF002369
:104E7000236545F6BF53A26B9A420AD9002394F8E2
:104E80004C10A36381F0010184F84C10204600F01F
:104E9000E9FA04F12000FEF79FF8594DF8B9594B93
:104EA0001B78E3B1584B1A7842B1187094F845302A
:104EB00023B1012229785548FDF72EFB544B1A786F
:104EC0004AB100221A7094F8453023B101222978A2
:104ED0004E48FDF721FB00212046FDF7FDFA2B7817
:104EE000022B0CBF4FF470624FF4F062494B19680B
:104EF000914229D300221A60404B1B7823BB236CBC
:104F000013BB94F83C30FBB13F4B1B78E3B9404BEB
:104F10001B78CBB994F8443094F845105A1CB2FB76
:104F2000F1F301FB132384F84430234493F8461033
:104F30002046FFF747FF94F844300122234493F8BA
:104F400046103248FDF7E8FA0C342046FEF744F8E4
:104F5000E0B10DF107020DF106012046FEF79EF8C3
:104F60002B78013B062B11D8DFE803F0121B242D10
:104F700036103F0028498B4208D990F84C108263C4
:104F800081F0010180F84C1000F06CFA03B030BDE4
:104F90009DF806102148003118BF0121FFF7F6FAED
:104FA000F4E79DF806101E48003118BF0121FEF7F6
:104FB00031FCEBE79DF806101A48003118BF0121BB
:104FC00002F0A4FFE2E79DF806101748003118BF71
:104FD000012101F041F9D9E79DF80610134800318D
:104FE00018BF012100F0A6FED0E79DF8061010487A
:104FF000003118BF012100F0EDFBC7E7280E0020AB
:10500000290E00202B0E00201E0E0020BC080020C0
:105010002A0E0020240E00207FA90300E8040020AF
:10502000F8030020D0120020D80E0020300E0020FF
:1050300014090020002310B580F845302E4B04469B
:105040001B7823B1012380F8463080F845302B4B84
:105050001B7843B1022194F84530E218013382F8FD
:10506000461084F84530264B1B7843B1032194F851
:105070004530E218013382F8461084F84530214B60
:105080001B7843B1042194F84530E218013382F8CB
:10509000461084F845301C4B1B7843B1052194F829
:1050A0004530E218013382F8461084F84530174B3A
:1050B0001B7843B1072194F84530E218013382F898
:1050C000461084F8453094F84530012B0AD9012365
:1050D00084F83C30237A23B9204600F04DF90123AF
:1050E000237210BD002384F83C30094B2046197808
:1050F000FFF768FEEEE700BF170000201600002053
:105100001C0000201A0000201900002018000020B8
:10511000280E002038B5064B0D461C788C421C46E4
:1051200003D00123036400F0E7F9257038BD00BF08
:105130001F0E002080F8341070470023036570476D
:10514000006D7047B0F854300B80B0F856301380C3
:105150000023A0F85430A0F8563070470C23434386
:10516000013B18460138FDD87047000008B50820FB
:1051700003F03EF838B10448FDF7E6F8BDE8084012
:10518000082003F043B808BDBC0800202DE9FF4704
:1051900001A803F0F9F801211D20634D03F07AFC0A
:1051A0000121624803F030F9614B624E01A92846A3
:1051B000019303F098F8604B01A930465F4F0193CB
:1051C00003F091F801A92846019703F08CF85C4B95
:1051D00001A92846019303F086F8284600224FF4DF
:1051E000006103F0EEF800224FF48051284603F0EE
:1051F000E8F842F21070FFF7B1FF4FF4C053ADF87A
:105200000430042328460DEB03018DF8073003F02A
:105210006AF800204B4C03F0B7FB01214FF400006B
:1052200003F046FCDFF844914FF4407002F024FF95
:1052300001A92046CDF8049003F055F8424B01A98E
:105240002046019303F04FF8404B01A920460193FB
:1052500003F049F83E4B01A92046DFF81481019381
:1052600003F041F801A93046CDF8048003F03BF883
:10527000384B01A92046019303F035F8364B01A9BC
:105280002046DFF8F0A0019303F02DF801A9304685
:10529000CDF804A003F027F8304B01A92046019374
:1052A00003F021F82E4B01A9204601932D4E03F067
:1052B0001AF801A92046CDF804A003F014F801A9BA
:1052C0002046019603F00FF8274B01A920460193D1
:1052D00003F009F801A92846019603F004F801A992
:1052E0002846CDF8049002F0FEFF01A92046CDF833
:1052F000048002F0F8FF01A92046019702F0F3FFB5
:105300000321012003F0B0F8082302934FF48053E7
:10531000ADF80C30012302A88DF80E3002F014FF16
:1053200004B0BDE8F08700BF000801400002300073
:105330000010034800100140008003480080031063
:1053400000180310000C014080000310400003040B
:1053500000010310100003040800030400020310FE
:1053600000100310020003100100031020000310BE
:10537000004003100020031007B5044B01A801935F
:1053800002F084FE03B05DF804FB00BF09010F01C9
:10539000032307B58DF8063010230029ADF804303B
:1053A00008BF042301A904488DF8073002F09BFFD1
:1053B00003B05DF804FB00BF000C01400A46024840
:1053C000202102F0FEBF00BF000C01400A46024847
:1053D000802102F0F6BF00BF000C014008B540215B
:1053E000034802F0D8FF431E5842584108BD00BF91
:1053F000000C01400A4602484FF4807102F0E1BF00
:10540000000C01400A4602484FF4804102F0D9BF27
:105410000010014008B51021034802F0BCFF431EF4
:105420005842584108BD00BF000C014008B5082192
:10543000034802F0B0FF431E5842584108BD00BF68
:10544000000C01400A460248102102F0BABF00BF1A
:10545000000C01400A460248082102F0B2BF00BF1A
:10546000000C01400A4602484FF4005102F0A9BF67
:10547000001001400A4602484FF4007102F0A1BF3B
:10548000000C01400A4602484FF4805102F099BFD7
:10549000000C01400A4602484FF4005102F091BF4F
:1054A000000C01400A460248022102F08ABF00BFF8
:1054B000000C01400A460248012102F082BF00BFF1
:1054C000000C01400A460248022102F07ABF00BFE8
:1054D00000080140FFF7F6BF0A460248202102F00B
:1054E00070BF00BF000801400A4602484FF48041E7
:1054F00002F067BF000C01400A4602484FF4004129
:1055000002F05FBF000C01400A4602484FF4004120
:1055100002F057BF0008014008B54FF4805103481E
:1055200002F039FF431E5842584108BD00080140AF
:1055300008B54FF40041034802F02DFF431E5842C6
:10554000584108BD0010014042F21070FFF706BE3E
:105550004FF49670FFF702BE0846FFF7FFBD00BF8D
:1055600000BF00BF70470023021D0370438000F19D
:10557000370102F8013B9142FBD1C363431D8363B2
:105580007047002303704380C363704710B543889E
:1055900004465B009BB2D9B96380608880F4AB405D
:1055A00080F0770002F070FBA8B91749174801F0A6
:1055B00013FC5522A36B01211A70F722A36B5A70BA
:1055C000134B2170E3631348BDE81040FFF7A2BD01
:1055D00043F00103E0E7608880F47F4080F05D00E5
:1055E00002F052FB78B90C49084801F0F5FBFF22A4
:1055F000A36B01211A705D22A36B5A70044BE36305
:1056000002232370DFE710BD06FA0008C411002052
:1056100010000400BC0800202BFA000810B5084850
:105620000C46FCF733FE030A84F8320084F831306C
:105630002146BDE810403322024801F00DBB00BFF7
:10564000BC080020C411002010B508480C46FCF727
:105650001DFE030A84F8320084F831302146BDE88B
:1056600010403322024801F025BB00BFBC080020D7
:10567000C411002070B504464388828F5B009BB242
:105680004C4E4380D01002F00702A56BB25C00299B
:1056900000F08B8043F0010363802B5C1A432A5493
:1056A000A38F5A1C92B2B2F5C07FA28704D90023FF
:1056B00023706380E36316E00E3B022B40D86088C2
:1056C00080F4AB4080F0770002F0DEFA02280BD8BD
:1056D000A28F3949103A12B2384801F09AFE384B7D
:1056E000E3630123237070BD608880F47F4080F005
:1056F0005D0002F0C9FA02280AD8A28F3149103A97
:1057000012B22E4801F085FE2D4BE3630223E9E738
:10571000608880F4AA4080F05D0002F0B5FA0228AB
:105720000ED8A28F2849103A12B2244801F071FE17
:1057300000212648FFF7EEFC204801F0E9FAB6E721
:10574000A38FB3F5C07FCED1E58F013DADB2E58724
:1057500075B91F49194801F03FFB29461B48FFF75F
:10576000D9FC164801F0F2FA25706580E563BAE7C6
:10577000EB1E5D425D412571254615F8043B012B6A
:1057800009D0022B0CD033220021284606F068FBFA
:105790000023A387A7E729462046FFF73FFFF2E74C
:1057A00029462046FFF750FFEDE72B5C23EA020273
:1057B00075E700BF82F900088AF90008C4110020CB
:1057C00010000400ACF90008CAF90008BC08002069
:1057D000E5F900080378013B012B01D8FFF74ABF28
:1057E000FFF7D4BE10B540F2DC51044602F074F964
:1057F000002304F1100204F5986102F8013B914284
:10580000FBD1F022C4F8C034A4F8C42484F8C63410
:10581000204610BD312A70B506460C460ED102F066
:105820006EF92F280CD904F1300514F8011F304609
:1058300002F09EF9AC42F8D1002070BD0420FCE7D4
:105840000520FAE773B50D460824094EEB098DF8DB
:105850000730012200230DF107013046013CFFF71C
:10586000A9F96D0014F0FF04EDB2EFD102B070BDE4
:10587000BC080020F8B5044602F05EF9B4F8C03464
:1058800030BB002B57D02C48FFF7B8F9002705464E
:105890000326082D4FD994F8C634002B3CD077212D
:1058A0002046FFF7CFFFB4F8C2340133A4F8C23466
:1058B000B4F8C224B4F8C034083D9A42ADB2E8D37B
:1058C00094F8C6349BB384F8C674C4F8C064E0E7A7
:1058D000002BD8D1194A127862B9012384F8C63452
:1058E000B4F8C434A4F8C0340023A4F8C234B4F823
:1058F000C034C6E7302584F8C634B4F8C064204606
:10590000731CA4F8C03402F056F9013D264415F08A
:10591000FF053074F1D1E7E7B4F8C23420465A1CD1
:10592000A4F8C2242344197CFFF78CFFC0E7C4F815
:10593000C03484F8C634F8BDBC0800202B0E00200B
:1059400001EB4101890001F51671A0F8C4147047FC
:1059500008B502F0D4F83023B0FBF3F0C0B208BDB4
:10596000014800F081BF00BFC411002038B53548A0
:10597000FFF764FA344801F077FD344B344C1B7860
:105980002BB12378012B02D13248FEF79BFF324B1B
:10599000324D1B783BB12378022B04D12B7813B9FD
:1059A0002F48FEF7E9F82F4B1B782BB12378032BF8
:1059B00002D12D4802F0FAFA2C4B1B782BB1237838
:1059C000042B02D12A4800F0A5FC2A4B1B782BB1EE
:1059D0002378052B02D1284800F0F6F9274B1B78D5
:1059E0002BB12378072B02D12548FFF743FF254B26
:1059F0001B782BB12378062B1DD1234800F082FDA4
:105A00002B785C3BDBB2082B0ED840F2411222FA15
:105A100003F3DB0702D51D48FDF702FC2B78602B52
:105A200002D11B48FDF764FC237853B9BDE8384028
:105A30001848FDF7A5BC144800F0F0FC0028DCD1A4
:105A4000DEE738BDBC080020C4110020170000208C
:105A5000280E002048080020160000201C0E002000
:105A6000800400201C000020681300201A00002081
:105A7000D00F002019000020800E00201800002008
:105A8000540900201B000020E410002084020020A4
:105A9000B0020020C002002008B5FFF761FFFFF749
:105AA00065FFFCE708B51C48FEF760F91B48FEF7E8
:105AB0007AFD1B48FDF726FD1A48FDF7FFFF1A483F
:105AC00002F02FF9194802F027FA194800F0FCF902
:105AD000184800F0CCFB1848FFF745FD1748FFF7C2
:105AE00081FE174800F03CF8164800F029F91648E6
:105AF00000F07EFC1548FDF711FB1548FDF7F0FBA3
:105B00001448FDF72DFC144800F056FDBDE8084090
:105B10001248FEF7E7BF00BFE80400204808002055
:105B2000F803002080040020D01200206813002019
:105B3000D80E0020D00F00201409002054090020A6
:105B4000300E0020800E0020E4100020840200208F
:105B5000B0020020C0020020C4110020BC080020B8
:105B600030B5002400250023C0E90245037000F190
:105B7000100200F1430102F8013B9142FBD1836422
:105B800000F11103436430BD30B50023002400252B
:105B90000370C0E90245836430BD000010B5D0E950
:105BA0000232DB180446524101BBC4E90232A0684C
:105BB0000021C0F313030F48584002F081F8C0B928
:105BC0000D490E4801F008F9CD22636C01211A70CD
:105BD000F522636C0A485A709022636C9A70094BE4
:105BE0002170A364BDE81040FFF794BA43F00103AD
:105BF000DBE710BD59DF0C0096FA0008C411002045
:105C0000BC0800201400060010B508480C46FCF73C
:105C10003DFB030A84F8320084F831302146BDE8A8
:105C200010403322024800F0CBBF00BFBC08002068
:105C3000C411002070B50446D0E90232DB1852418D
:105C4000C0E90232B0F84820334ED01002F007020B
:105C5000656CB25C00295AD043F00103A3602B5C51
:105C60001A432A54B4F8483001339BB2B3F5C07FCD
:105C7000A4F8483002D92046FFF786FFB4F8483030
:105C8000123B042B14D8A0680021C0F3130323484F
:105C9000584002F015F803280AD8B4F848202049E3
:105CA000143A12B21F4801F0B4FB1F4BA36470BD3D
:105CB000B4F84830B3F5C07FF9D1B4F84A50013D8B
:105CC000ADB2A4F84A507DB91849164801F084F8DD
:105CD00029461748FFF71EFA124800F09FFF20469A
:105CE000BDE87040FFF750BF26466B1F5D425D4127
:105CF00006F8105F31462046FFF786FF3322002169
:105D0000304606F0ADF80023A4F84830CFE72B5C0E
:105D100023EA0202A5E700BF4CFA000859DF0C0095
:105D200054FA0008C41100201400060074FA000898
:105D3000BC08002003780BB9FFF730BFFFF77ABF2C
:105D400010B540F2DC51044601F0C6FE002204F119
:105D5000100304F14C0103F8012B9942FBD1F0230D
:105D6000E2642365204610BD312A70B506460C4614
:105D70000ED101F0C4FE2F280CD904F1300514F81F
:105D8000011F304601F0F4FEAC42F8D1002070BD96
:105D90000420FCE70520FAE773B50D460824094EF8
:105DA000EB098DF80730012200230DF10701304681
:105DB000013CFEF7FFFE6D0014F0FF04EDB2EFD1E1
:105DC00002B070BDBC080020F8B5044601F0B4FE76
:105DD000B4F84C3040BB002B5ED03048FEF70EFFCD
:105DE0004FF4807605462E4F082D55D994F8523041
:105DF000002B3DD05F212046FFF7CEFFB4F84E3098
:105E00000133A4F84E30B4F84E20B4F84C30083DBD
:105E10009A42ADB2E8D394F85230002B39D0032324
:105E2000A4F85260E364DFE7002BD6D11D4A127854
:105E300062B90123A4F85230B4F85030A4F84C30C1
:105E40000023A4F84E30B4F84C30C4E73025A4F851
:105E50005230B4F84C602046731CA4F84C3001F06A
:105E6000AAFE013D264415F0FF053074F1D1E7E7A5
:105E7000B4F84E3094F853105A1C92B2A4F84E2045
:105E800021B1F95C2046FFF787FFBCE72344197C6A
:105E9000F8E7E364A4F85230F8BD00BFBC08002066
:105EA000B1FA00082B0E002001EB4101490001F579
:105EB0009671A0F85010704708B501F020FE30230D
:105EC000B0FBF3F080B208BD30B5002400250023FC
:105ED000C0E90245037000F1100200F1EB0102F885
:105EE000013B9142FBD1064AA0F8F43080F8F6302D
:105EF00000F11103C0F8F020C0F8EC3030BD00BF55
:105F000000000F27002330B500240025054A037048
:105F1000C0E90245C0F8F020A0F8F43080F8F6306F
:105F200030BD00BF00000F2710B5D0E90232DB18EA
:105F30000446524141BBC4E90232A189A368144816
:105F400081F4AA41584081F0750101F0B9FE0228A0
:105F50001DD81049104800F03FFF00230F4A12F8E7
:105F6000010BD4F8EC10C8540133062BF7D10423ED
:105F70000121A4F8F43030232170A4F8F03008484F
:105F8000BDE81040FFF7C6B843F00103D3E710BDEA
:105F9000FF77FFF508FB0008C4110020BCFA0008D9
:105FA000BC08002010B508480C46FCF76FF9030A3E
:105FB00084F8DA0084F8D9302146BDE81040DB22AD
:105FC000024800F0B3BD00BFBC080020C41100208F
:105FD00010B590F8F63004460F2B28D8DFE803F010
:105FE0000827271127272717272727271E27272096
:105FF0001049114800F0F0FE4FF44673A4F8F23057
:1060000010BD0E490C4800F0E7FE9023F6E70C495E
:10601000094800F0E1FE4FF4B473EFE70949F7E7F0
:106020000949054800F0D8FE4FF4D873E6E74FF46D
:10603000D863E3E722FB0008C41100203BFB000803
:1060400054FB00086EFB000887FB000870B504468F
:10605000D0E90232DB185241C0E90232B0F8F02038
:106060002A4ED01002F00702D4F8EC50B25C00299E
:1060700048D043F00103A3602B5C1A432A54B4F8C0
:10608000F03001339BB2B3F5D86FA4F8F03002D9E9
:106090002046FFF737FFB4F8F030402B1BD148F211
:1060A0008902D4F8EC30DB7903F00F0384F8F63082
:1060B00022FA03F3DB0705D40423A4F8F430022307
:1060C000237070BD2046FFF783FF94F8F620104937
:1060D000104801F09EF9B4F8F230B4F8F0209A427A
:1060E000EFD101232146D2081A4401F8103FD2B261
:1060F000084800F0EFFC0423A4F8F4300023A4F8CF
:10610000F030DCE72B5C23EA0202B7E7B4FA0008C0
:10611000C2FA0008C411002070B50446D0E902326A
:10612000DB185241C0E90232B0F8F020434ED010E3
:1061300002F00702D4F8EC50B25C002979D043F0A9
:106140000103A3602B5C1A432A54B4F8F0300133E6
:106150009BB2B3F5D86FA4F8F03002D92046FFF710
:10616000D1FEB4F8F0302E3B042B16D8A189A368D9
:10617000334881F4AA41584081F0750101F0A0FD37
:1061800004280AD82F49304800F026FE0423A4F83A
:10619000F4303023A4F8F03070BDB4F8F030402B68
:1061A0000FD1D4F8EC302046DB7903F00F0384F8EC
:1061B000F630FFF70DFF94F8F6202449224801F04D
:1061C00028F9B4F8F030B3F5D86FE5D1B4F8F4504D
:1061D000013DADB2A4F8F450C5B91D491A4800F00C
:1061E000FBFD29461B48FEF795FF174800F0CAFC47
:1061F0002046FFF787FE94F8F630032B01D00F2BD3
:10620000CAD12046BDE87040FFF77CBE2646EB1E93
:106210005D425D4106F8105F31462046FFF7C2FE41
:10622000DB220021304605F01BFE0023A4F8F030ED
:10623000E1E72B5C23EA020286E700BFB4FA00081C
:10624000FF77FFF5CEFA0008C4110020C2FA00085B
:10625000E7FA0008BC0800200378012B03D0022BCA
:1062600003D0FFF761BEFFF7F1BEFFF755BF10B5D2
:1062700040F2DC51044601F02FFC002304F110022F
:1062800004F5857102F8013B9142FBD14FF4700295
:10629000A4F80A31C4F80C2184F81031204610BD4E
:1062A000122AF8B506460F46144614D901F027FC09
:1062B000844212D8013CE1B2304601F059FC00257D
:1062C000EBB29C4205F1010509D93B4459783046AF
:1062D00001F04EFCF4E70420F8BD0520FCE70020A7
:1062E000FAE7000073B50D460824094EEB098DF856
:1062F0000730012200230DF107013046013CFEF773
:1063000059FC6D0014F0FF04EDB2EFD102B070BD86
:10631000BC080020F8B5044601F00EFCB4F80A51A0
:1063200028BB002D36D02848FEF768FC0546082D0E
:1063300030D9B4F80C3194F810115A1C92B2A4F868
:106340000C2100293CD077212046FFF7CBFFB4F881
:106350000C21B4F80A31083D9A42ADB2E7D30023CC
:10636000A4F80C31A4F80A3184F8103112E0002DA1
:10637000D9D1164B1B7873B9012384F81031B4F8C6
:106380000E31A4F80A310023A4F80C31B4F80A3114
:10639000002BC8D1F8BD204601F00DFC074684F85B
:1063A0001051EBB2BB42B4F80A61ECD2731CA4F8F2
:1063B0000A31204601F0FFFB264430740135F0E736
:1063C0002344197CC0E700BFBC0800202B0E00202E
:1063D00001EB4101890001F51671A0F80E1170471B
:1063E00008B501F08CFBD823B0FBF3F080B208BDF8
:1063F00010B54FF47A71044601F06EFB002204F1EF
:10640000100304F1D80103F8012B9942FBD1482372
:10641000C4F8D820C4F8DC30204610BD08B5B0F868
:10642000D8302BB901F088FB003018BF012008BD1F
:106430000120FCE7442A70B506460C460ED101F057
:106440005EFB43280CD9651E433415F8011F304606
:1064500001F08EFBA542F8D1002070BD0420FCE7BE
:106460000520FAE773B50D460824094EEB098DF8AF
:106470000730012200230DF107013046013CFEF7F1
:1064800099FB6D0014F0FF04EDB2EFD102B070BDC6
:10649000BC08002001EB41014908483196298ABF18
:1064A0009623A0F8DC10A0F8DC30704708B501F0A6
:1064B00026FB4423B0FBF3F0C0B208BD012A08B5A7
:1064C0000DD10B78012B0CBF0123002380F8DF30A6
:1064D00003D106210348FCF71FF8002000E0042048
:1064E00008BD00BFBC080020AA2100F1100300F184
:1064F000540203F8011B9342FBD14423C0F8D83067
:106500007047000070B590F8DF30044623B10023D7
:1065100080F8DE30FFF7E8FFB4F8D85005B3244820
:10652000FEF76CFB0546082D2FD9B4F8DA3094F845
:10653000DE105A1C92B2A4F8DA20B1B3AA21204688
:10654000FFF790FFB4F8DA20B4F8D830083D9A424B
:10655000ADB2E8D30023C4F8D83084F8DE3014E0BC
:10656000204601F0E9FA60B1124B1B7873B90123A0
:1065700084F8DE30B4F8DC30A4F8D8300023A4F876
:10658000DA30B4F8D830002BC9D170BD84F8DE50B1
:1065900004F1540604F11005204601F00CFB05F847
:1065A000010BB542F8D14423E6E72344197CC6E742
:1065B000BC0800202B0E00200246002300F580714D
:1065C00002F8013B9142FBD1A0F80031C0E9413310
:1065D00070471FB54FF49C63ADF80C3070238DF8F5
:1065E0000E30837803AA8DF80F3000230121009329
:1065F000042301F011FB05B05DF804FB1FB54FF457
:10660000BC63ADF808307F238DF80A3083788DF8AD
:106610000C108DF80B30002302AA009301210523F2
:1066200001F0FAFA05B05DF804FB00002DE9F04F27
:10663000834687B05D48FEF780FD5D4B02935D4B5E
:106640001A789A4612B101238DF80B305A4B1A78FA
:1066500099462AB19DF80B3043F002038DF80B30B8
:10666000564B1A7898462AB19DF80B3043F0040334
:106670008DF80B30524F3B782BB19DF80B3043F027
:1066800008038DF80B304F4E33782BB19DF80B304B
:1066900043F010038DF80B304B4D2B782BB19DF848
:1066A0000B3043F020038DF80B30484C23782BB18E
:1066B0009DF80B3063F07F038DF80B30444B3B4863
:1066C0001B788DF80C30434B1B788DF80D30FEF79E
:1066D0009BFA28B19DF80D3043F004038DF80D307E
:1066E0003248FEF78EFA28B19DF80D3043F00803CA
:1066F0008DF80D309AF80030002B3FD03648FEF769
:10670000ACF98DF80E0099F80030002B39D00A232F
:1067100032488DF80F30FDF797FA8DF8100098F891
:1067200000309BB32E4801F09FFC8DF811003B78A0
:106730007BB32C48FFF754FE8DF8120033785BB31F
:106740002948FFF7B9FB8DF813002B783BB3274896
:10675000FFF7ACFE8DF8140023781BB32448FFF735
:10676000F7F88DF81500002302AA009301210E23EB
:10677000584601F051FA07B0BDE8F08F8DF80E30A1
:10678000C1E78DF80F308DF81030C8E78DF8113063
:10679000CDE78DF81230D1E78DF81330D5E78DF8BD
:1067A0001430D9E78DF81530DDE700BFBC080020B4
:1067B000E00E010017000020160000201C00002041
:1067C0001A000020190000201B00002018000020E3
:1067D000280E00202B0E00204808002080040020F6
:1067E00068130020D00F0020800E0020E41000204D
:1067F0005409002010B50C4BA4B0039304230B4C98
:106800001A1FD2B2A25C32B124A91944013301F893
:10681000842CDBB2F4E70092012103AA8DF80D303D
:1068200001F0FAF924B010BDE0000001A2FB00085D
:10683000082A13B514D9092AD1F8050014BF4B7AD8
:10684000FF230D2A94BF0246D1F80A20D1F8014057
:106850000092214602460348FEF732FA02B010BD0C
:106860000420FBE7BC0800204FF4E132012101F0D5
:10687000B5B9000030B5134B91B01B78012B1FD870
:10688000114B1B78E3B1E023ADF80C30102300244A
:106890008DF80E30E5B2EB1CAA42DBB206D910AD82
:1068A0002B440D5D013403F8345CF3E70332D3B2BB
:1068B00000220121009203AA8DF80D3001F0ACF9FD
:1068C00011B030BD280E00201700002030B5134B4A
:1068D00089B01B78012B1FD8114B1B78E3B1E02343
:1068E000ADF80C30112300248DF80E30E5B2EB1C0E
:1068F000AA42DBB206D908AD2B440D5D013403F882
:10690000145CF3E70332D3B200220121009203AA00
:106910008DF80D3001F080F909B030BD280E00204F
:10692000170000201FB50C4B1B78012B10D80B4B08
:106930001B786BB14FF47873ADF80C3012238DF8DF
:106940000E30002303AA00930121032301F064F910
:1069500005B05DF804FB00BF280E002017000020E2
:106960001FB50C4B1B78012B10D80B4B1B786BB150
:106970004FF47873ADF80C3013238DF80E300023EC
:1069800003AA00930121032301F046F905B05DF845
:1069900004FB00BF280E00201700002030B5154C66
:1069A0008DB0247814F0FD0422D1134D2D78FDB163
:1069B000002914BF1A211821E0258DF80A1021465C
:1069C000ADF80850CDB2EC1CAB42E4B206D90CAD28
:1069D0002C44555C013104F8285CF3E700220333B2
:1069E000DBB20092012102AA8DF8093001F014F9FE
:1069F0000DB030BD280E0020160000201FB50D4B35
:106A00001B7813F0FD0312D10B4A12787AB14FF4C0
:106A100078720029ADF80C2014BF1B2219220093B4
:106A20008DF80E20032303AA012101F0F5F805B02B
:106A30005DF804FB280E00201600002030B5144B32
:106A4000A5B01B78032B00D0FBB9124B1B78E3B128
:106A5000E023ADF80C30202300248DF80E30E5B291
:106A6000EB1CAA42DBB206D924AD2B440D5D0134E8
:106A700003F8845CF3E70332D3B2002201210092D1
:106A800003AA8DF80D3001F0C7F825B030BD00BF66
:106A9000280E00201C0000201FB50C4B1B78032B78
:106AA00000D083B90A4B1B786BB14FF47873ADF803
:106AB0000C3021238DF80E30002303AA009301210E
:106AC000032301F0A9F805B05DF804FB280E0020AF
:106AD0001C00002030B5134BA1B01C7814F0FB044F
:106AE0001ED1114B1B78DBB1E023ADF80830302309
:106AF0008DF80A30E5B2EB1CAA42DBB206D920AD14
:106B00002B440D5D013403F8785CF3E70332D3B214
:106B100000220121009202AA8DF8093001F07CF8D0
:106B200021B030BD280E00201A00002030B5134BD4
:106B3000C3B01C7814F0FB041ED1114B1B78DBB1E1
:106B4000E023ADF80C3031238DF80E30E5B2EB1CAC
:106B5000AA42DBB206D942AD2B440D5D013403F8E5
:106B6000FC5CF3E70332D3B200220121009203AAB6
:106B70008DF80D3001F050F843B030BD280E0020E4
:106B80001A0000201FB50C4B1B7813F0FB030FD12C
:106B90000A4A127862B14FF47872ADF80C203222B2
:106BA00000938DF80E20032303AA012101F034F88D
:106BB00005B05DF804FB00BF280E00201A0000207D
:106BC00030B5144BA5B01B78052B00D0FBB9124B88
:106BD0001B78E3B1E023ADF80C30402300248DF89E
:106BE0000E30E5B2EB1CAA42DBB206D924AD2B4431
:106BF0000D5D013403F8845CF3E70332D3B2002265
:106C00000121009203AA8DF80D3001F005F825B09E
:106C100030BD00BF280E0020190000201FB50C4B0E
:106C20001B78052B00D083B90A4B1B786BB14FF44E
:106C30007873ADF80C3041238DF80E30002303AA91
:106C400000930121032300F0E7FF05B05DF804FB8A
:106C5000280E00201900002030B5144BA5B01B7879
:106C6000072B00D0FBB9124B1B78E3B1E023ADF842
:106C70000C30452300248DF80E30E5B2EB1CAA42FF
:106C8000DBB206D924AD2B440D5D013403F8845CDE
:106C9000F3E70332D3B200220121009203AA8DF858
:106CA0000D3000F0B9FF25B030BD00BF280E002028
:106CB0001800002030B5144BA5B01B78072B00D06E
:106CC000FBB9124B1B78E3B1E023ADF80C3046233F
:106CD00000248DF80E30E5B2EB1CAA42DBB206D9D7
:106CE00024AD2B440D5D013403F8845CF3E70332DB
:106CF000D3B200220121009203AA8DF80D3000F0DA
:106D00008BFF25B030BD00BF280E002018000020EA
:106D10001FB50C4B1B78072B00D083B90A4B1B788F
:106D20006BB14FF47873ADF80C3049238DF80E3009
:106D3000002303AA00930121032300F06DFF05B097
:106D40005DF804FB280E0020180000201FB50C4B36
:106D50001B78072B00D083B90A4B1B786BB14FF41B
:106D60007873ADF80C3048238DF80E30002303AA59
:106D700000930121032300F04FFF05B05DF804FBF1
:106D8000280E00201800002030B5124B8BB01B7865
:106D9000602B1CD1E023ADF80830092300248DF8C6
:106DA0000A30E5B2EB1CAA42DBB206D90AAD2B448D
:106DB0000D5D013403F8205CF3E70332D3B2002207
:106DC0000121009202AA8DF8093000F025FF0BB0D6
:106DD00030BD00BF1C0E002010B590F80A31A4B0E1
:106DE000C3B1E023ADF80C30F1238DF80E3003234E
:106DF000DA1ED2B28A5C32B124AC1C44013304F8EE
:106E0000842CDBB2F4E7012103AA00918DF80D3048
:106E100000F002FF24B010BD2DE9F04F0C2A8FB016
:106E2000074603D804200FB0BDE8F08F91F800B0FA
:106E3000CBF3001380F80A314D788E7805F01003FB
:106E4000089305F020030993322E05F0400305F066
:106E5000020A05F0040905F008080B93E2D8CC7883
:106E6000052C40F28E80072C00F0AF80062C00F03D
:106E7000AA80A4F15C03DBB2092BD3D840F2D13055
:106E800020FA03F313F0010FCCD08B790F2B0A9368
:106E9000C8D84B799E489B100370087B0F2A0D9031
:106EA0008CBFC87B8020112A8CBF91F811C04FF095
:106EB000800C152A98BF80224B7A88BF4A7D91F8B2
:106EC0000AE00C93CB7ACDE901020D9ACBF3C00115
:106ED000CDE903C1079100920C9972468D48FBF7EA
:106EE0006BFD1AF1000A18BF4FF0010ADFF870E2DB
:106EF00019F10009089B18BF4FF0010905F00105C1
:106F000018F1000818BF4FF001088EF80050003348
:106F10000B9D18BF0123003518BF01257E4A7F480D
:106F200013707F4B80F800901D70099DDFF82C9244
:106F3000003518BF012589F80050A4F15C05794996
:106F4000DFF820C2EDB2082D81F800808CF800A097
:106F5000CDE90801CDE90B23F246E046724B7349B7
:106F600035D9652C5ED1012289F8002006221A70DD
:106F700097F80B310C70002B41D06648FBF75CFD95
:106F80003DE0012C02D115F0010F7DE7022C04D168
:106F9000BAF1000F7FF479AF44E7032C04D1B9F1C3
:106FA000000F7FF472AF3DE7042C04D1B8F1000F5D
:106FB0007FF46BAF36E7052C7FF467AF089B002B9F
:106FC0007FF463AF2EE7099BF9E70B9BF7E740F2ED
:106FD0005112EA40D20725D501228CF80020022266
:106FE0001A7097F80B310C7013B14A48FBF724FD67
:106FF000602C04D1012202214648FBF78DFA4FFA9A
:107000008BF3D9434A4AC90F002B11700FDB474B52
:107010001B7863B9632C0AD046484749FFF7DCFE6A
:10702000062000E700221C70404B1A70E7E731464B
:107030004248FDF70BFD3146414801F00DF831465D
:107040004048FFF7C5F931463F48FEF72DFF31466E
:107050003E48FEF775FC31463D48FFF71BFA3146C6
:107060003C48FCF7F9FD0A993B48FCF7B9FB079946
:107070002848FEF75FF897F80B3133B1092D04D893
:1070800040F25133EB40DB0707D49AF80030BBB134
:10709000012211461F48FBF73FFA1E48FDF7CAFFC1
:1070A0001C48FBF7F5FE092D2FD840F25130E8407F
:1070B000C04310F0010028D1012387F80B31B2E65C
:1070C00098F8003013B101220221E3E7089B1B78F6
:1070D00013B101220321DDE7099B1B7813B10122C3
:1070E0000421D7E70B9B1B7813B101220521D1E7BF
:1070F0000C9B1B7813B101220721CBE7174B1B78A0
:10710000002BCAD001220621C4E700208BE600BF75
:1071100015000020BC080020190000201C000020E1
:10712000180000201A000020280E00201C0E00204D
:10713000200E0020C411002044FE00084808002052
:1071400068130020D00F0020800E0020540900207A
:10715000E410002080040020F80300201B00002021
:10716000170000201600002038B54B1E0C46062BD9
:107170007FD8DFE803F00C043843517662003F49C2
:107180003F48FFF729FE3F48FCF72DFE06E03C484C
:107190003D49FFF721FE3D48FCF7CAF93C4800F0A5
:1071A000D6FD3C48FEF7AEFE3B48FEF7EDFC3B4803
:1071B000FEF7E7F93A48FCF79DF93A4D2C7064B1B7
:1071C000394B1B78A34208D038492D48FFF704FEFD
:1071D000012221463648FBF79FF929783448BDE85B
:1071E0003840FDF7EFBD33492548FFF7F5FD274847
:1071F000FCF79EF92348FCF7F6FDD2E72E4920481C
:10720000FFF7EAFD2148FCF793F91E48FCF7EBFD78
:107210001F4800F09CFDC7E728491948FFF7DCFD2F
:107220001A48FCF785F91748FCF7DDFD184800F00F
:107230008EFD1848FEF766FEB9E721491048FFF7B2
:10724000CBFD1248FCF774F90E48FCF7CCFD104852
:1072500000F07DFD0F48FEF755FE0F48FEF794FC49
:10726000A8E718490648FFF7B7FD0848FCF760F99A
:1072700089E715490248FFF7AFFD9EE794FD000836
:10728000C4110020E8040020A4FD0008F803002039
:10729000D0120020D80E0020300E0020140900204B
:1072A000C0020020280E0020290E002026FE000823
:1072B000BC080020B7FD0008D1FD0008E1FD000872
:1072C000F2FD000802FE000815FE000810B5044695
:1072D0009AB12E4B09781B788B422FD0052921D9E2
:1072E000072941D0062941D0632921D0A1F15C03AF
:1072F000DBB2082B03D965293AD004212EE040F2F5
:10730000511222FA03F3DB07F7D50122204B1A7042
:10731000204B197090F80B3113B11F48FBF78CFB11
:10732000022108E001290BD11C4B1B78002BE4D073
:107330000022184B1A702046FFF716FF00210DE0BF
:10734000022901D1124BF0E7032901D1144BECE7DC
:10735000042905D1134B1B78002BE9D1084610BD39
:107360000529E5D1104BE0E7104BDEE7104BDCE7D9
:1073700001220F4B1A70074B197090F80B3113B1A3
:107380000548FBF759FB0621D5E700BF280E002072
:10739000160000201C0E0020BC0800201700002052
:1073A0001C0000201A0000201900002018000020F6
:1073B0001B00002070B590F80A31A4B0054633B325
:1073C000E023ADF80C30F12303248DF80E30E31EDA
:1073D000DBB2CE5C601C24ABC0B223441EB103F808
:1073E000846C0446F3E7202103F8841C03ABC0F14E
:1073F0008201184400F086FC012104F10A03DBB28B
:10740000009103AA28468DF80D3000F005FC24B049
:1074100070BD70B590F80A31A4B013B3E023ADF895
:107420000C30F2238DF80E300323DC1EE4B20E5D27
:1074300024AD5C1CE4B21D441EB105F8846C2346E7
:10744000F3E7111205F8841C24A90C44012102332E
:1074500004F8842CDBB2009103AA8DF80D3000F003
:10746000DBFB24B070BD0000F8B50446A84EA94D62
:107470000121204600F0BAFB0746002800F02582D3
:107480000121204600F0BCFB94F800214AB9E02815
:1074900004D101232070A4F80031E9E784F8012128
:1074A000E6E7012A06D10223607084F8010184F81E
:1074B0000031DDE7A0540132D1B294F8012184F803
:1074C00000119142D4D1A3781A2B00F04D8145D8F8
:1074D000082B00F0AF8017D8022B00F0988007D857
:1074E000002B00F09080012B00F089800121B6E094
:1074F000032B00F09880042BF8D1033AD2B2E11CA0
:107500002046FFF795F988E0112B00F0D9801ED8AE
:107510000A2B00F0B780102BE8D17F4B1B78002B93
:1075200000F0CA802B78012B00F2C680033AD2B259
:10753000E11C7A48FDF750F80746002840F0BD806E
:107540002B784BB901212046FFF70EFE04E0132BE8
:1075500000F0CB80182BC9D100239CE7402B00F012
:107560004F8123D8202B00F0178103D81C3B022B1E
:10757000F2D9BBE7302B00F02881312BB6D1684B14
:107580001B78002B00F03A812B7813F0FB0F40F0B2
:107590003581033AD2B2E11C6248FEF781FE07460C
:1075A000002800F021813AB25F4954E0492B00F0F5
:1075B0005B811BD8452B00F03C81462B96D15B4B61
:1075C0001B78002B00F04E812B7813B1072B40F075
:1075D0004981033AD2B2E11C5548FEF71BF9074630
:1075E000002800F035813AB2524934E0502B00F0C7
:1075F0005081FFF47BAF7033DBB2012BB8E720463C
:10760000FFF714F8A8E72046FFF7F4F8A4E7CA1E2E
:10761000D2B2E11C2046FFF7FFFB0146F8B9204635
:10762000FEF7D7FF98E7033AD2B2E11C2046FFF7F6
:107630004DFEF2E7404B1B78622B01D05C2B12D140
:10764000033AD2B2E11C3D48FBF72CFE0746002866
:10765000E5D03B493AB23B48FFF7DBFE39462046CE
:10766000FEF7CCFF78E7652B06D1033AD2B2E11CD6
:107670003548FEF723FFE9E703F0FB03602BCED08C
:107680000227E6E72B78ABB90122304B6121304865
:107690001A70FAF741FF94F80121E11C033AD2B2C3
:1076A0002C48FBF7B7FE074600283FF455AF3AB227
:1076B0002949D0E70527FAE702273AB22749CAE75E
:1076C000154B1B787BB12B78012B0CD8033AD2B227
:1076D000E11C1248FCF7A6FF074600283FF430AF34
:1076E0003AB21F49B7E70227FAE70B4B1B7863B1A1
:1076F0002B78012B09D80948FCF7BAFF0746002868
:107700003FF41EAF3AB21749A5E70227FAE700BFD8
:1077100016000020280E0020170000204808002036
:107720001A000020D00F0020E4FC00081800002000
:10773000540900203DFD00081C0E0020840200209A
:10774000FDFB0008C4110020E41000201E0E0020E4
:10775000BC080020C00200201FFC000832FC00080A
:1077600051FC00086EFC000833788BB12B7813F0C5
:10777000FD0F0DD1CA1ED2B2E11C5948FCF7B2F977
:10778000074630B92B78002B7FF4E6AE0221DAE60B
:1077900002273AB253495EE7534B1B788BB12B78E3
:1077A0000BB1032B0DD1033AD2B2E11C4F4800F0CC
:1077B000CCFB074630B92B78002B7FF4CDAE0321EC
:1077C000C1E602273AB24A4945E74A4B1B788BB1DA
:1077D0002B7813F0FB0F0DD1033AD2B2E11C4648CF
:1077E000FEF75EFD074630B92B78002B7FF4B4AE70
:1077F0000421A8E602273AB240492CE70227D2E644
:107800003F4B1B788BB12B780BB1052B0DD1033A75
:10781000D2B2E11C3B48FEF7A7FA074630B92B78F5
:10782000002B7FF499AE05218DE602273AB2364946
:1078300011E7364B1B788BB12B780BB1072B0DD191
:10784000033AD2B2E11C3248FDF7E4FF074630B9F3
:107850002B78002B7FF480AE072174E602273AB222
:107860002C49F8E60227BEE6284B1B787BB12B7823
:107870000BB1072B0BD1033AD2B2E11C2448FDF720
:10788000C9FF07460028E3D03AB22349E3E60227BE
:10789000FAE7224B1B78A3B12B780BB1062B10D142
:1078A00001211F4B033A1970D2B2E11C1D48FEF7AB
:1078B000C1FD074630B92B78002B7FF44DAE062171
:1078C00041E602273AB21849C5E61848FDF738FCE8
:1078D0004BF67F33984288BFA4F80071F8BD00BF13
:1078E000800400208AFC00081C000020681300208F
:1078F000A4FC00081A000020D00F0020C8FC0008DB
:1079000019000020800E0020FDFC00081800002057
:107910005409002018FD00085EFD00081B0000202F
:107920002A0E0020E410002077FD0008BC0800208B
:10793000F0B51E4690F80A31A5B073B3E023ADF858
:107940000C30F32303248DF80E30E31EDBB2CF5C42
:10795000651C24ABEDB223441FB103F8847C2C4694
:10796000F3E7111203F8841C012124AB1D4405F830
:10797000842CA21CD2B21A44331202F8843C221D79
:107980000334D3B2E4B224AA144404F8846C03AAE6
:1079900000918DF80D3000F03FF925B0F0BDF0B545
:1079A00090F80A41A5B0BDF9A860002C3CD0E024B5
:1079B000ADF80C40F4248DF80E400324E51EEDB222
:1079C00011F805C024AF651CEDB22744BCF1000FCF
:1079D00003D007F884CC2C46F0E7111207F8841C7A
:1079E00024A90D4405F8842CA21CD2B20A44191211
:1079F00002F8841CE21C24A9D2B20A4402F8843C96
:107A0000231DDBB20B44321203F8842CA31D053472
:107A1000E4B20C44012104F8846CDBB2009103AAA7
:107A20008DF80D3000F0F8F825B0F0BDF0B590F805
:107A30000A41A5B0BDF9A870BDF9AC60002C49D0D1
:107A4000E024ADF80C40F5248DF80E400324E51E2B
:107A5000EDB211F805E00DF1900C651CEDB2A444F7
:107A6000BEF1000F03D00CF884EC2C46EFE71112A6
:107A70000CF8841C24A90D4405F8842CA21CD2B255
:107A80000A44191202F8841CE21C24A9D2B20A4446
:107A900002F8843C231DDBB20B443A1203F8842C19
:107AA000631DDBB20B4403F8847CA31DDBB20B44E3
:107AB000321203F8842C04F108030734E4B20C44B6
:107AC000012104F8846CDBB2009103AA8DF80D301B
:107AD00000F0A2F825B0F0BD002310B503810446E4
:107AE0004381018043600373084603F0A0F860609F
:107AF000204610BD002303814381037370474189F1
:107B0000038902889BB28B4205D1037B002B0CBFFB
:107B100010460020704743890189994287BF038935
:107B200040894389008986BF8018C01A181A80B21C
:107B3000904288BF00207047428903899BB29342DC
:107B400005D1027B02F0FF0382B1008870474389B0
:107B500002899A429DBF42890389008803898BBFAD
:107B60004089C018181A801A80B2704718467047AA
:107B7000037B10B503F0FF02B3B9038944689BB2DD
:107B8000E1540389018801339BB20381038999423F
:107B900098BF0281028943899BB293424FF001034F
:107BA00000D10373184600E0002010BD43894268ED
:107BB0009BB2D05C704710B54289416892B20346CF
:107BC000885C002119735A891C88013292B25A814B
:107BD0005A89C0B2944298BF598110BD012902D17F
:107BE000014801F03BBB704708140020012902D175
:107BF000024801F093BA0020704700BF081400202B
:107C0000012908B504D1034801F099FAC0B208BDB2
:107C10000020FCE70814002010B5012910469DF84B
:107C200008400AD101461A46044801F03BFB24B142
:107C3000BDE81040014801F065BB10BD08140020EC
:107C400010B50346144609B9002010BD12F1090F02
:107C500008DA0A22013994FBF2F2FFF7F1FF03463A
:107C60000028F1D00A2194FBF1F2184601FB1242E0
:107C7000C2F1300200F8012BE7E70000014B185C6D
:107C8000704700BF71FE0008034AC3B2000AD35C0C
:107C9000105C1844C0B2704771FE0008074AC3B2B6
:107CA000C0F30721515CD35C0B44C0F30741515C26
:107CB000000E105C0B441844C0B2704771FE0008FF
:107CC0000F4A10B5C3B2C0F30724145DD35C23443C
:107CD000C0F30744145D000E105C23441844CBB27B
:107CE000D35C1844C1F30723D35C1844C1F30743A2
:107CF000D35C090E1844535C1844C0B210BD00BFD9
:107D000071FE000810B5044611B90024204610BDCC
:107D100052420139FFF794FF0028F6D00023037088
:107D2000F4E730B5002400250023C0E902450370C4
:107D300000F1100200F18B0102F8013B9142FBD1EE
:107D4000C0F8903000F11103C0F88C3030BD30B570
:107D50000023002400250370C0E90245C0F89030DC
:107D600030BD000010B5D0E90232DB1804465241A4
:107D700019BBC4E902321348A368217B584081F043
:107D8000D401FFF79DFF02281AD80F490F48FFF7CB
:107D900023F800230E4A12F8010BD4F88C10C854B3
:107DA0000133052BF7D101210A4B2170C4F8903023
:107DB0000948BDE81040FDF7ADB943F00103D8E72D
:107DC00010BD00BF4D63C971BEFF0008C411002083
:107DD00079FF000828000200BC08002010B5084800
:107DE0000C46FAF753FA030A84F87A0084F87930DB
:107DF0002146BDE810407B220248FEF71FBE00BFAF
:107E0000BC080020C411002070B50446D0E902323D
:107E1000DB185241C0E90232B0F89020344ED01045
:107E200002F00702D4F88C50B25C00295BD043F01A
:107E30000103A3602B5C1A432A54B4F89030013339
:107E40009BB2B3F5707FA4F8903002D92046FFF7BB
:107E50007EFFB4F89030263B042B15D8A368217B15
:107E6000244881F0D4015840FFF72AFF04280BD89A
:107E7000B4F890202049283A12B22048FFF7C9FAF6
:107E80001F4BC4F8903070BDB4F89030B3F5707FDC
:107E9000F9D1B4F89250013DADB2A4F892507DB939
:107EA00018491648FEF798FF29461748FDF732F99A
:107EB0001248FEF7F1FD2046BDE87040FFF747BFCE
:107EC00026466B1E5D425D4106F8105F3146204636
:107ED000FFF784FF7B220021304603F0C1FF00231F
:107EE000A4F89030CFE72B5C23EA0202A4E700BF9E
:107EF00071FF00084D63C9717EFF0008C4110020A6
:107F0000280002009DFF0008BC08002003780BB980
:107F1000FFF728BFFFF778BF10B540F2DC510446E9
:107F2000FFF7DAFD002304F1100204F1920102F8D8
:107F3000013B9142FBD14FF47002A4F89230C4F897
:107F4000942084F89830204610BD792A70B50646F2
:107F50000C460ED1FFF7D3FD77280CD904F1780534
:107F600014F8011F3046FFF703FEAC42F8D10020A1
:107F700070BD0420FCE70520FAE7000073B50D464C
:107F80000824094EEB098DF80730012200230DF17A
:107F900007013046013CFCF70DFE6D0014F0FF04B4
:107FA000EDB2EFD102B070BDBC08002070B5044640
:107FB000FFF7C2FDB4F8923018BB0BB32448FCF7AE
:107FC0001DFE0546082D1BD9B4F8943094F898107E
:107FD0005A1C92B2A4F89420B9B377212046FFF737
:107FE000CDFFB4F89420B4F89230083D9A42ADB277
:107FF000E8D30023A4F89430A4F8923084F89830A1
:1080000070BD002BDAD1134A127862B9012384F8CB
:108010009830B4F89630A4F892300023A4F8943045
:10802000B4F89230C9E7782584F89830B4F89260B3
:108030002046731CA4F89230FFF7BDFD013D264495
:1080400015F0FF053074F1D1E7E72344197CC5E74B
:10805000BC0800202B0E002001EB4101890001F536
:108060001671A0F89610704708B5FFF748FD782301
:10807000B0FBF3F080B208BD40F0BF60024B40F4AB
:108080000030D860704700BF00ED00E070B50125FA
:10809000017801F01F039D40C3784C09C3B10F4B19
:1080A000DA684378D243C2F30222C2F1040603FA2B
:1080B00006F683780F2020FA02F213403343084A71
:1080C0001B01DBB2114481F8003342F8245070BD2B
:1080D000034B203443F82450F9E700BF00ED00E0E3
:1080E00000E100E021F0604121F07F01014B0143FC
:1080F0009960704700ED00E0054B19B11969014323
:10810000196170471A6922EA00021A61704700BFBC
:1081100000ED00E0044B04281A680CBF42F0040292
:1081200022F004021A60704710E000E00022044BC5
:108130001A605A609A60DA60024A5A61704700BF5A
:1081400000040140FFFF0F00027930B58379056814
:1081500002F1804202F58232E9431BB3134B1C68E3
:108160000C401C605C682140596011682943116013
:1081700002689C68D1430C409C60DC682140D96057
:108180004179102906D1996811439960D9680A4349
:10819000DA6030BD01F1804303F5823319680A4388
:1081A0001A60F6E713680B401360F2E70004014021
:1081B00000234FF4406203608280837170470000A7
:1081C000024A136918431061704700BF0004014060
:1081D000034B5B69034214BF01200020704700BFBE
:1081E00000040140014B5861704700BF000401408A
:1081F000054B1A685B69034004D0024214BF01209A
:10820000002070471846704700040140014B586138
:10821000704700BF0004014008B5264B984209D1C1
:108220000121042000F052FC00210420BDE8084098
:1082300000F04CBC204B984206D10121082000F0F0
:1082400045FC00210820F1E71C4B984206D1012192
:10825000102000F03BFC00211020E7E7184B98426B
:1082600006D10121202000F031FC00212020DDE793
:10827000144B984206D10121402000F027FC002138
:108280004020D3E7104B984206D10121802000F016
:108290001DFC00218020C9E70C4B984208D1012128
:1082A0004FF4807000F012FC00214FF48070BDE7A5
:1082B00008BD00BF00080140000C01400010014053
:1082C0000014014000180140001C01400020014042
:1082D000012108B5084600F0F9FBBDE8084000217F
:1082E000012000F0F3BBCB782DE9F041DA0648BF5E
:1082F0008A780E8803F00F0548BF154316F0FF0F6C
:108300001AD000214FF0010C4FF00F0E02680CFA4A
:1083100001F737EA06040BD18C000EFA04F822EAC2
:10832000080205FA04F4282B42EA040224D147612A
:1083300001310829EBD10260FF2E1BD908244FF030
:10834000010C4FF00F0E41680CFA04F737EA0602F1
:108350000CD1A200203A0EFA02F821EA080105FA2F
:1083600002F2282B41EA02010AD147610134102CA4
:10837000EAD14160BDE8F081482B08BF0761D7E72B
:10838000482B08BF0761F1E74FF6FF73038040F207
:108390000243438070478368194214BF01200020C4
:1083A0007047806880B27047C368194214BF0120CB
:1083B00000207047C06880B270470161704741611A
:1083C00070470AB10161704741617047C1607047F1
:1083D00041F480338361816183618369836970477C
:1083E000054A136823F07F031B041B0C194341EA61
:1083F00000111160704700BF00000140014B186080
:10840000704700BF1C0020420028164A30B500F417
:108410004015B4BFD3695368B5F5401F84B210D17D
:10842000556823F0706325F07065556019B1420DF1
:108430001201944023430B4A0028B4BFD361536018
:1084400030BDC2024DBF0322420D1201C0F30345ED
:108450004CBFAA4004FA02F223EA020343F070631D
:10846000E4E700BF0000014010B50F2401F0030352
:1084700001F0FC0101F1804101F580318A689B0027
:108480009C4022EA04028A608A689840104388600F
:1084900010BD0000014B1860704700BFDC00204297
:1084A00008B50B4B012198420AD14FF4001000F09F
:1084B0001BFB00214FF40010BDE8084000F014BB86
:1084C0004FF4800000F010FB00214FF48000F3E730
:1084D0000054004070B586B00446868801A80D4659
:1084E00000F086FA039A2B4926F03F06B2FBF1F121
:1084F0003604360C88B20643A6802388264E23F025
:1085000001031B041B0C23802B68B3421ED85B00A5
:10851000B2FBF3F39BB2042B38BF0423013080B2CB
:108520002084A3832388AA8843F00103238023881F
:10853000698923F481630A4323F0020313432380F0
:108540002A89AB891343238106B070BD4BF6FF70B7
:10855000EE8886421BBF1920434303EB4303B2FB63
:10856000F3F30BBFB2FBF3F39BB29BB243F4804334
:10857000C3F30B020AB943F001034FF496724A4366
:108580004FF47A71B2FBF1F2013292B243F400433C
:108590002284C6E740420F00A086010041F28832E3
:1085A000044BC0E90023002383604FF480438381A0
:1085B000704700BF0000FFBF038819B143F00103FB
:1085C0000380704723F001031B041B0CF8E783882A
:1085D00019B143F400638380704723F400631B04E4
:1085E0001B0CF8E7838819B143F4805383807047EC
:1085F00023F480531B041B0CF8E7038819B143F4E0
:1086000080730380704723F480731B041B0CF8E70E
:10861000038819B143F400730380704723F4007397
:108620001B041B0CF8E7038819B143F48063038033
:10863000704723F480631B041B0CF8E7838901F067
:10864000FE019BB223F0FE030B43838170478389B5
:1086500019B143F001038381704723F001031B0428
:108660001B0CF8E7038819B143F0400303807047FF
:1086700023F040031B041B0CF8E7838812B1194355
:108680008180704723EA0101FAE701827047008A7E
:10869000C0B2704722B141F0010189B20182704736
:1086A00001F0FE01F9E7002382B001930190019BE4
:1086B00019440191019B188802B07047038819B1D1
:1086C00043F4004303807047C3F30E03FAE70388C3
:1086D000B1F5006F1BBF23F400631B0443F4006378
:1086E0001B0C038070470388B1F5005F1BBF23F4A8
:1086F00000531B0443F400531B0C03807047038892
:1087000019B143F480530380704723F480531B0452
:108710001B0CF8E7FFF7DBBF038819B143F0200318
:108720000380704723F020031B041B0CF8E7008B29
:10873000000A7047038819B143F0100303807047A3
:1087400023F010031B041B0CF8E7038819B943F04E
:1087500080030380704723F080031B041B0CF8E7A1
:10876000838BB1F5804F1DBF23F480431B041B0C8A
:1087700043F4804383837047838A008B43EA00433A
:108780000B4023F07F435B1A584258417047838A5D
:10879000008B43EA004020F07F407047002382B006
:1087A000009301930B0F01900093009B21F07F41F8
:1087B00053B1019B14330193019B1B680B4214BFFF
:1087C0000120002002B07047019B090C1833F2E72A
:1087D000C94389B2818270478388808A9BB20840EE
:1087E00006D003EA114313F4E06F14BF0120002008
:1087F0007047C94389B2818270470000014B1860FD
:10880000704700BF00300040014B5860704700BF08
:1088100000300040014B9860704700BF00300040BE
:108820004AF6AA22014B1A60704700BF0030004090
:108830004CF6CC42014B1A60704700BF003000403C
:10884000034BDB68184214BF01200020704700BFB3
:10885000003000400D4B1A6842F001021A6059685E
:108860000B4A0A405A601A6822F0847222F480325D
:108870001A601A6822F480221A605A6822F4FE02F2
:108880005A604FF41F029A60704700BF0010024008
:108890000000FFF80C4BB0F5803F1A6822F48032DC
:1088A0001A601A6822F480221A6003D0B0F5802F73
:1088B00005D070471A6842F480321A6070471A680F
:1088C00042F4A022F9E700BF00100240034A1368F7
:1088D00023F0F80343EAC000106070470010024024
:1088E000014B1860704700BF00004242034A5368C2
:1088F00023F47C1319430143516070470010024078
:10890000014B1860704700BF60004242034A536841
:1089100023F0030318435060704700BF001002406B
:10892000024B586800F00C00704700BF0010024076
:10893000034A536823F0F00318435060704700BFA8
:1089400000100240034A536823F4E0631843506068
:10895000704700BF00100240034A536823F460537D
:1089600043EAC0005060704700100240054B19B147
:1089700019780143197070471A7822EA00021A70B8
:10898000704700BF09100240014B1860704700BFDC
:10899000D8004242034A536823F4404318435060CE
:1089A000704700BF001002400022064B01281A70D9
:1089B0001A7002D0042802D0704718707047052240
:1089C0001A70704720100240014B1860704700BFBA
:1089D00080044242024A136A18431062704700BF83
:1089E00000100240014B1860704700BF3C04424237
:1089F0001C4A10B5536803F00C03042B01D0082B5C
:108A00001FD0194B03605368184CC3F30313E15C88
:108A10000368CB4043605168C1F30221615C23FAD3
:108A200001F181605168C1F3C221615CCB40C36038
:108A300052680F49C2F381328A5CB3FBF2F30361DF
:108A400010BD53685168C3F38343CC0303F10203A1
:108A500002D408494B43D5E751688903F9D4024948
:108A6000F8E700BF0010024000127A002100002049
:108A70001D00002000093D00054B19B15969014353
:108A8000596170475A6922EA00025A61704700BF73
:108A900000100240054B19B1996901439961704773
:108AA0009A6922EA00029A61704700BF00100240F2
:108AB000054B19B1D9690143D9617047DA6922EAD6
:108AC0000002DA61704700BF00100240054B19B187
:108AD000D9680143D9607047DA6822EA0002DA6097
:108AE000704700BF00100240054B19B119690143DE
:108AF000196170471A6922EA00021A61704700BFC3
:108B000000100240014B1860704700BF4004424211
:108B1000014B1860704700BF4C004242014B187077
:108B2000704700BF071002404209012A074B07D1D6
:108B30001B6800F01F0023FA00F000F001007047EE
:108B4000022A0CBF1B6A5B6AF3E700BF00100240F9
:108B5000002307B501933120FFF7E6FF019B0133A6
:108B60000193019BB3F5A06F01D00028F3D0312011
:108B7000FFF7DAFF003018BF012003B05DF804FBF7
:108B8000024A536A43F080735362704700100240F8
:108B9000034B9B68184214BF01200020704700BFA0
:108BA00000100240014B1870704700BF0A100240CD
:108BB00008B5214B98420BD101214FF48040FFF7BB
:108BC00085FFBDE8084000214FF48040FFF77EBFDD
:108BD0001A4B98420BD101214FF40030FFF784FF6C
:108BE00000214FF40030BDE80840FFF77DBF144B73
:108BF000984208D101214FF48020FFF775FF002132
:108C00004FF48020EFE70F4B984208D101214FF439
:108C10000020FFF769FF00214FF40020E3E70A4B33
:108C2000984208D101214FF48010FFF75DFF002129
:108C30004FF48010D7E708BD0038014000440040E1
:108C400000480040004C00400050004030B50D4648
:108C50000446038A8A899BB2C98823F440530B4394
:108C600003828389A98823F4B05323F00C030B43B8
:108C7000298987B00B4369890B438381838A9BB21F
:108C800023F440731343838201A8FFF7B1FEDDE9AB
:108C90000313154A944208BF19461923A2894B436E
:108CA000296810044CBF49008900B3FBF1F1642529
:108CB000B1FBF5F3A2891801120405FB13130BD5C0
:108CC000DA003232B2FBF5F202F0070242EA0003A8
:108CD0009BB2238107B030BD1B013233B3FBF5F3E8
:108CE00003F00F030343F3E7003801404FF416523B
:108CF0000023C0E900234FF4402283818260704743
:108D00000B8810B54C88028A23438C88C98892B29C
:108D100023430B4322F470621343038210BD0023EC
:108D2000038043808380C3807047838919B143F4F3
:108D300000538381704723F400531B041B0CF8E796
:108D400001F01F0310B5C1F342140121012C01FAF7
:108D500003F105D10C3003683AB11943016010BD2D
:108D6000022C0CBF10301430F5E723EA0101F5E7BF
:108D7000838A12B119438182704723EA0101FAE71D
:108D8000038A23F00F031B041B0C0382038A19437D
:108D900001827047838923F400631B041B0C8381C9
:108DA0008389194381817047838919B143F0020394
:108DB0008381704723F002031B041B0CF8E7038A2E
:108DC00023F020031B041B0C0382038A1943018236
:108DD0007047038A19B143F480430382704723F438
:108DE00080431B041B0CF8E7C1F308018180704726
:108DF0008088C0F308007047838943F001038381B2
:108E00007047038BDBB20383038B43EA01210183A9
:108E10007047038B03F47F430383038B1943018360
:108E20007047838A19B143F020038382704723F08F
:108E300020031B041B0CF8E7838A19B143F01003CD
:108E40008382704723F010031B041B0CF8E7838A0E
:108E500019B143F008038382704723F008031B0411
:108E60001B0CF8E7838919B143F4004383817047F1
:108E7000C3F30E03FAE7838A19B143F400638382D4
:108E8000704723F400631B041B0CF8E7838A23F06C
:108E900004031B041B0C8382838A1943818270475D
:108EA000838A19B143F002038382704723F00203DF
:108EB0001B041B0CF8E70388194214BF0120002093
:108EC0007047C94389B2018070470123C1F3421240
:108ED00010B5012A01F01F0403FA04F30DD18289B1
:108EE0001340028892B26BB10123090A03FA01F11F
:108EF0000A4214BF1846002010BD022A0CBF028A85
:108F0000828AEDE71846F7E70123090A8B40DB4325
:108F10009BB2038070470000364B82B01A6842F063
:108F200001021A605968344A0A405A601A6822F0ED
:108F3000847222F480321A601A6822F480221A6045
:108F40005A6822F4FE025A604FF41F029A6000220F
:108F5000009201921A6842F480321A601A6802F490
:108F600000320192009A01320092019A1AB9009AD5
:108F7000B2F5A06FF2D11A6812F4003218BF0122C4
:108F80000192019A012A30D11C4A116841F0100166
:108F90001160116821F003011160116841F00201B4
:108FA00011605A685A605A685A605A6842F480627E
:108FB0005A605A6822F47C125A605A6842F4E812E5
:108FC0005A601A6842F080721A601A689201FCD5E1
:108FD0005A6822F003025A605A6842F002025A604C
:108FE0005A6802F00C02082AFAD1054B054A9A6029
:108FF00002B07047001002400000FFF8002002405D
:1090000000ED00E000200008114B12495A6802F000
:109010000C02042A01D0082A0AD00F4A0A605B68B1
:109020000E4AC3F30313D25C0B68D3400B60704746
:109030005A685868C2F38342C00302F1020202D4A4
:1090400007484243EAE758688003F9D40248F8E742
:10905000001002404400002000127A00310000207D
:1090600000093D0038B504460D46AC4200D338BD7A
:1090700054F8043B9847F8E7FEE7000008B5104AAB
:10908000104B11498B4216D3144815494FF000027A
:109090008842B8BF40F8042BFADBFFF73DFF0B49CD
:1090A0000B48FFF7DFFF0B490B48FFF7DBFFBDE87D
:1090B0000840FCF7F1BC52F8040B43F8040BE1E75D
:1090C000A0000108000000208401002084000108A5
:1090D0008400010890000108840001088801002034
:1090E00074160020002382B0094A0193019B934229
:1090F00003D8019B01330193F8E70649064BCA6880
:1091000002F4E0621343CB60BFF34F8FFEE700BF72
:109110009F86010000ED00E00400FA0500F016BD96
:1091200007B501210DF1070000F032FD012814BF41
:109130004FF0FF309DF8070003B05DF804FB07B562
:1091400001210DF1070000F03FFD20B19DF807005F
:1091500003B05DF804FB4FF0FF30F9E70B7810B572
:10916000222B2DD1174C00F07BFD2378032B07D841
:10917000DFE803F01D021D22002808BF0223237030
:1091800000F08AFDB0F5966F1AD12378022B17D123
:1091900045F25550FFF732FB0020FFF735FB0A2060
:1091A000FFF738FBFFF744FBFFF73AFBFEE7002829
:1091B00014BF01230323E2E7002818BF0123DEE7E1
:1091C00010BD00BF041400201E4B73B51A78022A8C
:1091D00035D103221A7000F0B9FC03282FD900F012
:1091E000B5FC0422011F0DEB020000F007FD9DF805
:1091F0000430312B23D19DF80530452B1FD19DF82C
:109200000630412B1BD19DF80730462B17D10E4B52
:109210000E4C43F001036FF006054FF0C2462046A6
:1092200085464FF001001946324604B402B401B439
:1092300001B401B401B401B401B4AE46704702B048
:1092400070BD00BF04140020E59000080008002055
:10925000014B0360704700BFE0FF000808B54FF402
:109260008061064800F026FC0549012000F014FC4E
:10927000BDE808400349022000F00EBC000C01408C
:10928000C99100085D91000808B54FF48061044859
:1092900000F038FCBDE808400021032000F0FCBBD2
:1092A000000C014070B516460D4669B1074B1B68AE
:1092B0001B7B052B08D10024A64205D9311B281998
:1092C00000F03FFC0444F7E7002070BD4800002098
:1092D00007B501228DF807100DF10701FFF7E2FF36
:1092E000002003B05DF804FB70B50E46154600245F
:1092F000AC4205D2291B301900F066FC0444F7E7A4
:10930000204670BD13B5044600F020FC30B10122A8
:109310000DF107012046FFF7E7FFF5E702B010BDAA
:1093200008B500F029FCC0B208BD000008B5064B26
:109330001B681B7B052B05D100F092FC003018BF89
:10934000012008BD0020FCE74800002000F088BC98
:1093500000F08EBC014B024A1A60704708140020CE
:10936000E0FF000830B548F28005094C226822F47D
:10937000804222F070022A4342402260236823F494
:10938000E04323F040032B434B40236030BD00BF3C
:10939000005C0040284B072818BF18701A78052A6F
:1093A00048D8DFE802F003131E232B364FF6FB717B
:1093B000224A106C014011644FF43F4111640622AF
:1093C0001A701F4B1B685A7B1A7370474FF6FB715C
:1093D0001A4A106C014011644FF43F411164042299
:1093E00002E002225A7003221A7006E05A78013A0B
:1093F000D2B25A705A78002AF1D070470F490A6CDD
:1094000092B242F010020A6405221A700A225A70BF
:1094100070475A78013AD2B25A705A78002AECD181
:109420004FF6EF720549086C02400A64044A12685C
:10943000517B11730622D7E738160020005C0040EC
:109440004800002070B504460E464FF4000001218C
:109450001546FFF72DFB084A084B09491A60094BCE
:1094600009480B600949C4E90165086002211172CD
:109470001B68BDE870401847481600206816002099
:10948000401600206C000020B80000206416002068
:109490002DE9F0475F4E604A3368546C1B68A4B2F4
:1094A00023405D0506D56FF4806353645B4B1B68F6
:1094B0005B68984733681B682340580442BF6FF4C9
:1094C0008041554A5164990442BF6FF40051524A99
:1094D0005164DA0406D56FF4C0524F4B00205A6431
:1094E000FFF758FF30680268224013050FD54A493C
:1094F0000B6C9BB243F0080543F00C030D640B6446
:10950000037B4373032303736FF4C0534B649705CA
:1095100042BF6FF40071404B5964D50506D56FF416
:1095200080723D4B07205A64FFF734FF33681B6895
:109530001C40240407D56FF4004848F60F79364CD8
:10954000656C2B0401D4BDE8F08715F00F07C4F853
:10955000448036D148F6800327681F42F0D0BBB262
:109560002F4EDFF8C08003F440524FF4005003F058
:10957000300320213280A8F80030FFF7F3FEE80620
:1095800023680FD423F4E14323F070031B041B0C66
:10959000236000F067FF3088B8F80010BDE8F0479E
:1095A000FFF7E0BE3906EDD423F070031B051B0D59
:1095B0003A05236002D500F071FDECE700F0CEFE25
:1095C000E9E7BD0005F1804505F5B845D5F800A0EF
:1095D0001AF4004F0DD02B68326823F070031B057E
:1095E0001B0D2B60926807F18043013B52F823303A
:1095F00098471AF0800FA3D02B6807F1804703EA41
:1096000009032B603368013F5B6853F827309847A4
:1096100096E700BF48000020005C00404016002094
:109620003416002036160020800000F1804000F53E
:10963000B840036823F4804323F0700343F40043ED
:1096400043F08003594001607047000018B90722B9
:10965000024B1B681A820248704700BF6816002040
:109660001401002037B5114C2268127802F07F02F5
:10967000212A02D0022003B030BDA0F12003012B2B
:109680000B4B0C4D1B6888BF00252BB18DF80700D4
:109690000DF1070102209847002DEBD0236800242C
:1096A0009D615C822046A8472046E4E768160020BA
:1096B0000C1400204D96000813B5104B1A6813784F
:1096C00003F07F03212B17D1022806D0222811D1C5
:1096D000D3780B4A03F0030313700024094B1B6873
:1096E0002BB18DF807000DF10701022098472046A5
:1096F00002B010BD0224F1E70224F8E7681600204A
:10970000101400200C14002021B9022828BF0221C7
:10971000084670470221FBE7044B1B689B7A1BB18C
:109720000522034B1B681A73704700BF68160020A0
:10973000480000200422024B1B681A73704700BFC8
:1097400048000020054B1B68DB78032B04D8044934
:1097500001EBC30100F074BC0020704768160020C4
:10976000A0000020014900F06BBC00BF5C0000209D
:10977000014900F065BC00BF6400002037B500243B
:1097800001220D4B0D4D1B6829689C720C4B01A8E2
:109790001A644FF4E0521C645C641A644FF43F4254
:1097A0005C640A601A64074B0193FEF76FFC2B6838
:1097B0001C7303B030BD00BF6816002048000020B5
:1097C000005C0040140F0F012DE9F041194A1A4CBA
:1097D0001A4F2368116D02F23C424900555800218E
:1097E0000E46C5F3090502F5F272A94213D3144AD5
:1097F000236012689B1ADBB2BF2B04D84FF4405190
:109800000320FFF711FF0F4B1B6883B1BDE8F04148
:10981000002101201847C80757BF52F8040B300A2F
:1098200086B2C0B2F8540133DBB20131DDE7BDE8E6
:10983000F08100BF005C0040141400202C140020B4
:109840001C14002018140020F0B5204B204D214995
:109850002A681B689B1A13F0FF0305D10A78013AA6
:1098600052B20A70FAB1F0BD00240120402B28BF8B
:10987000402326460870184F1849B85C14F0010FB1
:10988000C0B218BF46EA002004F1010402F101024F
:109890000CBF86B241F8040BA342D2B2EDDCD8076C
:1098A00048BF0E602A600E4A0E49106D40000B50F2
:1098B000536823F4E04323F0400343F4004343F0B0
:1098C000800383F030035360CDE700BF24140020F1
:1098D00028140020201400202C1500208061004056
:1098E000005C00401460004070B5104A104C1368D2
:1098F00024681C1BE443E4B28C4228BF0C466CB1C4
:1099000000210C4E8DB2AC4201F1010108D8136068
:10991000094B1B781B0601D5FFF796FF204670BD4B
:10992000455DF5540133DBB2ECE700BF24140020A1
:10993000281400202C150020201400202DE9F047C9
:1099400000254FF0C00948F68F1648F280074FF007
:10995000400A434B434C1B68DFF838819D7283F803
:109960000990256523682846334043F4007323603B
:10997000236803EA08033B4383F010032360226D4E
:10998000394B520043F802A08022236D5B0003F1A3
:10999000804303F5C0431A60236823F4E24323F0B5
:1099A00070031B041B0C2360304B1B6893F82C10B6
:1099B00000F0C4FD4FF440512846FFF735FEA36880
:1099C0002946334043F4C063A360226D284B520004
:1099D00013444FF480721A60A268022002EA08025F
:1099E0003A4382F02002A260FFF71EFEE368514670
:1099F0003340E360226D1F4B520013444FF48872D2
:109A000003201A6000F09AFD4FF440510320FFF745
:109A10000BFE636829461E406660226D164B52009D
:109A200043F802906368012003EA08033B4383F094
:109A300020036360FFF7F8FD0122104B28461B68E6
:109A40001A7300F0EFFCFF220D4B1D600D4B1D60E3
:109A50000D4B1D600D4B1D600D4B1A70BDE8F0875E
:109A600068160020005C004008600040401600209E
:109A70002060004038600040106000404800002036
:109A8000141400201C14002024140020281400208A
:109A900020140020BF8FFFFFC20744BF034B196093
:109AA000830744BF024B1960704700BF18140020A1
:109AB0000C14002037B504460D4608200121FEF79E
:109AC000E9FF01A8FEF760FC41F2030301A920466B
:109AD000ADF80630ADF80450FEF705FC29462046E7
:109AE0000022FEF76EFC044B044A05491868FFF794
:109AF000A9FC03B030BD00BF48000020F8000020E2
:109B0000DC00002037B504460D46064B01A8019342
:109B1000FEF7BCFA012229462046FEF752FC03B0AC
:109B200030BD00BF140F0F0007B58DF807000121ED
:109B30000DF10700FFF7D8FE0028F8D003B05DF85C
:109B400004FB09B1FFF7D0BE08467047034B186805
:109B5000034B1B68C01AC0B2704700BF141400202A
:109B60001C140020034A13785BB2002BCCBF107882
:109B70000020704720140020034B1868034B1B681B
:109B8000C01AC0B2704700BF24140020281400205F
:109B90000A4B30B51A680A4B0A4C1B689B1ADBB299
:109BA000994228BF19460023994201DC084630BD7E
:109BB000A55C0132C554D2B20133F5E71C14002074
:109BC000141400202C14002010B5FFF7E1FF094AFF
:109BD000044613680344DBB21360074A1268D31AC1
:109BE000DBB2402B04D84FF440510320FFF71CFD9B
:109BF000204610BD1C140020141400200C4B30B55E
:109C00001B680C4C0B442468DBB2E41AE4B28D18D8
:109C1000A54288BF621A0021074C8A4201DC104627
:109C200030BDE55C01334554DBB20131F5E700BFDF
:109C30001C140020141400202C14002008B5FFF779
:109C400085FF28B1044B054A1B68D05CC0B208BD33
:109C50004FF0FF30FBE700BF1C1400202C14002045
:109C6000024B187800F00100704700BF101400206C
:109C7000024B1878C0F34000704700BF101400205A
:109C8000044B1A6802601A7902715A7942719B7901
:109C90008371704714010020014B1868704700BFA2
:109CA00014010020014B1879704700BF14010020F7
:109CB000014B5879704700BF14010020014B98797F
:109CC000704700BF1401002010B5064C18B90122DE
:109CD00023681A8210BD044B1B681B6898472068D4
:109CE0000A30F7E7681600206416002010B5064C0D
:109CF00018B9012223681A8210BD044B1B689B68A7
:109D0000984720680C30F7E768160020641600209A
:109D10001E4B10B51C68002310B90223238210BD0E
:109D20001B4803802178024611F07F0112D1617A2D
:109D30008C0644BF02230370037848064CBF43F0EF
:109D4000010323F001031370124B1B681B69984732
:109D50000F48E4E70129E2D0022915D1617901F029
:109D60000F039B0003F1804303F5B84309061B680A
:109D700005D503F03003102BE6D10123E3E703F40C
:109D80004053B3F5805FF7E71846C8E76816002030
:109D90003A160020641600202DE9F843234FDFF81F
:109DA000A0803D682C8AD4B92E7A042E17D1204980
:109DB0000B78012B0ED11F4B1A681F4B92B2134424
:109DC0005B001C6030230C70A8F800303B681E72EA
:109DD000BDE8F88310230726A8F80030F6E7AB8A21
:109DE0009C4294BF042602269C4228BF1C46AB69B5
:109DF000204698478146002000F076FD2246014625
:109E0000484600F079FB2146002000F089FD2B8AAE
:109E10004FF440521B1B2B826B8A1C443023A8F842
:109E20000030064B6C821A80D0E700BF6816002015
:109E30002C160020505C0040023000203416002018
:109E40003616002010B50A4B0A491B684978DA78A3
:109E500091420AD39C7844B9998831B99A72064BD9
:109E60001B685B689847204610BD0224FBE700BFD3
:109E7000681600209C0000206416002038B50E4AA9
:109E80000E4D12682B689269D978587990472B68E3
:109E90009A7A7AB170B91A7962B99C7854B9084B38
:109EA0001B68DB6898472B685A79DA72DA781A737C
:109EB000204638BD0224FBE740160020681600202B
:109EC0006416002070B52F4B1D682B7813F07F03AC
:109ED00005D16A7A22F020026A72184670BD022B00
:109EE0004DD16A88002AF8D12A79002AF5D16979FA
:109EF000254E21F08000840004F1804404F5B8442C
:109F0000226849B236780029B4BF02F0300202F468
:109F100040528642E1D9002ADFD0AA7A002ADCD05A
:109F20000029236811DA03F03003102B07D1C4B2E3
:109F3000204600F08CFC3021204600F07DFB134BC6
:109F40001B685B6998470023C7E703F44053B3F5E8
:109F5000805FF4D10E4D78B90E4B93F82C1000F0C1
:109F600001FD23682B409BB283F4405343F400432C
:109F700043F080032360E2E700F056FCF1E70223A0
:109F8000ABE700BF681600209C000020641600208C
:109F90008FBFFFFF6C00002038B51D4B1D4D1868AA
:109FA0002D78417921F08004A20002F1804202F56F
:109FB000B842136849B20029B4BF03F0300303F478
:109FC0004053A54221D94488FCB9F3B1837AE3B167
:109FD00013680029B5BF23F4E04323F4804323F042
:109FE000400323F07003B5BF9BB29BB283F0100314
:109FF00083F4805343F4004343F080031360064B23
:10A000001B689B699847002038BD0220FCE700BF11
:10A01000681600209C0000206416002008B5064B3E
:10A020001A68537A43F020035372044B1B68DB69B0
:10A030009847002008BD00BF681600206416002065
:10A04000054B10B51C68628A18B98B889B1A23824D
:10A0500010BD08681044FBE76816002008B50B4BDC
:10A06000002093F82C1000F07DFC094B1B68187A37
:10A07000082806D14FF48052064B1A801022064B56
:10A080001A80A0F109035842584108BD6C00002015
:10A09000681600203416002036160020F7B5974CBD
:10A0A000974E276832683B7A092B19D0954B92B2AC
:10A0B00013445B001D886D0005F1804505F5C04522
:10A0C0002B783B706B787B70A88800F0ABFD7880B4
:10A0D0002889276800F0A6FDB880AA892368DA805D
:10A0E000012223681A72DA885D78002A61D11A7811
:10A0F00012F07F024AD1092D03D1FFF7A3FE40BB26
:10A1000016E0052D20D193F90320002A07DA082351
:10A110002268137203B0BDE8F040FFF79FBF9A7842
:10A12000002AF4D19A88002AF1D19B7A002BEED133
:10A130003268754B92B2134400225B001A603022E1
:10A14000724B1A800623E3E7032D11D1DA78012A36
:10A1500008D06F4B28461B685B699847032825D1B8
:10A160000923D5E79B88002BF3D1FFF757FFC6E7FC
:10A17000012DEED1DA78012AEBD19A88002AE8D1B4
:10A180005B7A9F06E5D5FFF79DFEB8E7012A04D16B
:10A190000B2DDED1FFF772FEB1E7022AD9D1012DD6
:10A1A000F1D0032DD5D1FFF7F7FEA8E70028BFD0E7
:10A1B000ADE7062D13D11A7855065BD19B78544A2A
:10A1C000012B126803D1D369002B53D01AE0022B64
:10A1D00001D1136AF8E7032B4CD1536AF4E7002D41
:10A1E00054D15988002945D15A6822F47F42B2F5EA
:10A1F000003F3FD11A7812F07F0216D19B88002BC6
:10A2000038D1444B002522682846558293619847EF
:10A2100028464FF6FF7123681A8A8A4233D00228F3
:10A2200001D0002A55D108222EE0012A0AD1384A4D
:10A230005879126892699047E0B923689B7A002B9D
:10A24000DFD117E0022A15D15A7902F00F018B00F5
:10A25000100603F18043304803F5B8431B680078CB
:10A260004CBF03F0300303F44053884202D912F08C
:10A27000700FE4D0264B22681B6850781B69984702
:10A280000328C6D1236809221A7243E7082D04D196
:10A290001B785B06EED1214BB4E70A2DEAD11A7880
:10A2A00002F07F02012AE5D19A7A002AE2D0598889
:10A2B0000029DFD15A6822F47F42B2F5803FD9D11C
:10A2C000134A58791268926990470028D2D1144BEA
:10A2D00098E793F90010002935DAD9880C480191E4
:10A2E0000068019D90F82C00AA4284B21AD9019A04
:10A2F0001A829C82FFF750FD0CE700BF6816002011
:10A30000505C00400430002002300020361600204F
:10A3100040160020119D00089C000020C99C0008E8
:10A32000ED9C00088A42E4D2A24203D20021094AED
:10A330001170DEE7B2FBF0F100FB1122002AD8D148
:10A34000044A0121F4E703221A724FF44052024BEF
:10A350001A80DFE62C16002034160020F8B52B4EAC
:10A360003468237A022B4FD0042B4DD0032B01D01D
:10A37000052B43D1A369B3B1258A0DB3A28A9542B7
:10A3800028BF154628469847238A07465B1B238229
:10A39000638A00202B44638200F0B4FA2A46014607
:10A3A000384600F0B8F8238A53B100214FF44052E8
:10A3B000174B08461A8000F0B3FA3022154B1A806A
:10A3C000218AA38A32688B4208D803231372137A36
:10A3D00032681372BDE8F840FFF740BE09B10523AB
:10A3E000F4E7062313720C4B18680C4B80B203443D
:10A3F0005B0019603021074B1980E8E7072B03D178
:10A40000074B1B68DB6898470823E1E768160020C4
:10A410003416002036160020505C00400230002028
:10A420004016002070B5002140F60F7548F28006F6
:10A430000A4B1C78A14204D3094B40F080001860FD
:10A4400070BD8A0002F1804202F5B84213682B40C9
:10A450000B43334313600131ECE700BF9C00002045
:10A460004C5C004010B5134C23681A7A022A01D0C4
:10A47000042A09D1FFF790FC23681B7A2268137223
:10A48000BDE81040FFF7EABD062A10D15A78052A28
:10A4900009D11A78520606D1D878FFF7C3FF064BC8
:10A4A0001B681B6A9847054B1B689B6898470823E5
:10A4B000E4E700BF68160020641600204016002064
:10A4C00070470000064B074A0749136002221A72C0
:10A4D000064B074A1360074A1B681160184700BF04
:10A4E0004816002068160020B80000206C000020EC
:10A4F000401600206416002001F10051013201F5E0
:10A5000040515210490002B9704730F8023B013AFD
:10A5100021F8043BF7E7002310B501F100510132A7
:10A5200001F54051521049009A4200D110BD51F836
:10A53000234020F813400133F6E700000D4B0E4A8C
:10A540001B6D3E2903EBC0004FEA400002440AD9CC
:10A550004B09C80604BF03F1FF339BB29B0243F4CF
:10A560000043136070474B08C90748BF01339B0283
:10A57000F7E700BF005C00400C600040014B186032
:10A58000704700BF405C0040014B186880B27047C4
:10A59000405C0040014B1860704700BF445C0040C5
:10A5A000014B186880B27047445C0040014B18684A
:10A5B00080B27047485C0040014B1860704700BF94
:10A5C0004C5C0040014B186880B270474C5C004006
:10A5D0004FF6F873014A034013607047505C004027
:10A5E000014B186880B27047505C0040800000F159
:10A5F000804000F5B84001607047800000F1804065
:10A6000000F5B840006880B27047800000F18040DB
:10A6100000F5B840036823F4EC4323F070031943BA
:10A6200089B201607047800000F1804000F5B840B9
:10A63000006800F4C0607047800000F1804000F5C1
:10A64000B8400368CA0623F4E04323F040039BB2FA
:10A6500048BF83F010038A0648BF83F0200343F409
:10A66000004343F0800303607047800000F18040A6
:10A6700000F5B8400368CA0423F4804323F0700354
:10A680009BB248BF83F480538A0448BF83F40053CD
:10A6900043F4004343F0800303607047800000F1FF
:10A6A000804000F5B8400129036805D123F48053A8
:10A6B0001B041B0C036070470229FCD123F010031C
:10A6C000F6E7800000F1804000F5B840006800F037
:10A6D00030007047800000F1804000F5B84000680D
:10A6E00000F440507047800000F1804000F5B84011
:10A6F000036823F4E04323F040039BB283F030036C
:10A7000043F4004343F0800303607047800000F18E
:10A71000804000F5B840036823F4804323F07003C1
:10A720009BB283F4405343F4004343F0800303603F
:10A73000704740F60F73800000F1804000F5B8408C
:10A740000268134043F4014343F080030360704701
:10A75000800000F1804000F5B840036823F4F873EE
:10A760001B051B0D43F4004343F080030360704757
:10A77000FFF7EEBFFFF7DDBFFFF7DBBFFFF7E8BF77
:10A78000800000F1804000F5B840006800F0300023
:10A79000A0F11003584258417047800000F18040FA
:10A7A00000F5B840006800F44050A0F580535842CE
:10A7B00058417047800000F1804000F5B8400368C0
:10A7C00023F070031B051B0D03607047800000F130
:10A7D000804000F5B840036823F4E14323F07003A0
:10A7E0001B041B0C03607047800000F1804000F5E3
:10A7F000B840036823F0F0031B051B0D43F44043EE
:10A8000043F0800303607047800000F1804000F552
:10A81000B840036823F0F0031B051B0D43F400430D
:10A8200043F0C00303607047800000F1804000F5F2
:10A83000B84003685B0409D5036823F0F0031B05E7
:10A840001B0D43F4404343F08003036070478000D6
:10A8500000F1804000F5B84003685B0609D5036845
:10A8600023F0F0031B051B0D43F4004343F0C0032A
:10A8700003607047800000F1804000F5B840036835
:10A8800023F0F0031B051B0D194341F4004141F077
:10A89000800101607047800000F1804000F5B84001
:10A8A000006800F00F007047064B49081B6849001C
:10A8B0009BB203EBC00000F1005000F54050400097
:10A8C00001607047505C0040054B49081B68490017
:10A8D0009BB203EBC000034B03445B00196070475D
:10A8E000505C004004300020054B1B689BB203EB1A
:10A8F000C00000F1005000F5405040000088704753
:10A90000505C0040044B1B689BB203EBC000034B40
:10A9100003445B0018887047505C004004300020FE
:10A92000044B1B689BB203EBC000034B03445B006A
:10A9300019607047505C0040023000203E290AD95F
:10A940004B09C90604BF03F1FF339BB29B0243F4DA
:10A950000043036070474B08CA0748BF01339B029E
:10A96000F7E700000D4B0E4A1B683E299BB203EB34
:10A97000C00002444FEA42020AD94B09C80604BF8C
:10A9800003F1FF339BB29B0243F400431360704713
:10A990004B08C90748BF01339B02F7E7505C0040F2
:10A9A00006300020054B1B689BB203EBC000044B34
:10A9B00003445B001868C0F309007047505C004016
:10A9C00002300020054B1B689BB203EBC000044B18
:10A9D00003445B001868C0F309007047505C0040F6
:10A9E0000630002010B50B4CC000236849089BB20C
:10A9F000034403F1005303F540535B004900196021
:10AA0000236852089BB21844034B520003445B0076
:10AA10001A6010BD505C004004300020FFF744BFB6
:10AA2000FFF752BFFFF760BFFFF76CBF012910B5FA
:10AA30002CD1254CC00023683E2A9BB203EB0001B9
:10AA4000224B0B444FEA430119D9530912F01F0F4F
:10AA500004BF03F1FF339BB29B0243F400430B603E
:10AA600023681B499BB2184401443E2A4FEA410126
:10AA70001FD85308D20748BF01339B0222E0530876
:10AA800012F0010F18BF01339B02E8E702290FD132
:10AA90000D4CC00023689BB2C1180C4B0B445B00EB
:10AAA0001A6023689BB21844094B03445B001A6088
:10AAB00010BD5309D00604BF03F1FF339BB29B02C4
:10AAC00043F400430B60F3E7505C00400230002089
:10AAD0000630002001291BD1134B3E2A1968134B65
:10AAE00089B201EBC0010B444FEA43010AD9530973
:10AAF000D00604BF03F1FF339BB29B0243F4004333
:10AB00000B6070475308D20748BF01339B02F7E739
:10AB1000022908D1044B1B689BB203EBC000034B16
:10AB200003445B001A607047505C00400230002014
:10AB300001291BD1134B3E2A1968134B89B201EB33
:10AB4000C0010B444FEA43010AD95309D00604BFA0
:10AB500003F1FF339BB29B0243F400430B60704749
:10AB60005308D20748BF01339B02F7E7022908D1F7
:10AB7000044B1B689BB203EBC000034B03445B0018
:10AB80001A607047505C004006300020FFF70ABF93
:10AB9000FFF718BF0D49C0000B689BB2C2180C4BE1
:10ABA00013445B001B6813F47C4F0DD10B689BB200
:10ABB0001844084B03445B001B68C3F30903002BD4
:10ABC00014BF02200020704701207047505C0040F5
:10ABD000063000200230002001290FD1800000F152
:10ABE000804000F5B840036823F0F0031B051B0DFF
:10ABF00043F4004343F0C003036070470229FCD1D3
:10AC0000800000F1804000F5B840036823F0F003B5
:10AC10001B051B0D43F4404343F08003ECE741EA7E
:10AC200000207047C3B2000A40EA0320704700F0DA
:10AC300000B810B5041E08BF0124204601F000F939
:10AC400030B900F017F808B901F09AF88047F4E736
:10AC500010BD00000246BFF35B8F054B53E8000FA9
:10AC600043E800210029F9D1BFF35B8F704700BF93
:10AC700030160020024B1868BFF35B8F704700BF8F
:10AC80003016002000000000C1F30A522DE9F04107
:10AC9000A2F2FF36132E0B460D460446074631DC62
:10ACA000002E1FDB384A42FA06F808EA0102024386
:10ACB0002DD033A3D3E9002300F0AEF80022002307
:10ACC00000F0F0FC48B1002D04DA4FF4801343FA91
:10ACD00006F63544002725EA08053C462946204665
:10ACE000BDE8F08126A3D3E9002300F095F8002207
:10ACF000002300F0D7FC0028EFD0002D29DB00272F
:10AD00003D46EAE7332E06DDB6F5806F1CD01946C6
:10AD10002046BDE8F0814FF0FF38A2F2134228FA36
:10AD200002F818EA000FF2D015A3D3E9002300F0CF
:10AD300073F80022002300F0B5FC0028CDD0002DD0
:10AD400010DB27EA0807C8E7024600F065F804466A
:10AD5000DEE725F000430D4A1F43002F18BF1546BC
:10AD60000027BAE7142E08D00123C6F1340603FAEF
:10AD700006F6371928BFED18E3E70135E1E700BF14
:10AD80009C7500883CE4377EFFFF0F000000F0BF99
:10AD9000F8B520F00047FC0D7F3C162C054624DC5E
:10ADA000002C064614DB164F274138421BD01549AC
:10ADB00000F0F8FC002100F0B9FFA0B1002D04DA8A
:10ADC0004FF4000343FA04F4264426EA0700F8BDD2
:10ADD0000C4900F0E7FC002100F0A8FF18B1002D9D
:10ADE0000ADB0020F8BD2846F8BDB7F1FF4FFAD3C3
:10ADF000014600F0D7FCF8BD002FF4D00248F8BDA2
:10AE0000FFFF7F00CAF24971000080BF81F000415E
:10AE100002E000BF83F0004330B54FEA41044FEA3F
:10AE2000430594EA050F08BF90EA020F1FBF54EADA
:10AE3000000C55EA020C7FEA645C7FEA655C00F076
:10AE4000E2804FEA5454D4EB5555B8BF6D420CDD47
:10AE50002C4480EA020281EA030382EA000083EACA
:10AE6000010180EA020281EA0303362D88BF30BD6A
:10AE700011F0004F4FEA01314FF4801C4CEA1131C0
:10AE800002D0404261EB410113F0004F4FEA03331F
:10AE90004CEA133302D0524263EB430394EA050FAA
:10AEA00000F0A780A4F10104D5F1200E0DDB02FA19
:10AEB0000EFC22FA05F2801841F1000103FA0EF2AD
:10AEC000801843FA05F359410EE0A5F120050EF173
:10AED000200E012A03FA0EFC28BF4CF0020C43FAA4
:10AEE00005F3C01851EBE37101F0004507D54FF0B1
:10AEF000000EDCF1000C7EEB00006EEB0101B1F501
:10AF0000801F1BD3B1F5001F0CD349085FEA300046
:10AF10004FEA3C0C04F101044FEA445212F5800F51
:10AF200080F09A80BCF1004F08BF5FEA500C50F1EE
:10AF3000000041EB045141EA050130BD5FEA4C0CD1
:10AF4000404141EB010111F4801FA4F10104E9D15A
:10AF500091F0000F04BF01460020B1FA81F308BF51
:10AF60002033A3F10B03B3F120020CDA0C3208DD1D
:10AF700002F1140CC2F10C0201FA0CF021FA02F1F8
:10AF80000CE002F11402D8BFC2F1200C01FA02F168
:10AF900020FA0CFCDCBF41EA0C019040E41AA2BF8D
:10AFA00001EB0451294330BD6FEA04041F3C1CDA55
:10AFB0000C340EDC04F11404C4F1200220FA04F075
:10AFC00001FA02F340EA030021FA04F345EA03011F
:10AFD00030BDC4F10C04C4F1200220FA02F001FAE1
:10AFE00004F340EA0300294630BD21FA04F0294663
:10AFF00030BD94F0000F83F4801306BF81F48011FC
:10B000000134013D4EE77FEA645C18BF7FEA655C6E
:10B0100029D094EA050F08BF90EA020F05D054EA40
:10B02000000C04BF1946104630BD91EA030F1EBF45
:10B030000021002030BD5FEA545C05D14000494149
:10B0400028BF41F0004130BD14F580043CBF01F53C
:10B05000801130BD01F0004545F0FE4141F4700122
:10B060004FF0000030BD7FEA645C1ABF19461046FD
:10B070007FEA655C1CBF0B46024650EA013406BFFE
:10B0800052EA033591EA030F41F4002130BD00BFBD
:10B0900090F0000F04BF0021704730B54FF480647A
:10B0A00004F132044FF000054FF0000150E700BFFB
:10B0B00090F0000F04BF0021704730B54FF480645A
:10B0C00004F1320410F0004548BF40424FF0000147
:10B0D0003EE700BF42004FEAE2014FEA31014FEA8A
:10B0E00002701FBF12F07F4393F07F4F81F06051D9
:10B0F000704732F07F4208BF704793F07F4F04BF24
:10B1000041F40021704730B54FF4607401F0004500
:10B1100021F000411CE700BF50EA010208BF704760
:10B1200030B54FF000050AE050EA010208BF704751
:10B1300030B511F0004502D5404261EB41014FF4BA
:10B14000806404F132045FEA915C3FF4D8AE4FF0C2
:10B1500003025FEADC0C18BF03325FEADC0C18BFA5
:10B16000033202EBDC02C2F1200300FA03FC20FAF6
:10B1700002F001FA03FE40EA0E0021FA02F1144443
:10B18000BDE600BF70B54FF0FF0C4CF4E06C1CEA5C
:10B1900011541DBF1CEA135594EA0C0F95EA0C0FCD
:10B1A00000F0DEF82C4481EA030621EA4C5123EA40
:10B1B0004C5350EA013518BF52EA033541F480116F
:10B1C00043F4801338D0A0FB02CE4FF00005E1FB22
:10B1D00002E506F00042E0FB03E54FF00006E1FB6C
:10B1E00003569CF0000F18BF4EF0010EA4F1FF04AF
:10B1F000B6F5007F64F5407404D25FEA4E0E6D41EF
:10B2000046EB060642EAC62141EA55514FEAC520FF
:10B2100040EA5E504FEACE2EB4F1FD0C88BFBCF57B
:10B22000E06F1ED8BEF1004F08BF5FEA500E50F12C
:10B23000000041EB045170BD06F0004646EA0101F2
:10B2400040EA020081EA0301B4EB5C04C2BFD4EB24
:10B250000C0541EA045170BD41F480114FF0000E1D
:10B26000013C00F3AB8014F1360FDEBF002001F08B
:10B27000004170BDC4F10004203C35DA0C341BDC05
:10B2800004F11404C4F1200500FA05F320FA04F0D7
:10B2900001FA05F240EA020001F0004221F000410B
:10B2A00010EBD37021FA04F642EB06015EEA430E7E
:10B2B00008BF20EAD37070BDC4F10C04C4F12005AE
:10B2C00000FA04F320FA05F001FA04F240EA020061
:10B2D00001F0004110EBD37041F100015EEA430E32
:10B2E00008BF20EAD37070BDC4F1200500FA05F252
:10B2F0004EEA020E20FA04F301FA05F243EA0203D1
:10B3000021FA04F001F0004121FA04F220EA0200DF
:10B3100000EBD3705EEA430E08BF20EAD37070BD25
:10B3200094F0000F0FD101F00046400041EB010105
:10B3300011F4801F08BF013CF7D041EA060195F0E7
:10B34000000F18BF704703F00046520043EB0303A1
:10B3500013F4801F08BF013DF7D043EA060370478E
:10B3600094EA0C0F0CEA135518BF95EA0C0F0CD099
:10B3700050EA410618BF52EA4306D1D181EA0301DF
:10B3800001F000414FF0000070BD50EA410606BFD9
:10B390001046194652EA430619D094EA0C0F02D11E
:10B3A00050EA013613D195EA0C0F05D152EA033663
:10B3B0001CBF104619460AD181EA030101F0004181
:10B3C00041F0FE4141F470014FF0000070BD41F0CA
:10B3D000FE4141F4780170BD70B54FF0FF0C4CF4A4
:10B3E000E06C1CEA11541DBF1CEA135594EA0C0FC3
:10B3F00095EA0C0F00F0A7F8A4EB050481EA030E10
:10B4000052EA03354FEA013100F088804FEA0333F6
:10B410004FF0805545EA131343EA12634FEA0222C4
:10B4200045EA111545EA10654FEA00260EF0004185
:10B430009D4208BF964244F1FD0404F5407402D2D7
:10B440005B084FEA3202B61A65EB03055B084FEA68
:10B4500032024FF480104FF4002CB6EB020E75EB65
:10B46000030E22BFB61A754640EA0C005B084FEA8D
:10B470003202B6EB020E75EB030E22BFB61A75460A
:10B4800040EA5C005B084FEA3202B6EB020E75EB55
:10B49000030E22BFB61A754640EA9C005B084FEACD
:10B4A0003202B6EB020E75EB030E22BFB61A7546DA
:10B4B00040EADC0055EA060E18D04FEA051545EAC9
:10B4C00016754FEA06164FEAC30343EA52734FEA72
:10B4D000C2025FEA1C1CC0D111F4801F0BD141EAEB
:10B4E00000014FF000004FF0004CB6E711F4801F50
:10B4F00004BF01430020B4F1FD0C88BFBCF5E06F30
:10B500003FF6AFAEB5EB030C04BFB6EB020C5FEA3F
:10B51000500C50F1000041EB045170BD0EF0004E94
:10B520004EEA113114EB5C04C2BFD4EB0C0541EAC6
:10B53000045170BD41F480114FF0000E013C90E6C3
:10B5400045EA060E8DE60CEA135594EA0C0F08BF87
:10B5500095EA0C0F3FF43BAF94EA0C0F0AD150EA86
:10B5600001347FF434AF95EA0C0F7FF425AF104619
:10B5700019462CE795EA0C0F06D152EA03353FF441
:10B58000FDAE1046194622E750EA410618BF52EABE
:10B5900043067FF4C5AE50EA41047FF40DAF52EA92
:10B5A00043057FF4EBAE12E74FF0FF3C06E000BF2F
:10B5B0004FF0010C02E000BF4FF0010C4DF804CD3C
:10B5C0004FEA410C7FEA6C5C4FEA430C18BF7FEAFC
:10B5D0006C5C1BD001B050EA410C0CBF52EA430C2A
:10B5E00091EA030F02BF90EA020F0020704710F1AA
:10B5F000000F91EA030F58BF994208BF90422CBF39
:10B60000D8176FEAE37040F0010070474FEA410C31
:10B610007FEA6C5C02D150EA013C07D14FEA430C4F
:10B620007FEA6C5CD6D152EA033CD3D05DF8040BC0
:10B63000704700BF8446104662468C4619466346F2
:10B6400000E000BF01B5FFF7B7FF002848BF10F1C9
:10B65000000F01BD4DF808EDFFF7F4FF0CBF01200E
:10B6600000205DF808FB00BF4DF808EDFFF7EAFF8A
:10B6700034BF012000205DF808FB00BF4DF808ED45
:10B68000FFF7E0FF94BF012000205DF808FB00BF3A
:10B690004DF808EDFFF7CEFF94BF012000205DF8C4
:10B6A00008FB00BF4DF808EDFFF7C4FF34BF0120D1
:10B6B00000205DF808FB00BF4A0011D212F500120D
:10B6C00011D20DD56FF47873B3EB62520ED44FEAFA
:10B6D000C12343F0004343EA505323FA02F070477A
:10B6E0004FF00000704750EA013002D14FF0FF30B8
:10B6F00070474FF0000070474FEA4102B2F1E0435B
:10B7000024BFB3F5001CDCF1FE5C0DD901F0004C48
:10B710004FEAC0024CEA5070B2F1004F40EB830098
:10B7200008BF20F00100704711F0804F21D113F1C4
:10B730003872BCBF01F00040704741F480114FEAFD
:10B740005252C2F11802C2F1200C10FA0CF320FA86
:10B7500002F018BF40F001004FEAC1234FEAD323A3
:10B7600003FA0CFC40EA0C0023FA02F34FEA43030D
:10B77000CCE77FEA625307D150EA01331EBF4FF096
:10B78000FE4040F44000704701F0004040F0FE40B1
:10B7900040F40000704700BF80F0004002E000BFAE
:10B7A00081F0004142001FBF5FEA410392EA030FAC
:10B7B0007FEA226C7FEA236C6AD04FEA1262D2EBF6
:10B7C0001363C1BFD218414048404140B8BF5B42FB
:10B7D000192B88BF704710F0004F40F4000020F094
:10B7E0007F4018BF404211F0004F41F4000121F0AA
:10B7F0007F4118BF494292EA030F3FD0A2F10102F4
:10B8000041FA03FC10EB0C00C3F1200301FA03F131
:10B8100000F0004302D5494260EB4000B0F5000F54
:10B8200013D3B0F1807F06D340084FEA310102F113
:10B830000102FE2A51D2B1F1004F40EBC25008BFC5
:10B8400020F0010040EA03007047490040EB00008F
:10B8500010F4000FA2F10102EDD1B0FA80FCACF1BE
:10B86000080CB2EB0C0200FA0CF0AABF00EBC250BD
:10B8700052421843BCBFD0401843704792F0000FAB
:10B8800081F4000106BF80F400000132013BB5E7FE
:10B890004FEA41037FEA226C18BF7FEA236C21D074
:10B8A00092EA030F04D092F0000F08BF08467047D9
:10B8B00090EA010F1CBF0020704712F07F4F04D1A7
:10B8C000400028BF40F00040704712F100723CBFBA
:10B8D00000F50000704700F0004343F0FE4040F4E4
:10B8E000000070477FEA226216BF08467FEA2363A2
:10B8F0000146420206BF5FEA412390EA010F40F48D
:10B90000800070474FF0000304E000BF10F00043D8
:10B9100048BF40425FEA000C08BF704743F09643BF
:10B9200001464FF000001CE050EA010208BF7047DA
:10B930004FF000030AE000BF50EA010208BF704761
:10B9400011F0004302D5404261EB41015FEA010C76
:10B9500002BF84460146002043F0B64308BFA3F16E
:10B960008053A3F50003BCFA8CF2083AA3EBC25350
:10B9700010DB01FA02FC634400FA02FCC2F120026F
:10B98000BCF1004F20FA02F243EB020008BF20F0A6
:10B990000100704702F1200201FA02FCC2F120020C
:10B9A00050EA4C0021FA02F243EB020008BF20EA01
:10B9B000DC7070474FF0FF0C1CEAD0521EBF1CEA2F
:10B9C000D15392EA0C0F93EA0C0F6FD01A4480EA1D
:10B9D000010C400218BF5FEA41211ED04FF0006306
:10B9E00043EA501043EA5111A0FB01310CF0004032
:10B9F000B1F5000F3EBF490041EAD3715B0040EA58
:10BA0000010062F17F02FD2A1DD8B3F1004F40EB27
:10BA1000C25008BF20F00100704790F0000F0CF0FA
:10BA2000004C08BF49024CEA502040EA51207F3ABE
:10BA3000C2BFD2F1FF0340EAC250704740F4000099
:10BA40004FF00003013A5DDC12F1190FDCBF00F08A
:10BA500000407047C2F10002410021FA02F1C2F138
:10BA6000200200FA02FC5FEA310040F1000053EAD4
:10BA70004C0308BF20EADC70704792F0000F00F022
:10BA8000004C02BF400010F4000F013AF9D040EA28
:10BA90000C0093F0000F01F0004C02BF490011F4BC
:10BAA000000F013BF9D041EA0C018FE70CEAD153BA
:10BAB00092EA0C0F18BF93EA0C0F0AD030F0004C3A
:10BAC00018BF31F0004CD8D180EA010000F00040EE
:10BAD000704790F0000F17BF90F0004F084691F0AC
:10BAE000000F91F0004F14D092EA0C0F01D14202E6
:10BAF0000FD193EA0C0F03D14B0218BF084608D1AF
:10BB000080EA010000F0004040F0FE4040F40000F8
:10BB1000704740F0FE4040F4400070474FF0FF0C8B
:10BB20001CEAD0521EBF1CEAD15392EA0C0F93EAD2
:10BB30000C0F69D0A2EB030280EA010C49024FEA24
:10BB4000402037D04FF0805343EA111143EA1013DD
:10BB50000CF000408B4238BF5B0042F17D024FF495
:10BB6000000C8B4224BF5B1A40EA0C00B3EB510F70
:10BB700024BFA3EB510340EA5C00B3EB910F24BF59
:10BB8000A3EB910340EA9C00B3EBD10F24BFA3EBDE
:10BB9000D10340EADC001B0118BF5FEA1C1CE0D1A6
:10BBA000FD2A3FF650AF8B4240EBC25008BF20F059
:10BBB000010070470CF0004C4CEA50207F32C2BFAD
:10BBC000D2F1FF0340EAC250704740F400004FF04A
:10BBD0000003013A37E792F0000F00F0004C02BF7B
:10BBE000400010F4000F013AF9D040EA0C0093F045
:10BBF000000F01F0004C02BF490011F4000F013B9F
:10BC0000F9D041EA0C0195E70CEAD15392EA0C0F06
:10BC100008D142027FF47DAF93EA0C0F7FF470AF3E
:10BC2000084676E793EA0C0F04D14B023FF44CAF81
:10BC300008466EE730F0004C18BF31F0004CCAD116
:10BC400030F000427FF45CAF31F000437FF43CAF52
:10BC50005FE700BF4FF0FF3C06E000BF4FF0010C74
:10BC600002E000BF4FF0010C4DF804CD4FEA400256
:10BC70004FEA41037FEA226C18BF7FEA236C11D0A0
:10BC800001B052EA530C18BF90EA010F58BFB2EB53
:10BC9000030088BFC81738BF6FEAE17018BF40F0D3
:10BCA000010070477FEA226C02D15FEA402C05D187
:10BCB0007FEA236CE4D15FEA412CE1D05DF8040B0C
:10BCC000704700BF844608466146FFE70FB5FFF79F
:10BCD000C9FF002848BF10F1000F0FBD4DF808ED57
:10BCE000FFF7F4FF0CBF012000205DF808FB00BF48
:10BCF0004DF808EDFFF7EAFF34BF012000205DF8A2
:10BD000008FB00BF4DF808EDFFF7E0FF94BF0120EE
:10BD100000205DF808FB00BF4DF808EDFFF7D2FFEB
:10BD200094BF012000205DF808FB00BF4DF808ED2E
:10BD3000FFF7C8FF34BF012000205DF808FB00BFFB
:10BD400042000ED2B2F1FE4F0BD34FF09E03B3EB85
:10BD5000126209D44FEA002343F0004323FA02F0B1
:10BD600070474FF00000704712F1610F01D142029D
:10BD700002D14FF0FF3070474FF00000704700BF16
:10BD800008B5062000F00CFA012000F07DFB00BF92
:10BD9000002301461A46184600F03ABA08B5074B88
:10BDA000044613B1002100F08BFA054B1868836A32
:10BDB00003B19847204600F067FB00BFC1C20008EE
:10BDC0006800010838B50A4C0A4D641BA4100AD05B
:10BDD00004F18043013B05EB8305013C55F8043930
:10BDE0009847002CF9D1BDE8384004F045B900BFB0
:10BDF000940001089000010870B50D4E0D4D761BA2
:10BE0000B61006D00024013455F8043B9847A642EA
:10BE1000F9D1094E094D04F029F9761BB61006D068
:10BE20000024013455F8043B9847A642F9D170BD6F
:10BE300084000108840001089000010884000108C2
:10BE4000024B0146186800F0AFB800BF1C0100208B
:10BE5000024B0146186800F053B800BF1C010020D7
:10BE6000F0B4860746D0541E002A3CD0CAB203461E
:10BE700002E014F1FF3436D303F8012B9D07F8D10B
:10BE8000032C29D9CDB245EA05250F2C45EA0545F5
:10BE900033D9A4F11006360903F1200707EB061782
:10BEA00003F1100242E9045542E902551032BA4248
:10BEB000F8D1721C14F00C0F03EB021204F00F0601
:10BEC00013D0331F23F003030433134442F8045BFD
:10BED0009342FBD106F003042CB1C9B21C4403F811
:10BEE000011B9C42FBD1F0BC704734461346002C2A
:10BEF000F3D1F8E714460346C2E71A462646E0E7C0
:10BF000000293AD038B551F8043C0C1F002BB8BFBB
:10BF1000E418054600F022FA224B1A682AB1A24220
:10BF20000DD921686018824221D0626028461C60C9
:10BF3000BDE8384000F014BAA34203D81A4653684B
:10BF4000002BF9D111685018A04217D022D82168CF
:10BF50006018834203BFD3E900030918C4E9001342
:10BF6000636054602846BDE8384000F0F9B9D2E972
:10BF700000020144C4E90012D8E770472068014478
:10BF8000501883421160EDD1D3E900030144C2E9A6
:10BF90000013E7E70C2328462B60BDE8384000F08B
:10BFA000DFB900BFA4010020F8B5CD1C25F00305C2
:10BFB00008350C2D38BF0C25002D064633DBA94271
:10BFC00031D82A4F00F0CAF93A6852B113685B1BA6
:10BFD00004D43FE023685B1B29D522465468002C1B
:10BFE000F8D1796800293BD02946304600F040F866
:10BFF000431C28D0C41C24F00304A04205D0211AFD
:10C00000304600F035F801301DD02560304600F094
:10C01000A7F904F10B0020F00700231DC21A01D07C
:10C020001B1AA350F8BD0C2200203260F8BD0B2B68
:10C0300005D8A242636811D05360E7E71446236035
:10C040001C442560E2E70C233046336000F088F999
:10C050000020F8BD0B2BF1D8144653683B60D5E7A0
:10C06000304600F005F87860BEE700BFA40100206C
:10C0700038B50023064C05460846236000F0F6F963
:10C08000431C00D038BD2368002BFBD02B6038BD8B
:10C090007016002010B580210446FFF785FF60640C
:10C0A00040B10022031F7C3043F8042F8342FBD1B0
:10C0B000002010BD4FF0FF3010BD00BF436C0BB12E
:10C0C00000207047E6E700BF1F2970B5054608D875
:10C0D000436C16460C464BB153F8240043F82460D9
:10C0E00070BD16224FF0FF302A6070BDFFF7D2FFFF
:10C0F00008B96B6CF0E74FF0FF3070BD1F2938B501
:10C10000054620D8426C0C466AB152F8213053B132
:10C11000012B16D0591C10D00025204642F824507F
:10C120009847284638BD284600F070F82246014658
:10C130002846BDE8384000F055B8162301202B6092
:10C1400038BD002038BD16234FF0FF302B6038BDBE
:10C150001F2921D838B5436C05460C4683B153F8E6
:10C16000242003EB84034AB1511C10D0012A0CD0C7
:10C17000002520461D609047284638BD012038BD67
:10C18000FFF788FF28B96B6CE9E7032038BD022070
:10C1900038BD4FF0FF3038BD4FF0FF30704700BF63
:10C1A000024B01461868FFF7A9BF00BF1C01002021
:10C1B000024B0A4601461868FFF786BF1C010020A3
:10C1C000034B1868436C0BB10020704762E700BF57
:10C1D0001C010020024B01461868FFF7B9BF00BFE1
:10C1E0001C01002070B50D460023074C0646114681
:10C1F0002846236000F032F9431C00D070BD23684C
:10C20000002BFBD0336070BD7016002000F01EB90B
:10C210002DE9F041264C82B025680DB36C681F2CC7
:10C2200042DC9846064690B1D5F8880038B3D0F87D
:10C2300000310127A74047EA030C022E00EB8403DC
:10C2400040F82420C0F800C1C3F8808011D000203D
:10C25000631C02346B6045F8241002B0BDE8F08125
:10C26000144E154D2660EDB12C683546C6F8884051
:10C27000D4E7D0F804311F43C0F80471E7E70F4B4F
:10C28000CDE9001283B14FF48470FFF7D9FD58B1A6
:10C29000DDE9001200276C683B46C0E94077C5F82D
:10C2A0008800C6E73546B9E74FF0FF30D5E700BF55
:10C2B00038020020AC0100200000000041BE000850
:10C2C0002DE9F04F0F464FF0010ADFF88C8083B064
:10C2D000D8F8005001908DB16C68D5F88860013CA9
:10C2E0000CD405F1080B67B12EB106F1800353F8A9
:10C2F0002430BB4205D014F1FF34F4D203B0BDE8C2
:10C30000F08F6B685BF82420013BA34216BF00232B
:10C310006C604BF82430002AEDD0D5F80490B6B10B
:10C32000D6F800110AFA04F30B4210D0D6F8040133
:10C3300056F8241003420CD1019890476B68D8F846
:10C3400000204B4501D1AA42D5D01546C3E79047FE
:10C35000F4E708469047F1E738020020704700BF35
:10C36000704700BF38B50C460968054609B1FFF7AC
:10C37000F9FF21462846BDE83840FFF7C1BD00BFA0
:10C38000314B1B6883425AD0426A70B50546002A79
:10C3900050D0D3689BB10026995941B10C6828460A
:10C3A000FFF7AEFD2146002CF8D16B6ADB6804363E
:10C3B000802EF1D119462846FFF7A2FD6A6A11685E
:10C3C00000293DD02846FFF79BFD696911B1284639
:10C3D000FFF796FD6A6A1AB111462846FFF790FDED
:10C3E000A96B11B12846FFF78BFDE96B11B1284607
:10C3F000FFF786FD296C11B12846FFF781FDE96D35
:10C4000011B12846FFF77CFDA96D11B12846FFF751
:10C4100077FD696B11B12846FFF772FDAB696BB10F
:10C42000AB6A28469847A96C41B12846BDE87040E0
:10C43000FFF798BF41690029C9D1D1E770BD7047A6
:10C4400069690029C3D1C7E71C0100205822024BAB
:10C450004FF0FF301A607047701600205822024BD0
:10C460004FF0FF301A60704770160020044A0549EB
:10C470001368002B08BF0B4618441060184670471D
:10C480003C02002074160020FEE700BF56000000AA
:10C490003A26184D4D44564D5F4853204657206369
:10C4A0006F6E66696775726174696F6E3A00545891
:10C4B00020667265712028487A293A005258206611
:10C4C0007265712028487A293A00506F776572208A
:10C4D0007365743A00442D5374617220646576204C
:10C4E00028487A293A00444D52202B312073796D27
:10C4F000206465762028487A293A00595346202B33
:10C50000312073796D206465762028487A293A00B5
:10C51000503235202B312073796D206465762028C8
:10C52000487A293A004E58444E202B312073796DB9
:10C53000206465762028487A293A004D3137202B2F
:10C54000312073796D206465762028487A293A0075
:10C55000504F43534147206465762028487A293A52
:10C5600000804020100804020107F7D5DD57DFD016
:10C570000130000090091001700090000740017028
:10C5800000314007400150A171D1707001100000CE
:10C59000000E200000200808023815002CA01460AE
:10C5A000846D5D7F77FD757E30300110014003C0E2
:10C5B00013C11E806F00CEA8FE83ACC458200ACEE3
:10C5C000A8FE83A000000000000CC458200ACEA8DA
:10C5D000FE83ACC458200A00004F08DC028815789E
:10C5E0002CD014C084AD5D7F77FD75796524022859
:10C5F00006200F801BC107805C436F756E746572E7
:10C6000020494E54312F494E54323A004100000027
:10C61000000000B80800000042000000000080EAAE
:10C620000C000000430000000000A0EB0E00000022
:10C6300044000000000000EA0A000000450000007D
:10C64000000000800400000046000000000080AEF2
:10C650000C00000047000000000080EE0C0000000D
:10C6600048000000000000AA0A0000004900000085
:10C67000000000A0060000004A0000000000B8BB57
:10C68000100000004B000000000080EB0C000000D8
:10C690004C000000000080BA0C0000004D000000BB
:10C6A000000000EE0A0000004E000000000000E85C
:10C6B000080000004F0000000000E0EE0E00000047
:10C6C000500000000000A0BB0E0000005100000060
:10C6D0000000B8EE1000000052000000000000BA98
:10C6E0000A00000053000000000000A8080000003D
:10C6F00054000000000000E00600000055000000AB
:10C70000000000AE0A00000056000000000080ABF0
:10C710000C00000057000000000080BB0C0000006F
:10C72000580000000000E0EA0E0000005900000080
:10C730000000B8EB100000005A0000000000A0EE5E
:10C740000E000000310000000080BBBB14000000A0
:10C75000320000000000EEAE1200000033000000C6
:10C760000000B8AB10000000340000000000E0AA98
:10C770000E00000035000000000080AA0C00000040
:10C78000360000000000A0EA0E00000037000000A4
:10C790000000A8EE10000000380000000000EAEEE3
:10C7A00012000000390000000080EEEE14000000CE
:10C7B0003000000000E0EEEE160000002F00000048
:10C7C0000000E8EA100000003F0000000000EAAEB0
:10C7D000120000002C00000000E0AEEE1600000089
:10C7E0002D0000000000AEEA120000003D00000035
:10C7F0000000B8EA100000002E0000000080EBBA34
:10C8000014000000200000000000000004000000F0
:10C810000000000000000000000000008040201028
:10C82000080402014D657373616765206372656179
:10C830007465642077697468206C656E677468003D
:10C840008040201008040201444D52444D4F52587C
:10C850003A20646174612068656164657220666F66
:10C86000756E6420706F7300444D52444D4F5258A2
:10C870003A2064617461207061796C6F6164206634
:10C880006F756E6420706F7300444D52444D4F526B
:10C89000583A20766F696365206865616465722027
:10C8A000666F756E6420706F7300444D52444D4F37
:10C8B00052583A20766F6963652070692068656117
:10C8C00064657220666F756E6420706F7300444DEE
:10C8D00052444D4F52583A20766F69636520746513
:10C8E000726D696E61746F7220666F756E64207010
:10C8F0006F7300444D52444D4F52583A2063736257
:10C900006B20666F756E6420706F7300444D5244E7
:10C910004D4F52583A20766F6963652073796E6384
:10C9200020666F756E6420706F730063EA00766C2A
:10C9300076C452C878092DB87927579B31BC3EEA96
:10C9400045C330491793AE8B6DA4A5ADA2F135B5A3
:10C950003C1E00000000000001000000020000007A
:10C9600003000000040000000500000006000000B5
:10C970000700000008000000090000000A00000095
:10C980000B0000000C0000000D0000000E00000075
:10C990002040020010000000110000001200000002
:10C9A0001300000014000000150000001600000035
:10C9B0001700000018000000190000001A00000015
:10C9C0001B0000001C0000001D000000408004004F
:10C9D0008014000020000000210000002200000060
:10C9E00023000000240000002500000026000000B5
:10C9F0000840020028000000290000002A00000072
:10CA0000044002002C00000002400200014002002D
:10CA10000040020030000000310000003200000041
:10CA20008081000034000000400C0000360000004F
:10CA3000420C000038000000003004003A00000002
:10CA40000230040002290000124002000029000008
:10CA500010400200400000004100000042000000C1
:10CA600043000000440000004500000046000000B4
:10CA70004700000048000000490000004A00000094
:10CA8000002500004C0000004D0000001080040054
:10CA9000118004005000000051000000520000000E
:10CAA0000012020054000000200C00000880040066
:10CAB00009800400580000005900000004800400B0
:10CAC000058004000280040003800400008004004C
:10CAD00001800400600000006100000062000000AE
:10CAE0006300000064000000100C0000000301005F
:10CAF00000B000006800000069000000801800001D
:10CB000081180000810104008001040041400200FE
:10CB10004040020070000000040C000072000000A1
:10CB2000060C0000010C0000000C0000030C0000CB
:10CB3000020C0000045200000C0C000024800400D1
:10CB40002580040000520000080C00002080040032
:10CB500021800400800000008100000082000000AD
:10CB600083000000840000008500000086000000B3
:10CB70008700000088000000890000008A00000093
:10CB8000000205008C00000000A800001114000045
:10CB900010140000900000009100000092000000BE
:10CBA000208100009400000095000000004A000071
:10CBB000081400009800000099000000051400000F
:10CBC000041400000314000002140000011400000B
:10CBD00000140000A0000000A1000000A20000005E
:10CBE00010810000A4000000A50000000024040043
:10CBF00001240400A8000000A90000004018000063
:10CC0000411800004101040040010400814002007D
:10CC100080400200B000000002810000018100009D
:10CC200000810000B40000000681000005810000C2
:10CC300004810000010A0200000A020009810000CC
:10CC400008810000231400002214000021140000B9
:10CC500020140000C0000000C1000000C20000005D
:10CC6000C3000000C4000000C5000000C6000000B2
:10CC7000C7000000C8000000C90000002018000024
:10CC800021180000000602002001040000600100DD
:10CC900001600100D0000000D10000000128040064
:10CCA0000028040000310000008201000231000071
:10CCB00002820100D8000000D90000008480040036
:10CCC00044140000828004004214000080800400AC
:10CCD00040140000E00000000020030008180000DD
:10CCE0000046000009010400080104000C180000BF
:10CCF0000A010400021800000401040000180000EA
:10CD000001180000010104000001040004180000E3
:10CD10000201040008A400004281000041810000DB
:10CD200040810000810C0000800C0000830C00009A
:10CD3000820C000000A4000001A4000010180000F4
:10CD40001118000011010400100104001418000063
:10CD500012010400000100000101000002010000B6
:10CD600003010000040100000501000006010000AD
:10CD70000018040008010000090100000A01000079
:10CD8000402400000C0100000D0100000E01000015
:10CD900044240000100100001101000012010000F5
:10CDA000A080000014010000150100001601000021
:10CDB000A4800000180100001901000000500100CB
:10CDC0000150010022280000232800002028000034
:10CDD00021280000200100002101000022010000A4
:10CDE00090800000240100002501000040020100A5
:10CDF0004102010028010000290100002A01000071
:10CE00000441020000940000C0000400102800004B
:10CE1000004102003001000082800000818000009B
:10CE200080800000011003000010030008280000AB
:10CE300084800000062800008A800000042800008A
:10CE4000888000000228000003280000002800005D
:10CE500001280000400100004101000042010000E3
:10CE600008240000440100004501000020020100E8
:10CE700021020100480100000224000001240000FA
:10CE800000240000A1000400A0000400052400000C
:10CE90000424000050010000510100005201000074
:10CEA0001824000080300000813000008230000033
:10CEB0008330000001980000009800001124000059
:10CEC0001024000002810400049800000081040086
:10CED0000181040060010000610100000402010002
:10CEE00005020100020201008800040000020100A6
:10CEF00001020100850004008400040021240000D8
:10CF000020240000810004008000040008020100C9
:10CF10008200040002140400C28000000014040017
:10CF2000C0800000010D0000000D00001002010093
:10CF30001102010095000400940004004428000040
:10CF4000C880000091000400900004004028000008
:10CF500041280000800100008101000082010000E2
:10CF60003080000084010000004401000122020022
:10CF70000022020088010000890100008A010000EF
:10CF800038800000610004006000040063000400B9
:10CF90006200040090010000228000002180000057
:10CFA000208000004030000041300000258000005B
:10CFB00024800000000C0400010C04002980000003
:10CFC0002880000000C0020001C00200011500001E
:10CFD00000150000A0010000128000001180000078
:10CFE0001080000049000400480004001580000083
:10CFF00014800000006200004400040000040300EC
:10D0000018800000410004004000040043000400B8
:10D010004200040003800000028000000180000044
:10D0200000800000078000000680000005800000EE
:10D03000048000000B8000000A80000009800000CE
:10D040000880000051000400500004008028000007
:10D050000C800000C0010000C1010000004006007B
:10D06000014006001030000028000400008C000081
:10D07000018C00002500040024000400812400002D
:10D08000802400002100040020000400230004008C
:10D090002200040004300000053000006180000020
:10D0A000608000000030000001300000023000000D
:10D0B000033000000C3000003400040005080300B9
:10D0C00004080300083000003000040001080300D9
:10D0D000000803000D0004000C0004005180000053
:10D0E00050800000090004000800040080020100D4
:10D0F0000A000400050004000400040000190000F8
:10D100000600040001000400000004000300040005
:10D11000020004000048010042800000418000003D
:10D12000408000002030000018000400458000000E
:10D130004480000015000400140004004980000031
:10D1400048800000110004001000040013000400D7
:10D1500012000400000200000102000002020000B0
:10D1600003020000040200000502000006020000A5
:10D170000702000008020000090200000A02000085
:10D18000800005000C0200000D0200000E020000ED
:10D1900084000500100200001102000012020000CD
:10D1A0004010020014020000150200008048000038
:10D1B00081480000180200001902000001E0000090
:10D1C00000E000001C0200001D0200008848000072
:10D1D00004E0000020020000210200002202000002
:10D1E000230200002402000025020000400101008B
:10D1F0004101010028020000290200002A0200006B
:10D200000442020001240100002401000142020046
:10D210000042020030020000310200003202000031
:10D220006010020000A0020001A0020002A00200A3
:10D2300003A00200810802008008020083080200A7
:10D24000820802004050000041500000425000009F
:10D2500010420200400200004102000042020000B1
:10D2600010100200440200000060040020010100D0
:10D270002101010048020000490200004A020000AA
:10D2800018100200800402008104020082040200DF
:10D29000830402005002000002100200011002008C
:10D2A0000010020081800100808001000510020052
:10D2B00004100200002801000128010009100200EA
:10D2C00008100200205000002150000000820400DD
:10D2D00001820400600200006102000004010100FC
:10D2E000804400000201010003010100000101006F
:10D2F00001010100022006000320060000200600B4
:10D30000012006001050000011500000080101002B
:10D31000090101000C50000022100200211002003F
:10D320002010020008500000000E00001001010053
:10D3300011010100045000000550000006500000DB
:10D3400028100200005000000150000002500000B0
:10D3500003500000800200008102000082020000F1
:10D36000080005008402000085020000104800004B
:10D3700000210200880200000200050001000500F3
:10D380000000050040040200410402000500050001
:10D390000400050090020000910200000448000013
:10D3A00005480000024800004080010000480000DD
:10D3B00001480000210802002008020011000500B9
:10D3C000100005000A48000002160000084800008E
:10D3D00000160000A0020000A1020000414400006D
:10D3E00040440000A4020000A502000030480000F4
:10D3F0004444000000610000100802002100050004
:10D40000200005000461000014080200250005004A
:10D41000240005000908020008080200003001008D
:10D4200000830000224800000C0802002048000091
:10D430002148000001080200000802000308020061
:10D440000208020005080200040802002848000043
:10D4500006080200C0020000C102000021440000D2
:10D460002044000008040200108001000A040200A9
:10D4700012800100040402000504020041000500BE
:10D480004000050000040200010402000204020042
:10D4900003040200058001000480010081100200E5
:10D4A000801002000180010000800100404800005F
:10D4B00002800100140402000C80010089100200A7
:10D4C000881002001004020008800100120402000B
:10D4D0000A800100034400000244000001440000EF
:10D4E00000440000820101000644000080010100A8
:10D4F00004440000021A00000A440000001A000060
:10D50000084400002004020000030400220402007A
:10D510000203040013440000124400001144000000
:10D5200010440000218001002080010090010100D2
:10D53000228001004108020040080200101A000089
:10D54000420802008050000081500000825000001C
:10D5500083500000000300000103000002030000EC
:10D560000303000004030000050300006000010045
:10D570008020020008030000090300000088020068
:10D580000188020002440400034404000044040033
:10D59000014404001003000011030000010C01000D
:10D5A000000C0100140300001503000070000100CE
:10D5B000040C010018030000190300001088020089
:10D5C000080C010012440400000000001044040094
:10D5D0001144040020030000000406004400010080
:10D5E000450001004200010000C8000040000100A9
:10D5F0004100010080600000816000008260000046
:10D60000836000004A00010008C8000048000100D3
:10D61000490001000880050082820000818200002C
:10D62000808200005200010010C80000500001007C
:10D630005100010000800500018005000280050006
:10D6400088820000022A0000032A0000002A00004D
:10D65000012A0000400300004103000024000100F3
:10D66000250001002200010023000100200001002C
:10D6700021000100014003000040030001260000DA
:10D68000002600002A0001000440030028000100D9
:10D690002900010000C4000001C4000001110200C3
:10D6A0000011020000080600010806003000010019
:10D6B0003100010008C400001040030009110200FD
:10D6C00008110200080806000908060038000100D9
:10D6D0002084020006000100070001000400010090
:10D6E000050001000200010003000100000001002C
:10D6F000010001000E000100840204000C00010082
:10D700000D0001000A000100800204000800010071
:10D7100009000100160001001700010014000100BB
:10D7200015000100120001001300010010000100AB
:10D7300011000100045100000248040001480400E7
:10D7400000480400005100000151000018000100D1
:10D750000084020080030000810300000520020015
:10D760000420020003200200022002000120020027
:10D77000002002002060000021600000010105007F
:10D780000001050000180100011801000920020035
:10D790000820020001500400005004002182000013
:10D7A000208200000249000012200200004900000F
:10D7B00010200200306000000850040029820000A0
:10D7C000288200001018010011180100084900000B
:10D7D00018200200086000000960000011820000AB
:10D7E00010820000C200010022200200C0000100DF
:10D7F00020200200006000000160000002600000C4
:10D8000003600000046000004002040006600000A5
:10D810004202040003820000028200000182000034
:10D8200000820000078200000682000005820000DE
:10D83000048200001060000000090200098200005C
:10D840000882000002100600040902000010060011
:10D85000011006002090020021900200A4000100A7
:10D8600044200200A200010042200200A0000100AA
:10D8700040200200040502002402040005D000003C
:10D8800004D00000000502002002040001D00000C6
:10D8900000D0000004320000048101006182000019
:10D8A00060820000003200000081010002320000AE
:10D8B0000281010021140100201401000000000079
:10D8C00022140100083200000881010011D000007C
:10D8D00010D00000009002000190020084000100BE
:10D8E00000450000820001000802040080000100E1
:10D8F000810001004060000004020400426000005A
:10D900000602040001020400000204008800010075
:10D9100002020400109002004282000041820000D6
:10D9200040820000920001001802040090000100F3
:10D930009100010001140100001401000314010012
:10D9400002140100110204001002040098000100FA
:10D9500012020400000400000104000002040000A0
:10D960000304000004040000050400000604000095
:10D970000704000008040000090400000A04000075
:10D98000402100000C0400000D0400009110000074
:10D9900090100000100400001104000012040000A8
:10D9A0001304000014040000600800008910000047
:10D9B000881000001804000000800300851000009B
:10D9C000841000008310000082100000811000000D
:10D9D0008010000020040000210400002204000048
:10D9E00023040000240400005008000080200400EC
:10D9F000812004002804000029040000018804009C
:10DA0000008804000091000000220100014402008F
:10DA1000004402003004000044080000320400000A
:10DA200046080000410800004008000000C0010056
:10DA300042080000380400004C080000A510000057
:10DA4000A41000004908000048080000A1100000D0
:10DA5000A010000040040000410400004204000047
:10DA60000821000044040000300800000100070005
:10DA7000000007004804000002210000012100000E
:10DA80000021000080020200810202000521000046
:10DA9000042100005004000024080000520400008B
:10DAA00026080000210800002008000023080000CC
:10DAB0002208000002480200122100000048020073
:10DAC000102100002908000028080000008404003C
:10DAD000C010000060040000140800008142000033
:10DAE0008042000011080000100800001308000028
:10DAF000120800000040050001400500212100003F
:10DB00002021000019080000180800001B08000070
:10DB10001A080000050800000408000000110400B5
:10DB200006080000010800000008000003080000CB
:10DB30000208000080A000000C08000082A0000085
:10DB40000E08000009080000080800000B0800008B
:10DB50000A08000080040000810400008204000024
:10DB60008304000084040000004101002020040020
:10DB7000181000008804000089040000151000003F
:10DB800014100000400202001210000011100000EA
:10DB90001010000090040000910400000D1000001F
:10DBA0000C1000000B1000000A100000091000000B
:10DBB0000810000000090400061000000510000015
:10DBC000041000000310000002100000011000000B
:10DBD00000100000A0040000A104000004200400C4
:10DBE0004042000002200400032004000020040042
:10DBF00001200400020103000301030000010300EF
:10DC0000010103000A200400321000000820040073
:10DC10003010000000500200015002000185000099
:10DC200000850000C1080000C008000010200400AA
:10DC30002810000040A0000041A0000025100000B6
:10DC4000241000002310000022100000211000000A
:10DC500020100000C00400000090040021420000D9
:10DC600020420000080202000902020000890000B0
:10DC70000189000004020200050202008121000067
:10DC800080210000000202000102020002020200E4
:10DC90005010000028A00000A40800004D10000053
:10DCA0004C100000A1080000A0080000491000006E
:10DCB0004810000020A0000021A000004510000036
:10DCC0004410000010020200421000004110000049
:10DCD0004010000003420000024200000142000028
:10DCE000004200009108000090080000402004005D
:10DCF0000442000010A0000011A00000001C000061
:10DD00000842000020020200000504002202020076
:10DD10000205040008A00000840800001142000071
:10DD20001042000081080000800800008308000005
:10DD30008208000000A0000001A0000002A0000076
:10DD400003A0000004A0000088080000611000008B
:10DD50006010000000050000010500000205000041
:10DD60004820000004050000804001000605000076
:10DD70008240010008050000422000004120000010
:10DD8000402000002090000021900000004204008C
:10DD9000442000001005000011050000010A0100E8
:10DDA000000A010001A0040000A0040003A0040078
:10DDB00002A0040080080400810804005120000033
:10DDC000502000008408040082110000811100002E
:10DDD000801100002005000000020600220500005E
:10DDE0000202060008900000099000000A9000005E
:10DDF0000B900000049000000590000080000300DC
:10DE000060200000009000000190000002900000DF
:10DE100003900000421004008284000040100400BF
:10DE20008084000041090000400900004410040003
:10DE3000420900001490000015900000042C00001E
:10DE4000888400001090000011900000002C000059
:10DE5000012C0000400500000A20000009200000FD
:10DE600008200000828800000E200000808800004A
:10DE70000C20000003200000022000000120000010
:10DE80000020000007200000062000000520000000
:10DE90000420000000C2000001C2000020100400A5
:10DEA00018200000210900002009000024100400AF
:10DEB00022090000132000001220000011200000A1
:10DEC0001020000017200000162000001520000080
:10DED00014200000121004002A200000101004007A
:10DEE0002820000000600200100900000006010068
:10DEF0000106010023200000222000002120000054
:10DF00002020000040900000800404002520000034
:10DF10002420000002100400040900000010040086
:10DF200001100400010900000009000004100400B1
:10DF3000020900000A10040032200000081004004A
:10DF400030200000090900000809000001820200D9
:10DF500000820200800500000440010082050000EC
:10DF6000064001000140010000400100408800001F
:10DF70000240010010080400110804002000030002
:10DF8000C0200000094001000840010011110000FC
:10DF90001011000008080400090804002184000092
:10DFA0002084000011400100104001000911000010
:10DFB0000811000000080400010804000208040021
:10DFC0000411000004080400021100000111000007
:10DFD00000110000013800000038000008000300B4
:10DFE00010840000214001002040010000210400B5
:10DFF00001210400020003000300030000000300ED
:10E0000001000300809000004004040004000300AD
:10E010000500030003840000028400000184000066
:10E0200000840000078400000684000005840000CE
:10E0300004840000200804002108040010000300EC
:10E0400008840000240804002211000021110000AF
:10E0500020110000068800008A20000004880000CB
:10E060008820000002880000404001000088000075
:10E070000188000083200000822000008120000031
:10E080008020000000030200200404000888000033
:10E0900084200000043400000534000014880000CF
:10E0A00098200000003400000134000010880000B7
:10E0B000118800004008040041080400912000007D
:10E0C00090200000440804004211000041110000AB
:10E0D0004011000003430000024300000143000020
:10E0E0000043000009040400080404002088000024
:10E0F000218800000504040004040400400003001B
:10E10000A020000001040400000404000304040033
:10E110000204040082100400428400008010040005
:10E120004084000081090000800900008410040080
:10E130008209000000A100000012010002A10000FD
:10E14000021201001104040010040400130404006E
:10E150001204040000060000010600000206000090
:10E160000306000004060000050600000606000085
:10E170000706000008060000005800000A0600001C
:10E1800002580000C00002002020010000410400ED
:10E190000141040010060000110600000109010001
:10E1A0000009010000100500011005000210050023
:10E1B0000409010018060000105800008512000034
:10E1C0008412000008100500821200008112000075
:10E1D000801200002006000000010600C14000007F
:10E1E000C0400000092001000820010000180200C2
:10E1F0000118020005200100042001000720010091
:10E200000620010001200100002001000320010080
:10E210000220010030060000440A0000D140000046
:10E22000D0400000410A0000400A0000101802001F
:10E23000420A000015200100142001000000000027
:10E240001620010011200100102001001320010000
:10E25000122001004006000041060000A14000001D
:10E26000A040000088000200890002008A0002002D
:10E27000A44000008400020085000200009001001C
:10E2800000230000800002008100020082000200E2
:10E290008300020000C1000001C10000011402005F
:10E2A00000140200210A0000200A0000230A0000D6
:10E2B000220A000094000200950002001090010064
:10E2C0000814020090000200910002009200020077
:10E2D0002081020083400000824000008140000055
:10E2E00080400000110A0000100A00000005010033
:10E2F00084400000A40002008A4000008940000021
:10E3000088400000A000020040200100A20002009E
:10E3100042200100050A0000040A000091400000AC
:10E3200090400000010A0000000A0000030A0000FB
:10E33000020A0000045400000C0A000005810200DB
:10E340000481020000540000080A0000018102005C
:10E35000008102008006000081060000614000008C
:10E360006040000048000200490002004A0002002C
:10E370006440000044000200450002000104050062
:10E3800000040500400002004100020042000200BB
:10E3900010120000028006000380060000800600C4
:10E3A00001800600024C00000A120000004C000030
:10E3B00008120000540002000612000005120000BE
:10E3C00004120000500002000212000001120000BE
:10E3D000001200000088010042400000414000009F
:10E3E00040400000022204004640000000220400D9
:10E3F00044400000640002004A4000004940000020
:10E40000484000006000020080200100620002001D
:10E41000822001001088010052400000514000009D
:10E420005040000009C0040008C00400102204008D
:10E4300054400000010C0200000C0200030C02001A
:10E44000020C020001C0040000C004002112000000
:10E45000201200000C0002002240000021400000B9
:10E460002040000008000200090002000A0002002B
:10E470002440000004000200050002000600020023
:10E48000284000000000020001000200020002001B
:10E49000030002001C000200324000003140000076
:10E4A0003040000018000200008401001A00020041
:10E4B0000284010014000200150002001600020090
:10E4C00044120000100002001100020012000200BD
:10E4D0004012000003400000024000000140000024
:10E4E0000040000028000200064000000540000037
:10E4F00004400000240002000A400000094000001F
:10E50000084000002000020021000200220002005A
:10E510000C400000134000001240000011400000B9
:10E5200010400000810A0000800A00001540000031
:10E530001440000000A2000000110100194000007A
:10E540001840000030000200310002000008050001
:10E550000108050000070000200006001108010066
:10E56000100801000A4004002400060008400400CE
:10E570000940040006400400422200000440040058
:10E580004022000002400400034004000040040058
:10E590000140040040C00000020801000108010021
:10E5A0000008010044C00000060801000508010041
:10E5B00004080100003002000130020009080100D7
:10E5C0000808010012400400134004001040040039
:10E5D00011400400010006000000060003000600D0
:10E5E00002000600050006000400060040040100C9
:10E5F0004104010009000600080006002440040050
:10E600000A000600009200000021010020400400E2
:10E61000214004001100060010000600210801003E
:10E62000200801000370000002700000017000006B
:10E630000070000020300200180006004580020033
:10E6400044800200109200004280020041800200DB
:10E650004080020010C0000011C00000092200002C
:10E66000082200002204010023040100200401000C
:10E670002104010003220000022200000122000008
:10E6800000220000800102008101020040400400DD
:10E690000422000000C0000001C0000002C0000011
:10E6A0004008010004C0000005C0000006C00000D2
:10E6B0004408010008C0000009C000001122000049
:10E6C000102200000CC00000228002002180020005
:10E6D0002080020041000600400006000404010002
:10E6E0008041000002040100030401000004010055
:10E6F0000104010023220000222200002122000048
:10E70000202200000A040100128002000804010017
:10E710001080020020C0000021C000000012040090
:10E7200001120400010B0000000B000010040100A6
:10E7300008800200811001008010010005800200A5
:10E7400004800200038002000280020001800200B7
:10E750000080020040200500044201000524020060
:10E7600004240200014201000042010001240200D1
:10E77000002402004401020045010200844004001C
:10E78000C02200004001020041010200804004005C
:10E7900081400400080A0400820801008108010089
:10E7A00080080100114201001042010008A0010090
:10E7B00084080100000A0400010A0400020A04009F
:10E7C0000413000002A001000213000000A00100D9
:10E7D0000013000081000600800006004141000097
:10E7E000404100008500060084000600C0040100CE
:10E7F00044410000006400000164000000020300C6
:10E800000102030004640000400604000402030047
:10E810000502030003860000028600000186000056
:10E82000008600000000000006860000058600004B
:10E830000486000041100100401001001002030096
:10E8400042100100451001004410010020A0010009
:10E8500020130000002005000120050021410000D8
:10E86000204100000801020009010200008A0000A6
:10E87000018A00000401020005010200812200005B
:10E8800080220000000102000101020002010200DA
:10E890000301020080C0000081C0000082C00000AF
:10E8A0003041000084C0000008680000108A0000A9
:10E8B000118A000021100100201001002310010026
:10E8C0002210010010010200006800001201020085
:10E8D0000268000003410000024100000141000005
:10E8E0000041000082040100064100008004010094
:10E8F0000441000011100100101001000941000046
:10E90000084100002001020000060400220102006C
:10E91000020604000910010008100100002802008E
:10E92000104100000D1001000C100100042802002D
:10E93000144100000110010000100100031001004B
:10E940000210010005100100041001008180020086
:10E950008080020000008EB093E01D50A97027C097
:10E960003A90B420DC6052D04F80C1307510FBA0CB
:10E97000E6F068403670B8C0A5902B209F0011B01B
:10E980000CE08250EA1064A079F0F7404360CDD0EB
:10E99000D0805E306CD0E260FF307180C5A04B103B
:10E9A0005640D8F0B0B03E002350ADE019C097708B
:10E9B0008A2004905AA0D410C94047F0F3D07D605B
:10E9C0006030EE8086C0087015209B902FB0A100AB
:10E9D000BC5032E0D99057204A70C4C070E0FE505D
:10E9E000E3006DB005F08B40961018A0AC8022308B
:10E9F0003F60B1D0EFE061507C00F2B04690C8209B
:10EA0000D5705BC03380BD30A0602ED09AF014402A
:10EA1000091087A0B5403BF026A0A8101C309280BA
:10EA20008FD001606920E790FAC07470C0504EE04A
:10EA300053B0DD0083300D8010D09E602A40A4F0DA
:10EA4000B9A037105F50D1E0CCB04200F6207890EA
:10EA500065C0EB703DA0B310AE4020F094D01A60BA
:10EA600007308980E1C06F707220FC9048B0C6000A
:10EA7000DB5055E00BD0856098301680A2A02C109A
:10EA80003140BFF0D7B059004450CAE07EC0F070AA
:10EA9000ED2063905170DFC0C2904C20F80076B03A
:10EAA0006BE0E5508D1003A01EF090402460AAD0CA
:10EAB000B78039306700E9B0F4E07A50CE7040C0DA
:10EAC0005D90D320BB6035D02880A63012109CA06A
:10EAD00081F00F40E4306A8077D0F9604D40C3F098
:10EAE000DEA050103850B6E0ABB0250091201F904A
:10EAF00002C08C70D2405CF041A0CF107B30F5801A
:10EB0000E8D066600E2080909DC01370A75029E069
:10EB100034B0BA0088E006501B0095B02190AF20B9
:10EB2000B2703CC05480DA30C76049D0FDF0734009
:10EB30006E10E0A0BE9030202D70A3C017E0995059
:10EB400084000AB062F0EC40F1107FA0CB80453029
:10EB50005860D6D00000891112239B322446AD574D
:10EB60003665BF74488CC19D5AAFD3BE6CCAE5DB15
:10EB70007EE9F7F88110080193331A22A5562C4735
:10EB8000B7753E64C99C408DDBBF52AEEDDA64CBF5
:10EB9000FFF976E802218B30100299132667AF76D1
:10EBA0003444BD554AADC3BC588ED19F6EEBE7FAD5
:10EBB0007CC8F5D983310A2091121803A7772E66F5
:10EBC000B5543C45CBBD42ACD99E508FEFFB66EAB5
:10EBD000FDD874C904428D5316619F702004A91595
:10EBE0003227BB364CCEC5DF5EEDD7FC6888E19995
:10EBF0007AABF3BA85520C4397711E60A1142805B5
:10EC0000B3373A26CDDE44CFDFFD56ECE998608974
:10EC1000FBBB72AA06638F7214409D512225AB3450
:10EC20003006B9174EEFC7FE5CCCD5DD6AA9E3B854
:10EC3000788AF19B87730E6295501C41A3352A2474
:10EC4000B1163807CFFF46EEDDDC54CDEBB962A834
:10EC5000F99A708B088481951AA793B62CC2A5D314
:10EC60003EE1B7F04008C919522BDB3A644EED5F24
:10EC7000766DFF7C899400859BB712A6ADD224C324
:10EC8000BFF136E0C1184809D33B5A2AE55E6C4F04
:10EC9000F77D7E6C0AA583B4188691972EE3A7F2C0
:10ECA0003CC0B5D14229CB38500AD91B666FEF7EE4
:10ECB000744CFD5D8BB502A499961087AFF326E2E4
:10ECC000BDD034C1C3394A28D11A580BE77F6E6EC4
:10ECD000F55C7C4D0CC685D71EE597F42880A19184
:10ECE0003AA3B3B2444ACD5B5669DF78600CE91DA4
:10ECF000722FFB3E8DD604C79FF516E4A9902081A4
:10ED0000BBB332A2C55A4C4BD7795E68E11C680D83
:10ED1000F33F7A2E0EE787F61CC495D52AA1A3B03F
:10ED20003882B193466BCF7A5448DD59622DEB3C63
:10ED3000700EF91F8FF706E69DD414C5ABB122A063
:10ED4000B9923083C77B4E6AD5585C49E33D6A2C43
:10ED5000F11E780F7FBFDFEFF7FBFDFE8040201034
:10ED600008040201FEFDFBF7EFDFBF7F010204088C
:10ED700010204080704F934064746D302BE72D5409
:10ED80005F8A1D7FB8A7492032BA369895F316AA34
:10ED90002FC58E3FDCD32410195D1BCCCA790BD54F
:10EDA0009762C71FEE6912888CAE0D66E5BC85EAD6
:10EDB0004BB1E30FF734094446D706B372DE42F590
:10EDC000A5D8F1877B9A0422A36B8359396F000081
:10EDD000000300060009000C000F001200150018C7
:10EDE000001B001E002100240027002A002D0030F7
:10EDF000003300360039003C003F00420045004827
:10EE0000004B004E00510000010301060109010CF6
:10EE1000010F011201150118011B011E012101241E
:10EE20000127012A012D0130013301360139013C4E
:10EE3000013F014201450148014B014E01510100D2
:10EE4000020302060209020C020F02120215021846
:10EE5000021B021E022102240227022A022D023076
:10EE6000023302360239023C023F024202450248A6
:10EE7000024B024E02510200030303060309030C76
:10EE8000030F031203150318031B031E032103249E
:10EE90000327032A032D0330033303360339033CCE
:10EEA000033F034203450348034B034E0351030052
:10EEB000040304060409040C040F041204150418C6
:10EEC000041B041E042104240427042A042D0430F6
:10EED000043304360439043C043F04420445044826
:10EEE000044B044E04510400050305060509050CF6
:10EEF000050F051205150518051B051E052105241E
:10EF00000527052A052D0530053305360539053C4D
:10EF1000053F054205450548054B054E05510500D1
:10EF2000060306060609060C060F06120615061845
:10EF3000061B061E062106240627062A062D063075
:10EF4000063306360639063C063F064206450648A5
:10EF5000064B064E06510600070307060709070C75
:10EF6000070F071207150718071B071E072107249D
:10EF70000727072A072D0730073307360739073CCD
:10EF8000073F074207450748074B074E0751070150
:10EF900000040007000A000D0010001300160019FD
:10EFA000001C001F002200250028002B002E00312D
:10EFB00000340037003A003D00400043004600495D
:10EFC000004C004F0052000101040107010A010D2D
:10EFD0000110011301160119011C011F0122012555
:10EFE0000128012B012E013101340137013A013D85
:10EFF0000140014301460149014C014F0152010109
:10F0000002040207020A020D02100213021602197C
:10F01000021C021F022202250228022B022E0231AC
:10F0200002340237023A023D0240024302460249DC
:10F03000024C024F0252020103040307030A030DAC
:10F040000310031303160319031C031F03220325D4
:10F050000328032B032E033103340337033A033D04
:10F060000340034303460349034C034F0352030188
:10F0700004040407040A040D0410041304160419FC
:10F08000041C041F042204250428042B042E04312C
:10F0900004340437043A043D04400443044604495C
:10F0A000044C044F040105040507050A050D05106D
:10F0B000051305160519051C051F0522052505283C
:10F0C000052B052E053105340537053A053D05406C
:10F0D000054305460549054C054F0501060406078D
:10F0E000060A060D0610061306160619061C061F4C
:10F0F000062206250628062B062E0631063406377C
:10F10000063A063D0640064306460649064C064FAB
:10F11000060107040707070A070D0710071307165C
:10F120000719071C071F072207250728072B072E8B
:10F13000073107340737073A073D074007430746BB
:10F140000749074C074F070200050008000B000E97
:10F15000001100140017001A001D002000230026D3
:10F160000029002C002F003200350038003B003E03
:10F17000004100440047004A004D005000020105D4
:10F180000108010B010E011101140117011A011DE3
:10F190000120012301260129012C012F0132013513
:10F1A0000138013B013E014101440147014A014D43
:10F1B0000150010202050208020B020E02110214A4
:10F1C0000217021A021D0220022302260229022C23
:10F1D000022F023202350238023B023E0241024453
:10F1E0000247024A024D0250020203050308030BC4
:10F1F000030E031103140317031A031D0320032333
:10F2000003260329032C032F033203350338033B62
:10F21000033E034103440347034A034D03500302E3
:10F2200004050408040B040E041104140417041A42
:10F23000041D0420042304260429042C042F043272
:10F2400004350438043B043E044104440447044AA2
:10F25000044D0450040205050508050B050E0511B3
:10F2600005140517051A051D052005230526052982
:10F27000052C052F053205350538053B053E0541B2
:10F2800005440547054A054D0550050206050608D3
:10F29000060B060E061106140617061A061D062092
:10F2A000062306260629062C062F063206350638C2
:10F2B000063B063E064106440647064A064D0650F2
:10F2C000060207050708070B070E071107140717A3
:10F2D000071A071D0720072307260729072C072FD2
:10F2E000073207350738073B073E07410744074702
:10F2F000074A074D0750079E8D3288261A3F61E85E
:10F30000552D16445374617252583A20466F756EEB
:10F310006420656E642073796E6320696E20446199
:10F32000746100445374617252583A20646174618C
:10F330002073796E632074696D6564206F75742C19
:10F34000206C6F7374206C6F636B00445374617234
:10F3500052583A20666F756E64206672616D652042
:10F3600073796E6320696E204E6F6E652C20667512
:10F370007A7A7900445374617252583A20666F75F4
:10F380006E6420646174612073796E6320696E20FD
:10F390004E6F6E652C20657861637400804020108C
:10F3A0000804020100F734094446D706B372DE426E
:10F3B000F5A5D8F1877B9A0422A36B8359396FA1F5
:10F3C000FA52ECF8C33D4D0291D1B5C1AC9CB75097
:10F3D0007D2976FCE19E2681C8E8DA6056CE5BA8DE
:10F3E000BE143BFE704F934064746D302BE72D5478
:10F3F0005F8A1D7FB8A7492032BA369895F3060078
:10F4000004040007040B000E041200150419001C6C
:10F41000042000230427002A042D07310234053874
:10F42000003B033E064201450448074C024F0500DD
:10F4300005040107050B010E051201150519011C34
:10F44000052001230527012A052E00310334063843
:10F45000013B043E074202450549004C034F0600AC
:10F4600006040207060B020E061202150619021CFC
:10F47000062002230627022A062E0131043407380B
:10F48000023B053F004203450649014C044F07007B
:10F4900007040307070B030E071203150719031CC4
:10F4A000072003230727032A072E023105350038DA
:10F4B000033B063F014204450749024C0550000149
:10F4C00000040408000B040F001204160019041DA8
:10F4D000002004240027042B002E033106350138B8
:10F4E000043B073F024205460049034C0650010118
:10F4F00001040508010B050F011205160119051D70
:10F50000012005240127052B012E0431073502387F
:10F51000053C003F034206460149044C07500201E6
:10F5200002040608020B060F021206160219061D37
:10F53000022006240227062B022E0532003503384E
:10F54000063C013F044207460249054D00500301B5
:10F5500003040708030B070F031207160319071DFF
:10F56000032007240327072B032E06320135043816
:10F57000073C023F054300460349064D0150040184
:10F5800004050008040C000F04130016041A001DE3
:10F59000042100240428002B042E073202350539EB
:10F5A000003C033F064301460449074D0250050154
:10F5B00005050108050C010F05130116051A011DAB
:10F5C000052101240528012B052F003203350639BA
:10F5D000013C043F07430246054A004D0350060123
:10F5E00006050208060C020F06130216061A021D73
:10F5F000062102240628022B062F01320435073982
:10F60000023C054000430346064A014D04500701F1
:10F6100007050308070C030F07130316071A031D3A
:10F62000072103240728032B072F02320536003950
:10F63000033C064001430446074A024D05510002BF
:10F6400000050409000C041000130417001A041E1E
:10F65000002104250028042C002F0332063601392E
:10F66000043C074002430547004A034D065101028E
:10F6700001050509010C051001130517011A051EE6
:10F68000012105250128052C012F043207360239F6
:10F69000053D004003430647014A044D075102025D
:10F6A00002050609020C061002130617021A061EAE
:10F6B000022106250228062C022F053300360339C5
:10F6C000063D014004430747024A054E005103022C
:10F6D00003050709030C071003130717031A071E76
:10F6E000032107250328072C032F0633013604398D
:10F6F000073D024005440047034A064E01510402FB
:10F7000004060009040D001004140017041B001E59
:10F71000042200250429002C042F07330236053A61
:10F72000003D034006440147044A074E02510502CA
:10F7300005060109050D011005140117051B011E21
:10F74000052201250529012C053000330336063A30
:10F75000013D044007440247054B004E0351060299
:10F7600006060209060D021006140217061B021EE9
:10F77000062202250629022C063001330436073AF8
:10F78000023D054100440347064B014E0451070268
:10F7900007060309070D031007140317071B031EB1
:10F7A000072203250729032C073002330537003AC7
:10F7B000033D064101440447074B024E0552000336
:10F7C0000006040A000D041100140418001B041F95
:10F7D000002204260029042D003003330637013AA5
:10F7E000043D074102440548004B034E0652010305
:10F7F0000106050A010D051101140518011B051F5D
:10F80000012205260129052D013004330737023A6C
:10F81000053E004103440648014B044E07520203D3
:10F820000206060A020D061102140618021B061F24
:10F83000022206260229062D023005340037033A3B
:10F84000063E014104440748024B054F00520303A2
:10F850000306070A030D071103140718031B071FEC
:10F86000032207260329072D033006340137043A03
:10F87000073E024105450048034B064F0152040371
:10F880000407000A040E001104150018041C001FD0
:10F8900004230026042A002D043007340237053BD8
:10F8A000003E034106450148044B074F0252050341
:10F8B0000507010A050E011105150118051C011F98
:10F8C00005230126052A012D053100340337063BA7
:10F8D000013E044107450248054C004F0352060310
:10F8E0000607020A060E021106150218061C021F60
:10F8F00006230226062A022D063101340437073B6F
:10F90000023E054200450348064C014F04520703DE
:10F910000707030A070E031107150318071C031F27
:10F9200007230326072A03445374617254583A206C
:10F9300068656164657220737061636520617661DA
:10F94000696C61626C6500445374617254583A206A
:10F95000454F5420737061636520617661696C6105
:10F96000626C6500445374617254583A2064617447
:10F970006120737061636520617661696C61626C9E
:10F98000650080402010080402014D313752583A7A
:10F9900020666F756E64206C696E6B20736574757C
:10F9A000702073796E632C20706F73004D31375265
:10F9B000583A20666F756E642073747265616D20AD
:10F9C00073796E632C20706F73004D313752583A43
:10F9D00020666F756E6420656F742073796E632C7A
:10F9E00020706F73004D313752583A2073796E632F
:10F9F0002074696D6564206F75742C206C6F73744E
:10FA0000206C6F636B004D313752583A206C696E31
:10FA10006B2073657475702073796E6320666F75E3
:10FA20006E6420696E204E6F6E65004D31375258FE
:10FA30003A2073747265616D2073796E6320666F0E
:10FA4000756E6420696E204E6F6E650080402010D8
:10FA5000080402014E58444E52583A20666F756EA3
:10FA6000642073796E6320696E20446174612C2078
:10FA7000706F73004E58444E52583A2073796E633B
:10FA80002074696D6564206F75742C206C6F7374BD
:10FA9000206C6F636B004E58444E52583A20737975
:10FAA0006E6320666F756E6420696E204E6F6E65A2
:10FAB000005775FD80402010080402015575F5FFC0
:10FAC00077FF50323552583A20445549440050325D
:10FAD0003552583A20666F756E642073796E6320D4
:10FAE000696E204C44550050323552583A20737993
:10FAF0006E632074696D6564206F75742C206C6F63
:10FB00007374206C6F636B0050323552583A207317
:10FB1000796E6320666F756E6420696E204E6F6E1D
:10FB2000650050323552583A2073796E6320666F03
:10FB3000756E6420696E2048445500503235525825
:10FB40003A2073796E6320666F756E6420696E204B
:10FB50005444550050323552583A2073796E632020
:10FB6000666F756E6420696E2054534455005032A0
:10FB70003552583A2073796E6320666F756E642033
:10FB8000696E205044550050323552583A207379EE
:10FB90006E6320666F756E6420696E205444554C08
:10FBA00043005A554D73706F742D76312E362E31B9
:10FBB0002032303233313131355F575053442031A8
:10FBC000342E373435364D487A204144463730326A
:10FBD00031204657206279204341364A41552C2036
:10FBE00047344B4C582C2057304348502E204769FF
:10FBF00074494420233561356539613100526563AC
:10FC0000656976656420696E76616C6964206361FC
:10FC10006C6962726174696F6E206461746100491D
:10FC20006E76616C69642043572049642064617476
:10FC30006100526563656976656420696E76616C02
:10FC4000696420442D537461722068656164657233
:10FC500000526563656976656420696E76616C69DA
:10FC60006420442D53746172206461746100526594
:10FC700063656976656420696E76616C69642044A9
:10FC80002D5374617220454F540052656365697647
:10FC9000656420696E76616C696420444D5220640D
:10FCA00061746100526563656976656420696E768A
:10FCB000616C69642053797374656D20467573694E
:10FCC0006F6E206461746100526563656976656476
:10FCD00020696E76616C69642050323520686561F8
:10FCE00064657200526563656976656420696E7645
:10FCF000616C696420503235204C44550052656374
:10FD0000656976656420696E76616C6964204E5819
:10FD1000444E206461746100526563656976656470
:10FD200020696E76616C6964204D3137206C696E94
:10FD30006B20736574757020646174610052656333
:10FD4000656976656420696E76616C6964204D3101
:10FD5000372073747265616D20646174610052654F
:10FD600063656976656420696E76616C6964204DAF
:10FD7000313720454F5400526563656976656420CC
:10FD8000696E76616C696420504F4353414720642B
:10FD9000617461004D6F64652073657420746F2019
:10FDA000444D52004D6F64652073657420746F205C
:10FDB000442D53746172004D6F6465207365742027
:10FDC000746F2053797374656D20467573696F6E17
:10FDD000004D6F64652073657420746F2050323558
:10FDE000004D6F64652073657420746F204E584415
:10FDF0004E004D6F64652073657420746F204D3123
:10FE000037004D6F64652073657420746F20504F08
:10FE100043534147004D6F64652073657420746FD0
:10FE20002049646C65007365744D6F64653A2063A6
:10FE30006F6E6669677572696E6720486172647774
:10FE40006172650046756C6C206475706C65782015
:10FE50006E6F7420737570706F727465642077694B
:10FE600074682074686973206669726D7761726561
:10FE70000000010102010202030102020302030366
:10FE80000401020203020303040203030403040443
:10FE90000501020203020303040203030403040432
:10FEA0000502030304030404050304040504050513
:10FEB0000601020203020303040203030403040411
:10FEC00005020303040304040503040405040505F3
:10FED00006020303040304040503040405040505E2
:10FEE00006030404050405050604050506050606C3
:10FEF00007010202030203030402030304030404D0
:10FF000005020303040304040503040405040505B2
:10FF100006020303040304040503040405040505A1
:10FF20000603040405040505060405050605060682
:10FF30000702030304030404050304040504050580
:10FF40000603040405040505060405050605060662
:10FF50000703040405040505060405050605060651
:10FF60000704050506050606070506060706070732
:10FF7000088040201008040201D471C9634D595310
:10FF80004652583A20666F756E642073796E63200E
:10FF9000696E20446174612C20706F730059534660
:10FFA00052583A2073796E632074696D6564206FCE
:10FFB00075742C206C6F7374206C6F636B005953D5
:10FFC0004652583A2073796E6320666F756E6420CE
:10FFD000696E204E6F6E650000000000000000009A
:10FFE0001D910008219100083F9100080593000829
:10FFF00009024300020100C03209040000010202AC
:020000040801F1
:100000000100052400011005240103010424020657
:100010000524060001070582034000FF09040100D2
:10002000020A0000000705030240000007058102E4
:100030004000001201000202000040AF1E04000058
:1000400002010200010403090412034C006500616F
:100050000066004C006100620073000C034D0061FB
:100060000070006C0065000020010020F8B500BFA2
:10007000F8BC08BC9E467047F8B500BFF8BC08BC89
:100080009E46704775210008A55A00085593000840
:040090004D210008F6
:040094000000000068
:08009800FC20FF7F01000000C5
:1000A000000000000200000001000000010000014B
:1000B00000010101001E010101010101010204060C
:1000C00008000000000102030401020304060708FF
:1000D00009000000000000000001020304060708F8
:1000E0000900000000A24A044C00002000BF0000EC
:1000F000000000000000000000000000F0FF000809
:100100004300000033000108120000007D97000842
:100110003D990008C1A40008C1A400086596000824
:10012000B9960008099700087197000865970008BC
:100130004597000800000000400000000401000096
:1001400045000108040000004900010812000000F9
:100150005B0001080C000000C1A40008199700080A
:10016000C1A40008C1A40008C1A40008C1A40008DB
:10017000C1A40008C1A400083597000849980008E8
:10018000C1A40008C1A40008C1A40008C1A40008BB
:10019000C1A40008C1A40008C1A40008C1A40008AB
:1001A000C9970008C1A40008C1A40008C1A40008A0
:1001B000C1A4000800C201000000080020010020C6
:1001C000000000000000000000000000000000002F
:1001D000000000000000000000000000000000001F
:1001E000000000000000000000000000000000000F
:1001F00000000000000000000000000000000000FF
:1002000000000000000000000000000000000000EE
:1002100000000000000000000000000000000000DE
:04022000C1C200084F
:040000050800907DE2
:00000001FF
